:1000000000800020BD01000095A200004DA200006C
:100010004DA200004DA200004DA200004DA2000024
:100020004DA200004DA200004DA2000095A20000CC
:1000300095A200004DA2000015990000199A000039
:1000400095A2000095A2000095A2000095A20000D4
:1000500095A2000095A2000095A2000095A20000C4
:1000600095A2000095A2000095A2000095A20000B4
:1000700095A2000095A2000095A2000095A20000A4
:1000800095A2000095A2000095A2000095A2000094
:1000900095A2000095A2000095A2000095A2000084
:1000A000517E00005D7E000095A2000095A2000038
:1000B00095A2000095A2000095A2000095A2000064
:1000C00095A2000095A2000095A2000095A2000054
:1000D00095A2000095A2000095A2000095A2000044
:1000E00095A2000095A2000095A2000095A2000034
:1000F00095A2000001C3000095A200002DC40000DD
:1001000095A200006DAC000095A2000095A2000031
:1001100095A2000095A2000095A2000095A2000003
:1001200095A2000095A2000095A2000095A20000F3
:1001300095A2000095A2000095A2000095A20000E3
:1001400095A2000095A2000095A2000095A20000D3
:10015000059B0000199B00002D9B0000419B0000A7
:1001600095A2000089AF000095A2000095A20000B2
:1001700095A2000095A2000095A2000095A20000A3
:1001800095A2000095A2000095A2000095A2000093
:1001900095A2000095A2000095A2000095A2000083
:1001A00095A2000095A2000095A2000095A2000073
:1001B00095A2000095A2000095A20000564B4CF2BB
:1001C000205210B51A804DF628121A8000BF00BFC9
:1001D0000AF064F8514B4FF010621A60504A9A606E
:1001E000504ADA60504A136813F4807304D14F49BF
:1001F0000B604FF4A85313604D4B1A78110703D5C9
:100200001A7842F008021A704A4B4B492A221A7097
:100210004A4A4B4B8B4204D252F8040F43F8040B6A
:10022000F8E7484B484900228B4202D243F8042B9E
:10023000FAE74649464A002352F8230041F82300D2
:1002400001336F2BF8D1434B434A802103F8011B44
:100250009342FBD1414B3D4A1A60414B8A221A70AE
:10026000A3F5805324225A70A0221A709A7992071B
:10027000FCD59A79D406FCD43A4A937903F00C035E
:10028000082B384BF9D103221A7140225A719A79FE
:100290009006FCD5334A9179324B4906FBD5324A58
:1002A000324911600221516020221A709A7902F0BD
:1002B0000C020C2AFAD12E4B2E4A1A602E4B2F4AD2
:1002C0001A6000225A60072243F8042C2C4AC3F813
:1002D0000C2D62B60AF092FB144B1B68DA0705D5A9
:1002E00028480AF05FF9284B284A1A60284B1B78E7
:1002F0005B0609D5244C254B22689A4204D121483B
:100300000AF050F9002323600DF04AFB09F0CCFFFE
:1003100009F0FAFEFEE700BF0E20054030800440E1
:10032000823F04000100002B10D0034014D0034092
:1003300002D0074000E00740A49AFF1F64070100B5
:100340004088FF1FA49AFF1FB0A1FF1F0082FF1F5C
:100350000000000000E400E05FE400E008ED00E0E1
:100360000050064000400640448004400000030165
:1003700004800440C010050014E000E0FF76010096
:1003800000002020000F7A5E1CE00340A5C3945AB1
:1003900000F00740FFFFFFFFFFFFFFFFFFFFFFFF32
:1003A000FFFFFFFFFFFFFFFFFFFFFFFFFFFFFFFF5D
:1003B000FFFFFFFFFFFFFFFFFFFFFFFFFFFFFFFF4D
:1003C000FFFFFFFFFFFFFFFFFFFFFFFFFFFFFFFF3D
:1003D000FFFFFFFFFFFFFFFFFFFFFFFFFFFFFFFF2D
:1003E000FFFFFFFFFFFFFFFFFFFFFFFFFFFFFFFF1D
:1003F000FFFFFFFFFFFFFFFFFFFFFFFFFFFFFFFF0D
:10040000FFFFFFFFFFFFFFFFFFFFFFFFDEF9FFFF23
:1004100010B5054C237833B9044B13B10448AFF33E
:1004200000800123237010BDA49AFF1F000000006C
:1004300068070100084B10B51BB108490848AFF325
:1004400000800848036803B910BD074B002BFBD0A0
:10045000BDE81040184700BF00000000A89AFF1F29
:1004600068070100A49AFF1F0000000038B5044689
:10047000104621700A491D460DF074F801464FF0F0
:100480007E500DF023F907490DF06CF8E5606060CF
:10049000256165610AF042FAE061204638BD00BF7F
:1004A000DB0FC9400024744938B50446104621705A
:1004B00009491D460DF056F801464FF07E500DF0EB
:1004C00005F906490DF04EF8E5606060256165614B
:1004D0000AF024FAE06138BDDB0FC94000247449FA
:1004E00038B503780446032B20D8DFE803F01A1848
:1004F0001002C16840690CF02BFF0D490546606889
:100500000DF0E4F8014628460DF0E0F838BD084942
:1005100040680DF0DBF8E1680DF024F838BDC068E4
:1005200038BDC16840690CF013FF38BD002038BDEC
:100530000024744970B504460E460AF0EFF90546EA
:10054000E069281A0CF0BAFFE3682361E56166618F
:10055000A061014660680DF0B9F80146A06010483E
:100560000DF0B4F80CF08AFB0CF02AF80CF09CFEAD
:10057000054601464FF07E500CF0EAFE61690CF032
:10058000F1FF2169064628460CF0ECFF0146304693
:100590000CF0E0FEE0602046BDE87040FFF7A0BF31
:1005A000000080BF38B50E201C4C09F087FC218864
:1005B0001B4B884205461A881DDA0023511AB1F5F3
:1005C000805FAABF1B03C3EB03330131142093FBED
:1005D000F1F109F0F9FF134B1988F1B923889D4215
:1005E00010DAC3F57F630F33282091FBF3F1BDE8E8
:1005F000384009F0E9BF9042D4BFC1EB0003C1EB22
:100600000203DBE740F6FF718D42D4BFC3EB050167
:10061000C3EB0101C1EB0131E3E738BD829BFF1F52
:100620004C9CFF1F049CFF1F10B5044609F048FABC
:10063000204610BD70B44C88A04220D9012301335C
:10064000DBB21CB2660031F8144084421D46F6D37A
:10065000A04211D005F10045013D965B31F815101F
:1006600032F81530401AF21A00FB02F0641A90FBBF
:10067000F4F4E01870BC7047905B70BC70470226C1
:100680000125E5E700280CDA064A434282FB0320F5
:10069000DA17C2EB600000EB4000A3EB8000C0F172
:1006A0000C007047ABAAAA2A2DE9F0470C2009F0EC
:1006B000D1FB0C200AF086F89A4914200AF092F82F
:1006C00099499A4807F0CAF8022103200AF020F954
:1006D000022104200AF01CF9022105200AF018F971
:1006E000022106200AF014F901210A200AF010F96B
:1006F000012109200AF00CF901210D200AF008F966
:10070000012128200AF004F9012114200AF000F93F
:10071000012116200AF0FCF8172001210AF0F8F850
:1007200004200AF0E7F8002833D005200AF0E2F8A8
:100730000446002834D0002420467D4D287004F063
:10074000FBFD2D780DBB204606F0ACF8794B7A49BD
:100750001B887A4C09882170794A7A4EA3F5AF71CB
:1007600040F23A7303FB01F382FB0312DB17A3EBA6
:100770006213323301210D2033600AF0B5F85D2198
:10078000714807F015FC90B9FEE7BDE8F04706F0A8
:1007900075BF06200AF0AEF80028C6D10124CCE7C8
:1007A00003200AF0A7F8B0FA80F04009C5E75C2101
:1007B000664807F0FDFB00B9FEE75B21644807F0DF
:1007C000F7FB00B9FEE729460D200AF08DF8614AD3
:1007D00061481268DFF8CCA1DFF888915F4EDFF83E
:1007E000C8815F4F00230121FFF75EFE0123C9F896
:1007F00000503560C8F800508AF8003004250F20FA
:100800000AF0A0FAD8F8003003440E20C8F80030EF
:1008100009F054FBD9F800309AF800200344C9F8D5
:1008200000301520002A6BD009F048FB33681844CB
:10083000306005F0010080F0010003F033FD3B88DB
:10084000002B14BF4B20FA200AF08AF8013DD6D1C4
:10085000D8F80030D9F80020424930683D88DFF8E8
:100860004CE1414F002BB8BF0333002AB8BF03321D
:1008700092100A603D493E4A098812880028B8BF94
:1008800003309B10801030605E1A19443E60CEF831
:100890000010384F384E3949C8F80030C2EB000E0E
:1008A0000244C7F800E032600B605DB94FF4FA70A3
:1008B00003F008FD03F0F2FC04F0F2FF40F2DC501C
:1008C0000AF04EF82E4B012504201D600AF012F8A4
:1008D00010B92C4B20701D702B4B1B881C2B16D075
:1008E0002A4A2B4B1078187005F0E6FE03F0D2FC74
:1008F00045F6BF5227492848BDE8F04709F096B8A9
:1009000011200AF01FFA33681844306091E7234B36
:1009100018880028E4D0224BC0B2197805F014FEE4
:10092000DEE700BF001B3746801A0600AC8FFF1FB2
:10093000F99AFF1F489CFF1FC89BFF1F509BFF1F7A
:10094000B5814E1BC489FF1FF89AFF1F809BFF1FB4
:10095000249BFF1F2489FF1FCC9BFF1FC09AFF1FF2
:10096000FA9BFF1FD89AFF1F1C9CFF1FD689FF1FF1
:100970002C89FF1F189BFF1F549BFF1F5C9CFF1FB0
:10098000209CFF1FE79AFF1F269CFF1FB49BFF1FA1
:100990009B9BFF1FA5050000409CFF1F589BFF1F4E
:1009A000109BFF1F149CFF1F189CFF1FA09BFF1F85
:1009B000F0B40E8886420DD203F10043013B31F8BA
:1009C0001350854202D9F0BCFFF734BE32F8130051
:1009D000F0BC70471088F0BC704700BF094B1B8803
:1009E0000C2B09D8084A80B252F8232028B143F6CC
:1009F000FE73984203D9108C7047108870470349E2
:100A0000FFF718BEF49AFF1F60EA000048EB0000F1
:100A1000374A38491088384AF8B5384B12881B686D
:100A2000834248DB9342A8BF134698420B60C8BF7D
:100A3000002342DD101AB0F5804FAABF9B03C3EB21
:100A40008333013093FBF0F0FFF7C8FF2C4B2D4FA1
:100A50001C883B68C0F3C61505FB04F47F2CA8BFB7
:100A60007F249D42064608D0274B1B88002B38D197
:100A7000264B1B88002B30D13D60254D2B689E42B4
:100A800005D0214B1B885A1F032A1DD92E60214DEA
:100A90002B689C420ED0204B188848B11A4B1F4A35
:100AA0001B88D35C834203D0C0B2E1B205F04CFD99
:100AB0002C60F8BDF8BD034608609A42D4BFC0EB75
:100AC0000203C0EB0303B5E7144AD05C2030C0B288
:100AD00006F07F0105F038FDD8E7284605F0A8FDAF
:100AE000CAE70E4A2946D05C05F02EFDC0E700BFDC
:100AF000829BFF1FC89AFF1F4C9CFF1F009CFF1F7B
:100B0000DC9AFF1F2C9BFF1FF09BFF1F7A9BFF1F90
:100B1000549CFF1F7C9BFF1F2A9CFF1FC889FF1F3F
:100B20002DE9F04F012089B00AF00CF9AF4B1860A5
:100B300000200AF007F9AE4BAE4A1B8810600C2B60
:100B400000F03B81AC4BAD4A19880093AC4B52F896
:100B5000214000221A70AB4BAB4D1B88AB4A2E884C
:100B6000013B32F91370002E5CD0A94BA94A1B88B7
:100B7000A9491278013B31F91380002A40F0DF8047
:100B800011200AF0DFF8A54B0193D3F800A0064628
:100B9000B24540F3DF80A24BDFF8A4921B88A14A44
:100BA000012BD9F80030B2F800B09F4A02922046DB
:100BB000C8EB030800F09A820CF080FC029A52F80D
:100BC0002B100CF0CFFC014600200CF0C1FB0CF008
:100BD0008FFECAEB0802B045B8BFB0469042CAEBE0
:100BE000080880F2968200FB0888013298FBF2F038
:100BF0008E4BDFF850820293D8F80030034403EBA9
:100C0000D3735B10C8F800302B88012B12D1884BAE
:100C1000DFF834B20393874BDBF8005004934FF0B6
:100C2000000A47E07D4B0193DFF814927F4BDFF819
:100C3000148202937E4B03931D460F200AF082F824
:100C40002B689842824641DA754A1288012A00F0E0
:100C50001D82744A05931288734D049220460CF04D
:100C60002DFC049ADFF8E0B155F82210DBF80050B3
:100C70000CF078FC014600200CF06AFB0CF038FE0A
:100C8000EF1B059B5745A7EB0302B8BF5746FF1A5A
:100C90009042BABF013200FB0777474397FBF2F758
:100CA000D8F80020634B0493BB1803EBD3735B109D
:100CB000C8F80030604B1B88013B032B00F2B08268
:100CC000DFE813F06301A901C4008601594B0493C6
:100CD0001B68984240F3C281514A1288012A00F0F1
:100CE000A682504A079311884F4A069120460592E2
:100CF0000CF0E4FB059A0699DFF84CB152F821108C
:100D0000DBF800500CF02EFC0CF0F2FD079B2F449A
:100D10005745A7EB0302A8BF5746FF1AD8F8003083
:100D20009042BABF00FB07770132474397FBF2F7C7
:100D30003B4403EBD3735B10C8F80030BAE71520CF
:100D400009F0BCF8354B0193D3F800A00646B24534
:100D50003FF721AF354B0293D3F800A0B24580F2A4
:100D600089812F4BDFF8D8901B882E4A012BD9F8A8
:100D70000030B2F800B02C4A03922046984400F0AC
:100D800070820CF09BFB039A52F82B100CF0EAFBDC
:100D90000CF0AEFDB045CAEB0802A8BFB046CAEBE6
:100DA00008089042B6BF00FB088800FB08F8013233
:100DB00098FBF2F0DFF88C801EE7204B1B78002BAD
:100DC0003FF4C0AE0C4B0D4A198800930C4B52F8FF
:100DD000210001221A700CF071FB4FF07C510CF0D5
:100DE000C1FB0CF085FD0446B5E600BF209BFF1F4C
:100DF000269CFF1F689CFF1F269BFF1F8C89FF1FDF
:100E0000CE9AFF1FD489FF1FA69BFF1FD8EC0000BE
:100E1000248AFF1F149CFF1F24EB0000189BFF1F58
:100E20006C9BFF1FF09AFF1FF0EC0000549BFF1F0C
:100E30001C9CFF1FA09BFF1F6089FF1FE69AFF1FDE
:100E4000C09AFF1F309CFF1F189CFF1F28460CF004
:100E500035FBB2490CF086FB054650460CF02EFBE4
:100E6000AF490CF07FFB014628460CF073FA0CF0FA
:100E70003FFD0546CBF80050D9F800000CF01EFBF2
:100E8000A6490CF06FFB074630460CF017FBA4494F
:100E90000CF068FB014638460CF05CFA0CF028FDBB
:100EA000C9F800009F4AA04B168819889F4AA04B9A
:100EB00012681B889F4FC6EB050E3544039EC6F88B
:100EC00000E0461A084404990D6001990E600299E9
:100ED0003E8808609A4280F289810025C3EB060EA5
:100EE000954974450F6880F27681611C9F4205FB2D
:100EF00001F50EF1010E95FBFEF5C0F2BE81BE427A
:100F0000A8BF3E46F61A01FB06F494FBFEF49A4293
:100F100000F33681BB42C0F23381884C20680CF06C
:100F2000CDFA87490CF01EFB86490CF013FA0CF041
:100F3000DFFCA0F5FF531C3B082B98BF4FF400507B
:100F4000D8F80030184400282060C0F24281B0F583
:100F5000804F80F252817C4B1B781BB1B0F5005F53
:100F600040F05381794D2B78002B40F05481784D1F
:100F700020682B68714C984204D080B205F0C2FB07
:100F800023682B6009B0BDE8F08F28460CF096FA74
:100F900070490CF0E7FA054650460CF08FFA6E499E
:100FA0000CF0E0FA014628460CF0D4F90CF0A0FC55
:100FB0000546CBF80050D9F800000CF07FFA6549DF
:100FC0000CF0D0FA074630460CF078FA62495FE739
:100FD00028460CF073FA5A490CF0C4FA05465046FC
:100FE0000CF06CFA5D490CF0BDFA014628460CF095
:100FF000B1F90CF07DFC0546CBF80050D9F80000A3
:101000000CF05CFA4E490CF0ADFA074630460CF095
:1010100055FA52493CE728460CF050FA50490CF07A
:10102000A1FA054650460CF049FA4E490CF09AFADE
:10103000014628460CF08EF90CF05AFC0546CBF818
:101040000050D9F800000CF039FA45490CF08AFA42
:10105000074630460CF032FA424919E7D8F800301A
:10106000DFF810B103EBD3735B10DBF80050C8F866
:1010700000301FE6DFF80081DFF80091D8F800307B
:1010800003EBD3735B10C8F80030BDE5364A069316
:101090001188364A059120460492DFF8D8B00CF04A
:1010A0000DFA049A0599DBF8005052F821100CF063
:1010B00059FA0CF01DFCEF1B069B5745A7EB0302EA
:1010C000B8BF5746FF1AD8F800309042BABF013275
:1010D00000FB0777474397FBF2F73B4403EBD373DF
:1010E000234A04925B10C8F80030E3E50CF0E6F9FF
:1010F000029A52F82B100CF035FA0CF0F9FBCAEBFF
:101100000802B045B8BFB0468242CAEB08083FF7B4
:101110006AAD00FB08F898FBF2F069E5CDCC4C3FD6
:10112000CDCC4C3ED689FF1F2C89FF1F209BFF1F73
:10113000FE9BFF1F089BFF1F689CFF1FC089FF1FAE
:101140009A99193FCDCC4C45FA9CFF1F789BFF1F05
:101150002089FF1F3333733FCDCC4C3DCDCCCC3EEB
:101160006666663FCDCCCC3DF09AFF1FF0EC0000E8
:10117000A09BFF1F189CFF1F309CFF1FC09AFF1FE2
:10118000009B1B88002B3FF4C8AE2B1B002BB8BF65
:101190005B42092B47DD05F500500130001B0CF0C8
:1011A0008DF93B493B4C0CF0DDF9054620680CF00D
:1011B00085F939490CF0D6F9014628460CF0CAF8F1
:1011C0000CF096FBD8F80030184400282060BFF6D9
:1011D000BEAE002213E09F4205FB04F5B8BF00211C
:1011E00095FBFEF54BDA91FBFEF490E6B242D4BFDC
:1011F000C3EB0205C3EB060570E643F6FF72274B0F
:1012000022601B78002B3FF4ADAE03F047F8244B6F
:1012100001221A70ABE603F03DF800232B70A6E61E
:10122000D9F800003EE64FF400501A4C88E61D49FC
:101230001D4A069320460D8805920CF03FF9059A49
:10124000DFF868B052F82510DBF800500CF08AF98E
:10125000014600200CF07CF80CF04AFB2F44069B62
:1012600056E50CF02BF9039A52F82B100CF07AF992
:10127000014600200CF06CF88AE51E4642E6B742B3
:10128000D4BFC3EB0701C3EB060104FB01F1AAE7DE
:10129000CDCCCC3EC089FF1F9A99193FFA9CFF1F05
:1012A000789BFF1FF09AFF1FF0EC0000189CFF1FB7
:1012B0002DE9F84FAB4C20680CF000F9AA490CF06E
:1012C00051F90546102009F03DFD0CF0F7F8A7494B
:1012D0000CF048F929460CF03DF80CF009FBA44B42
:1012E00020601B88192B00F08C801A2B00F0A48042
:1012F0000126B1469F4D2B88002B2DD020689E4F94
:101300003A88824233DD9D4A1178002977D0002443
:10131000012B147000F09D80022B40F03F81002EC5
:1013200000F09D80964D2B68002B00F098800420E3
:10133000214605F009F9934B2C60188800285ED0EF
:10134000B9F1000F5BD0C0B2002105F0FDF88E4B63
:1013500000221A60BDE8F88F8A4A1288002ACDD18F
:10136000864B1978002972D01A70BDE8F88F83492E
:1013700091F80080B8F1000F33D14FF0010E042B2B
:1013800081F800E02DD1002E40F02C812B88022B1B
:1013900001D0032B66D07B4B188800282FD0B9F1E1
:1013A000000F2CD023683C88784AA342128880F230
:1013B000D1800023141B7E2C734DD5BFC3EB831348
:1013C000C3EBC3135B00013493FBF4F42B680134CB
:1013D000A34203D0C0B2E1B205F0B6F82C60BDE87C
:1013E000F88F2B88012B67D0022BD2D1002ED2D0C0
:1013F000DFF88CB1DFF894A1DBF8003087E0BDE8BE
:10140000F88F634D634F2B784BB15E4A128832B12F
:101410003978994200F0D980D0B27F2105E03A783E
:101420009A4246D0574B1878002105F08DF80026D7
:101430002B783B70B1465DE7554B1B78002B0BBFFB
:10144000012600264FF000094FF0010952E7BDE8E0
:10145000F88F26B14A4D2A68002A40F0BB80494BDC
:1014600018886BE74C4B1B88092B94D0002E92D028
:1014700023683D88454AAB42128880F2D980002318
:10148000551B7E2DDFF8F8B0D5BFC3EB8313C3EB3C
:10149000C3135B00013593FBF5F5DBF80030013534
:1014A000AB4203D0E9B24A2005F04EF8CBF8005029
:1014B00071E70026B1461DE7002E3FF46CAFDFF860
:1014C000CCA0BAF800309842D4BFC2EB0008C2EBFF
:1014D00003089A1A7E2A40F3A280C8EBC81002F1D2
:1014E000010890FBF8F808F10108DFF894B0DBF888
:1014F0000030434504D05FFA88F1012005F024F85C
:101500002B88CBF80080022B7FF443AF4346226840
:10151000B7F80080BAF80010424579DA0022C8EB2B
:101520000108B8F17E0FD3BFC2EB8212C2EBC21228
:1015300008F10108520092FBF8F808F101089845FB
:1015400004D05FFA88F1042004F0FEFF2B88CBF86A
:1015500000801EE79342D4BFC4EB0303C4EB020335
:1015600028E700BF149BFF1F9A99193FCDCCCC3EB2
:10157000269CFF1F1E9BFF1FE09AFF1F2C9CFF1F36
:10158000889BFF1F369CFF1FFC9AFF1FAA9BFF1F13
:10159000E69AFF1FE29AFF1FF09BFF1F032B2CD13F
:1015A0002C4B1B88092B3FF45AAF002E3FF457AF4A
:1015B000294D2B68002B3FF452AF4A20214604F0FE
:1015C000C3FF264B2C601888B8E6254D00262B88D3
:1015D000B14694E61846214604F0B6FF1F4B2C6036
:1015E0001888ABE67F21402004F0AEFF2B88012B4A
:1015F00025D0022B7FF4CDAEFAE6042B7FF42FAF7B
:10160000002E3FF42CAF2146402004F09DFF26E73A
:101610008A42D4BFC8EB0202C8EB01027FE7C8EBE5
:1016200088184FEA480898FBF2F808F101085CE7CF
:101630009342D4BFC5EB0303C5EB020320E7206848
:101640003A88DFF820A09042BAF80030FFF641AFA8
:1016500039E700BFF09BFF1F889BFF1F369CFF1FD1
:101660001E9BFF1FAA9BFF1F08B50F4B1B88022B59
:101670000FD0032B12D0042B03D00C4B01221A7075
:1016800008BD7F21092004F05FFF084B01221A707A
:1016900008BD7F21412004F057FFEEE740210920DB
:1016A00004F052FFE9E700BF869BFF1F409BFF1F2E
:1016B00038B51C4B1B881D2B26D01B4B1B88012BC0
:1016C00025D01A4A1A4B14881B681A4AA34212885A
:1016D00018DB9342D4BFC4EB0303C4EB0203141B17
:1016E0007F2CC6BFDB010134C3EBC31393FBF4F4BF
:1016F000114D2B689C4203D0E1B2052004F024FF79
:101700002C6038BD0023EAE70C4B1C88F0E70C4B3B
:101710000C4A0D491B6812680C689B1A1C1B84F349
:101720000704E5E7269CFF1FA69BFF1F3A9BFF1FB0
:10173000D49AFF1F249CFF1F3C9CFF1F109BFF1F80
:101740005C9CFF1F2889FF1FB09BFF1F10B50F4C2B
:1017500023685BB90E4B1B88022B11D0033B012B76
:1017600009D90C4A00231370236010BD0021052005
:1017700004F0EAFEEEE70021092004F0E5FEF0E7C0
:101780000021412004F0E0FEEBE700BF3C9CFF1F7E
:10179000869BFF1F409BFF1F08B5274B1B78ABB1F3
:1017A000152008F08BFB254A254B128818601D2A4E
:1017B00015D0244A1288EAB1012A25D0224B1B7881
:1017C000002B34D0BDE80840FFF7C0BF112009F05E
:1017D000B9FA1A4A1A4B128818601D2AE9D11B4B14
:1017E0001B78002BEAD0184B1B780BB3BDE80840E0
:1017F000FFF75EBF164A1288002ADFD0154A1B6821
:1018000012889A42DADCEEE70F2009F09BFA104BBF
:10181000114A1B88106033B1104B114A1B681268C3
:101820009B1A9842DFDD084B1B78002BCAD108BDFC
:10183000FFF71AFFDAE700BF149CFF1F269CFF1F6B
:10184000D49AFF1FA69BFF1F409BFF1FE69AFF1F16
:10185000869BFF1F3A9BFF1FB09BFF1F5C9CFF1FD7
:101860002889FF1F2DE9F04FDFF870B39BF8006067
:10187000012E93B000F00F82C0F0E181022E00F043
:10188000B480B248B24BB34DDFF844E3B24AB34937
:10189000B34FB44C00940078B34C1B782D789EF86D
:1018A00000E01278097897F800A0DFF834C3DFF879
:1018B0003483DFF834930194012EAC4C94BF01368D
:1018C000002622708BF80060A94CAA4E237030705D
:1018D000A94CAA4E21703570A94CAA4E84F800A0DC
:1018E0003270BEF1000F40F0E680A74C24880D2C2A
:1018F00000F08081DFF8E0E2002426468EF8004008
:10190000A3462BB1A04B1C88002C40F080812346BD
:101910009E4C248803EB0B0E002C40F0D9809C4B8E
:101920009C4C1B7899F8009024780133A3EB490371
:10193000002C40F06F81019C24781B1B002C40F090
:1019400027824FF0000BDFF88492934C99F80090B7
:101950002478CBEB0303A3EB49032B44181A002C88
:1019600000F06B81B5FA85F56D099CF800300544EF
:10197000ED1A002B00F05F8119F1000018BF012063
:10198000009C98F800302778844C281AC31AA3EBDF
:1019900047030B449B1A2078814A82491468A3EBC1
:1019A0004A034FF00C0A1AFB00330B607E4909888A
:1019B00019440C3971440EB17C480360A14200F017
:1019C00015817B4B7B4C18680590059820601B683F
:1019D0000693794C069B248811601B1AA34284BF8E
:1019E000764B196013B0BDE8F08F754F06AE002539
:1019F000E9B2744806F0A0FA57F8043B0135C01A62
:101A00000C2D46F8040BF3D16F4B079FB3F800C0C1
:101A10000E9B0D9E0F9D1098534C01946345ACBFD7
:101A20004FF0000E4FF0010EBC45D4BF0027012738
:101A3000B445D4BF00260126AC45D4BF4FF0000802
:101A40004FF00108119B84F8008084455F4C604989
:101A5000504ADFF894911770D4BF4FF0000A4FF04E
:101A6000010A9C45099B84F800A03A4C81F800E0EB
:101A7000D4BF002501259C450A9B2570334C344F6B
:101A8000354A89F80060D4BF00200120344E334924
:101A900020709C45D4BF00230123324C96F800A04F
:101AA0003B70127809789BF80060DFF834C1DFF8EA
:101AB0003481009400E7474E474CB6F800B0012649
:101AC000BBF1180F267040F2B2804FF0000B18E700
:101AD000012C00F09181022C00F03082032C00F0E8
:101AE0005E812B4B9CF800B01D78009B99F800207C
:101AF0001978019C284B98F8008093F800C027784B
:101B0000A5EB4B05A1EB8104C2EB8273C8EB050189
:101B10002144C2EB83028B1803EB4C0303EB8A0ACC
:101B200027B12A4B1B78002B40F0A58201231B49CB
:101B30001B4A09781B481468C1F10601534401EBA4
:101B4000410103EB8103036030E700BF3D9BFF1FB2
:101B50003E9BFF1F3C9BFF1FED9BFF1FEC9BFF1F4E
:101B6000EE9BFF1F299CFF1F3A9CFF1F6D9CFF1FD0
:101B70006F9CFF1F6E9CFF1F719CFF1F709CFF1FBF
:101B8000739CFF1F729CFF1F749CFF1FCC9AFF1F4A
:101B9000D889FF1F609CFF1F4A9CFF1FA59BFF1F4A
:101BA000349BFF1FF49BFF1FDE9AFF1F0C9BFF1F40
:101BB0005C9DFF1F5C9BFF1F349CFF1F649CFF1FED
:101BC0003089FF1F809BFF1F489CFF1F3B9CFF1F0E
:101BD0003F9BFF1F269CFF1FE69AFF1F9A9BFF1F3C
:101BE0006C9CFF1F289CFF1F399CFF1FB648B74BFA
:101BF0000068ECE6002B3FF47DAEB54EB54FB6F86D
:101C000000B00126BBF1180F3E7010D9F346A4F1C5
:101C10000D037DE6019C2478B9F1000F40F09D8012
:101C2000013B1B1B002C3FF48CAECB468BE6ABF18B
:101C30000C0B012665E61846A2E6254695E6A64F5A
:101C400006AE0025E9B2A54806F076F957F8043B40
:101C50000135C01A062D46F8040BF3D1A04B0B9AA0
:101C60001B88A04800219A420170C0F282800A9A23
:101C7000934240F3E2819C4B9C4A9D4993F800A01B
:101C800012780978DFF8A0C2DFF8A082052303707C
:101C9000984B009351E0984F06AE0025E9B2974863
:101CA00006F04AF957F8043B0135C01A0C2D46F8E6
:101CB000040BF3D18A4B099C18880A9F904B0E9A0B
:101CC000DFF86882DFF860C206A962C98442ACBF4F
:101CD0004FF000094FF00109B842D4BF0027012797
:101CE000B042D4BF0026012683F80090A842814B61
:101CF0000093D4BF0025012588421D70D4BF002168
:101D000001217A4B0D9C88F800609042D4BF0022DC
:101D100001221A70109B764E734D8CF80070A04211
:101D2000D4BF4FF0000A4FF0010A9842317085F895
:101D300000A018DC002373480370734E7348744B83
:101D4000744D754C96F800E000781B782D789BF860
:101D50000060DFF8DC910194AEE5002C40F0838157
:101D6000013BA346EFE50F9B9842D4BF002301231C
:101D7000E1E75D4B5D4A5E4993F800A05D4B05705D
:101D800012780978DFF8A0C1DFF8A0810093D4E7CA
:101D9000B9F1000F3FF4D5AD4FF0010BD3E55F4A29
:101DA0009CF800301478009A98F800C0117899F8DF
:101DB0000020534F019D3F782D78A4EB4303A1EB06
:101DC0008101CCEB0303C2EB82740B44C2EB8402AF
:101DD000134403EB470303EB8A0A002D40F04F81C5
:101DE0000120404B4E491B784E4A82440C2010FB88
:101DF00003A30B601468D9E5484BDFF838B11F78AE
:101E000099F800309BF80090029307F1010BABEBBF
:101E100043031F46B9F1000F40F00081019C94F884
:101E200000B0C9EB0703CBEB03030193BBF1000F39
:101E300040F0EF805B46324CDFF8FC90247803944E
:101E40002746019C99F80090E31AA3EB49032B4421
:101E5000181A002F00F0D880B5FA85F464099CF8B0
:101E600000302044C41A002B00F0CC8019F100058A
:101E700018BF0125009B98F800C01878631BCCEBB5
:101E80000303A3EB40030B449B1A029AA3EB4A0300
:101E9000002A40F0B480BBF1000F40F0FE805B44AC
:101EA000002840F0C880BAF1000F0CBF00216FF08D
:101EB00009010C4A1A4814781A4A19440C2313FBD6
:101EC00004130360146871E55C9BFF1F5C9DFF1F9A
:101ED000269CFF1FE69AFF1F0C8AFF1FF89AFF1F20
:101EE000489CFF1FA59BFF1FEE9BFF1FED9BFF1F45
:101EF000EC9BFF1F299CFF1FDC89FF1F249BFF1FFA
:101F00004A9CFF1F0A9BFF1F3F9BFF1F3D9BFF1F1C
:101F10003E9BFF1F3C9BFF1F3A9CFF1FD889FF1F62
:101F2000F49BFF1F349BFF1F6C9CFF1F289CFF1F0F
:101F3000399CFF1F609CFF1F3B9CFF1F019C774B40
:101F400024780194009CDFF804B22778744C98F848
:101F50000080247800949CF800C099F800909BF8C9
:101F600000B09DF8044083F806805A72DFF8E081E3
:101F70009DF8002083F805C0DA709C7083F800900B
:101F80001D71DF71197283F80AA083F801B04FF058
:101F9000000C01220023614F194645464C4607E0DC
:101FA000022A09D00B2B0BD017F8014F15F8012F7F
:101FB000944203F10103F3D101310B2BC9B2F3D1E8
:101FC0000A2907D80CF1010CBCF1110F4DD018F8FB
:101FD0000B2FDFE7534A544B1478544953F82C2005
:101FE000534B09781B78534D01342244101A08448E
:101FF000514A0C2111FB03032B601468D6E44FF007
:10200000000B4CE71D4635E7039C28E7CBEB0703A5
:102010000193029B003318BF01230CE7029B002BA6
:1020200036D0019B93F800B0BBF1000FEED17B1EC0
:1020300001935B46FFE600213BE7099A934234DCBB
:10204000089A934241DD3D4B3D4A3E4993F800A03A
:1020500012780978DFF8FCC0DFF8FC8003230370F6
:10206000394B009369E61B1B96E6334A314B1468E3
:102070001C6023469AE4031C18BF012357E5284B34
:102080001B78002B3FF4ACAE003018BF0120A8E64F
:10209000019BA14693F800B0C3E6B9F1000F0CBF55
:1020A0004FF0000B4FF0090BF9E6244B244A254969
:1020B00093F800A012780978DFF898C0DFF89880CC
:1020C00004230370204B009337E6079A93420FDDF9
:1020D0001A4B1B4A1B4993F800A012780978DFF8C5
:1020E00074C0DFF8748002230370174B009324E65A
:1020F000069A1449DFF85CC00978DFF85C809342E7
:102100000F4A0E4B127893F800A004DD01230370F0
:102110000D4B009311E60C4B00930EE6609BFF1FE6
:102120003B9CFF1FD889FF1F94EC00004A9CFF1FB7
:10213000A59BFF1FF49BFF1F349BFF1FEE9BFF1F00
:10214000ED9BFF1FEC9BFF1F299CFF1F609CFF1F47
:102150006CEB00006C9CFF1F289CFF1F2DE9F04FCB
:10216000354B1B788BB0002B61D10E2007F0A6FEFB
:102170000BF0A4F901463148314C324DFEF7DAF943
:102180002E48FEF7ADF90BF0B3FB80F30C00206096
:10219000FFF768FB2E68012E6CD0022E00F08C82B7
:1021A000032E00F09B83284C2368284A284E09936D
:1021B000099B17783068274C07210122181A11FB58
:1021C00007229042236000F23182234E32689A1A2D
:1021D0000D2A00F22482214E32689A1A132A00F244
:1021E00019821F4E32689A1A252A0ED91D4A128862
:1021F0001B3A92B2022A04D81B4A1278002A40F0F5
:10220000488102F071F823683360184D2A689B1AE0
:10221000502B00F21082164B1B88012B00F02882F5
:1022200004F026FA04F054F80BB0BDE8F08F05F086
:10223000ADF80BB0BDE8F08FF99AFF1FCC9BFF1FE4
:10224000009CFF1F209CFF1F5C9DFF1F9C9BFF1F8E
:10225000AC9BFF1FC49BFF1F709BFF1F489BFF1F72
:102260004C9BFF1F269CFF1FE69AFF1FB89BFF1F7A
:10227000049CFF1FDFF80C839D4AB8F80000137818
:10228000834204D0C3B21846137004F02DF9DFF86E
:10229000F092984AB9F800301178994204D0964FDC
:1022A0003978002940F07087944A23681288944C4A
:1022B0009A42C0F2F380934A1278002A40F0EE80EE
:1022C000DFF8C4A2BAF8003023B98F4B1B88002B6B
:1022D00000F010858D4A8E4B11881B888D4A0B4467
:1022E00012685B1093428C4A126880F2B38400211A
:1022F0009342B4BF01230B4604910093ACBF4FF04F
:10230000010B8B4605910E2007F0D8FD834B844AC4
:102310001B68176803930133A7F25232002B8446DF
:10232000029240F34287802BA8BF80237D4A7E49DA
:1023300012780191002A00F0BB800978914200F0E8
:10234000B780B9F80010DFF838E2994201F039811E
:102350006949AEF80030754B4FF0010E81F800E08E
:102360001978DFF828E2019B8EF800101A70009BA4
:10237000002B00F00D81BAF80030002B00F008812E
:102380006B4B1B685A1C002A40F31387802A00F30A
:102390000F87684E68496948368809880068314463
:1023A000B0EB610FC1F2E181A3F148020F2A02D81C
:1023B000473BA8F800300E2007F080FD6FF45473FF
:1023C0001F44874202DC5E4B00221A705D4B1B8863
:1023D000002B00F037845C4B5C4A1B7811789942E3
:1023E00040D0002B3ED05A490E78002E00F0C68710
:1023F000584991F800C0BCF1000F40F0BD87564F1E
:102400000097564F56480297534F007887F800C000
:10241000524F4FF0010E87F800C081F800E000280D
:1024200041F061814F490978002901F022804E492D
:1024300003910E460978002941F018804B48474F18
:102440000078397001210297317058B142484149F2
:102450000090002008700099029F087003990126DF
:102460003E7008701370424B1B88A3F11B02012AB7
:1024700040F265861D2B7FF497AE3C4F3B78002BD6
:1024800041F0E4803B4E3378002B40F0638433709E
:102490008AE62A68012A7FF4B4AEB5E62168364A96
:1024A000069106983549106002220B602A6007E702
:1024B0001E49DFF8D8E0097800293FF454AF9EF8B0
:1024C000000081423FF44FAF03984B2841F3258031
:1024D0001833802BB9F80000A8BF802398423FF43E
:1024E00042AF274803800448012303703BE700BF45
:1024F0009B9BFF1F509BFF1FE79AFF1F829BFF1FA5
:102500005C9DFF1FF29AFF1F769BFF1F089BFF1F1A
:10251000FE9BFF1F209BFF1F689CFF1F0C9BFF1F44
:10252000D89AFF1F589CFF1F309BFF1F599CFF1F0D
:10253000F49BFF1FE09AFF1FAA9BFF1F149BFF1F26
:10254000A49BFF1F069CFF1F0A9BFF1FC49AFF1F2F
:10255000709CFF1FFC9BFF1F389CFF1F849BFF1F6D
:10256000719CFF1F6D9CFF1FC59AFF1FE69AFF1FFE
:10257000269CFF1FE29AFF1F449BFF1FC09BFF1F6B
:10258000C89BFF1FB49BFF1F389BFF1F319BFF1F82
:10259000029B9C45BFF60FAFAC4B1B88002B3FF452
:1025A0000AAFBBF1000F7FF4EBAEA94B1B881BB148
:1025B000059B002B7FF4E4AE049B002B3FF4FBAEA5
:1025C000A44B1A78002A7FF4F6AEDFF8048398F85B
:1025D000006001221A70002E40F059839E4B1B7838
:1025E000002B01F004819D4B1B78002B01F015811D
:1025F0009B4B1B78002B7FF4DEAE9A4B1B78002B95
:102600003FF4D9AEB9F8003097490A3BA9F8003039
:102610000A70D0E6FFF7C0F823683360E1E5FEF703
:102620007FFAFEF745FE23683360D4E5FEF7F0F944
:1026300023683360C9E502F0C7FE8C4B1B7873B981
:102640008B4B1B785BB98B4B1B7843B98A4B1B7840
:102650002BB98A4B1B7813B901F01CFE01E001F085
:1026600025FE23682B60864B1B88012B7FF4D8AD99
:10267000844A854B116885481A78A1F118032A21EC
:1026800001FB03F10160002A00F0C682804A136852
:10269000994200F3338380F23D837E480068D0F195
:1026A0007F0048BF0330801001301B1A994200F3AD
:1026B000318313601946B1E2774A26681288B24224
:1026C00004DB6E4B1B78002B00F03F83734C744887
:1026D00023680793734B079900681B88091A99426E
:1026E00063D8002B61D0704B198800293FF45CAD92
:1026F0006E4B6F481B680088B342B8BF33469A429E
:1027000041F32C806B4B1A60DFF8C88188F8001009
:102710005C4FFEF77DF938687F2840F32986664BC9
:102720007F3883FB0032C317C3EB620303EB430321
:10273000A0EB83007330614B01931B883860002B42
:1027400040F031874B4B00931B78002B00F05A84EC
:102750005B4E3378002B00F05584DFF87C91DFF876
:1027600058A14FF0000B0CE003F17300C0B298F8D1
:10277000001003F011FF33780BF1010B5B4540F3C0
:1027800041843B6859F8040F1844A0F17F038AFB89
:102790000321DA17C2EB610202EB42027F28A3EBAE
:1027A0008203E1DCFDF76EFFE0E7404B40491B6828
:1027B00008883D49B342B8BF33469A4200F3AC8221
:1027C0003C4E09888342A8BF0346336000299BD151
:1027D0009A42C8BF0B4640F3A682801AB0F5804FDC
:1027E000AABF9B03C3EB8333013093FBF0F0FEF7EA
:1027F000F5F8C0F3C6100AF061FE324B06461888A1
:102800000AF05CFE3049074630460AF0ABFE01464E
:1028100038460AF0A7FE31460AF09CFD4FF07E5183
:1028200006460BF03DF8002840F08D8727493046DA
:102830000BF054F8002840F04A8730460BF07EF841
:10284000C0B2DFF8908088F8000061E7769BFF1F38
:10285000BC9BFF1FA49BFF1F6D9CFF1F6E9CFF1F57
:102860006F9CFF1F709CFF1FE79AFF1F849BFF1F39
:10287000FC9BFF1F389CFF1FC59AFF1FF29AFF1F8A
:10288000049CFF1F649CFF1F409BFF1F509CFF1F69
:10289000EC9AFF1F3C9CFF1F829BFF1F5C9DFF1F4C
:1028A000449BFF1F749BFF1FE49AFF1FC09BFF1FE9
:1028B0004C9CFF1FC89AFF1FABAAAA2A1C9BFF1F94
:1028C0008889FF1FD09AFF1FCDCCCC3D0000FE426F
:1028D000A59BFF1F6E9BFF1F6089FF1FB94B2668DA
:1028E0001988B14253DDB84B1B78002B4FD1DFF86C
:1028F000209399F800007F2840F3A486A3F1553374
:102900007F3803F1004383FB0032C317C3EB62033C
:1029100003EB4303A0EB83007330AC4B01931B88A4
:10292000C0B289F80000002B40F0ED86A84B009360
:102930001B78002B00F04D85A64E3378002B00F05D
:102940004885A54FDFF898824FF0000A0AE003F1AE
:102950007300C0B203F048FE33780AF1010A534510
:1029600040F3378557F8043F99F800001844A0F168
:102970007F0388FB0321DA17C2EB610202EB4202FC
:102980007F28A3EB8203E2DCFDF77CFEE1E7934FB7
:1029900038687F2840F3CE81914B7F3883FB00322B
:1029A000C317C3EB620303EB4303A0EB8300733055
:1029B000DFF85C9299F800A0824500F02582894BEF
:1029C0001B88002B43D1884A8848126800889142AE
:1029D00005DC8242D4BFC1EB0203C1EB0003411A04
:1029E000B1F5804FA6BF9B030131C3EB833393FB4B
:1029F000F1F0FDF7F3FFC0F3C6100AF05FFD7C4B6A
:102A0000064618880AF05AFD7A49804630460AF090
:102A1000A9FD014640460AF0A5FD31460AF09AFCA0
:102A20004FF07E5106460AF03BFF002840F06886D2
:102A3000714930460AF052FF002840F03786304690
:102A40000AF07CFFC0B2DFF8CC8188F80000BAF150
:102A50007F0F40F388846248AAF17F0A80FB0A3026
:102A60004FEAEA73C3EB600000EB4000AAEB800082
:102A70007330574B00931B78C0B289F80000002BCD
:102A800040F0E8835D4B03931B78002B40F0B58545
:102A90005B4B02931B78002B40F058864B4B019305
:102AA000029B1B78002B3AD0564B1B88182B17D053
:102AB00099F800201344A3F118007F2840F3F9850A
:102AC000474A973B82FB0321DA17C2EB610202EB14
:102AD0004202A3EB820303F17300C0B203F084FD52
:102AE000494A4A4B127833F81230182B17D099F80C
:102AF00000201344A3F118007F2840F3E485384AEE
:102B0000973B82FB0321DA17C2EB610202EB420220
:102B1000A3EB820303F17300C0B203F065FD009BD9
:102B20001B78002B00F0B584019B284E19880029E2
:102B300000F05C8538687F2840F35783284B7F3846
:102B400083FB0032C317C3EB620303EB4303A0EB29
:102B5000830073303860002940F0F084009B1B78BC
:102B6000002B00F05C811B4E3378002B00F0578166
:102B7000DFF864A0DFF89C804FF0000B0CE003F15D
:102B80007300C0B298F8001003F006FD33780BF123
:102B9000010B5B4540F343813B685AF8040F104A30
:102BA0001844A0F17F0382FB0321DA17C2EB610214
:102BB00002EB42027F28A3EB8203E0DCFDF762FD1B
:102BC000DFE700BF829BFF1FF29AFF1F1C9BFF1FC6
:102BD000389CFF1F8889FF1F6089FF1F649CFF1FAF
:102BE000ABAAAA2AE49AFF1FC89AFF1F4C9CFF1F9A
:102BF000D09AFF1FCDCCCC3D0000FE42C59AFF1FEE
:102C0000849BFF1F029BFF1F6F9BFF1F0C9CFF1FDE
:102C1000F89BFF1F6E9BFF1FA84B1960A84B1B68FA
:102C2000A92202FB03F3002BBCBF03F57F533F3304
:102C30009B13543B194481F30C01282007F0C4FC7A
:102C4000FFF7EEBA9F4EA048A049A14A3370037027
:102C50000B7007E493424FF0000B6EDA0123CDF8BE
:102C600000B0CDF814B00493FFF74DBB994B1B781F
:102C7000002B7FF4A0AB039B974A243B83F34703CD
:102C8000D9B25B20136003F05FFC98F80060032E5C
:102C900030D1DFF8948298F80030002B40F0408665
:102CA0008E4F3B78002B40F02E868A4E3378002BD7
:102CB00040F01C868A4B1B78002B40F00A86894A1C
:102CC0001380894B1B78002B40F0F685874B7F22C1
:102CD0001A8098F800306BB93B785BB933784BB900
:102CE000834A7F210720138003F02EFC7F210B20D5
:102CF00003F02AFC7F4B1F68FFF75DBB7E4800682E
:102D0000D0F17F0048BF033003EBA00301339942A9
:102D1000BFF6CFAC116081E7784B09881A600029B3
:102D20007FF4F2AC13469842D4BFC2EB0003C2EB6F
:102D3000030352E5FDF7A6FC3AE60123CDF810B0F7
:102D4000CDF800B00593FFF7DEBA01232B606C4C81
:102D5000FFF72ABA6B4B6A20198803F079FD3B789C
:102D60003370FFF721BA574B1B78002B3AD0664BD4
:102D70001B88182B17D099F800201344A3F11800D2
:102D80007F2840F3F784614A973B82FB0321DA17DF
:102D9000C2EB610202EB4202A3EB820303F1730078
:102DA000C0B203F021FC5A4A5A4B127833F8123061
:102DB000182B17D099F800201344A3F118007F288E
:102DC00040F3DC84514A973B82FB0321DA17C2EBC4
:102DD000610202EB4202A3EB820303F17300C0B273
:102DE00003F002FC019B1B88002B00F09684364BFD
:102DF0001B78002B40F08B84474B404A198826688B
:102E00000020012310602B60B1423D4CBFF6CCA9DD
:102E10002268424B0892089A1A60FFF7C5B9039BD3
:102E20001B78002B00F084803B68A3F10C007F2806
:102E300040F3FB8335488B3B80FB0320DA17C2EB62
:102E4000600000EB4000A3EB800303F17300DFF8A8
:102E5000D480C0B298F8001003F09EFB009B1B7852
:102E6000002B65D02E4E3378002B61D0DFF8BCA04C
:102E70004FF0000B0BE003F17300C0B298F80010A4
:102E800003F08AFB33780BF1010B5B4550DD3B68A7
:102E90005AF8040F1D4A1844A0F18B0382FB03214A
:102EA000DA17C2EB61020C3802EB42027F28A3EB77
:102EB0008203E0DCFDF7E6FBDFE700BFEC9AFF1FD3
:102EC000C089FF1F849BFF1FFC9BFF1F389CFF1FB7
:102ED000C59AFF1F709CFF1F049BFF1F6F9CFF1F65
:102EE0006E9CFF1F7A9BFF1F719CFF1FE49AFF1FC0
:102EF000F09BFF1FD89AFF1F3C9CFF1FC89AFF1F23
:102F00005C9DFF1F109BFF1F029BFF1FABAAAA2AFD
:102F10006F9BFF1F0C9CFF1F829BFF1F049DFF1FC9
:102F20008889FF1F6E9BFF1F6D9CFF1F6089FF1F1D
:102F3000029B1B78002B3AD0AD4B1A88182A18D068
:102F40003B681344A3F118007F2840F3B683A94AD5
:102F5000973B82FB0321DA17C2EB610202EB4202CC
:102F6000A3EB820303F17300A34BC0B2197803F003
:102F700013FBA2490B78022B00F253830133DBB21F
:102F80000B701A469E4830F81260182E40F090825E
:102F90000422032B03F10106F3B208BF002330F82B
:102FA0001360182E40F08382013AF2D10B70019B1E
:102FB0001B88002B00F0CB82009B1B783BB9039B46
:102FC0001B7823B9029B1B78002B00F0E0838D4B0C
:102FD0001B78002B00F0D6808B490B78082B00F271
:102FE000D1808A483A680068894E0133DBB25F1E9F
:102FF000101A46F827000B70864B2668198889F846
:10300000002001E77F4B1B78002B40F0C1823B681A
:10301000814A1278002A45D0A3F10C007F2840F3A2
:103020000A83744A8B3B82FB0321DA17C2EB6102ED
:1030300002EB4202A3EB820303F17300C0B298F8E3
:10304000001003F0A9FA009B1B7853B36E4E33783F
:103050003BB3DFF8FC91DFF89CA14FF0000B0BE0D5
:1030600003F17300C0B298F8001003F095FA3378BA
:103070000BF1010B5B4514DD3B6859F8040F184454
:10308000A0F18B038AFB0321DA17C2EB61020C3833
:1030900002EB42027F28A3EB8203E1DCFDF7F2FAA8
:1030A000E0E73B685D4A1278002A3DD0504A12881A
:1030B000182A18D01344A3F118007F2840F30D8379
:1030C0004C4A973B82FB0321DA17C2EB610202EB09
:1030D0004202A3EB820303F17300C0B298F8001020
:1030E00003F05AFA3B6845490A78022A00F2A682A0
:1030F0000132D2B20A701646414830F816E0BEF1ED
:10310000180F40F0F0810426032A02F1010E5FFA45
:103110008EF208BF002230F812E0BEF1180F40F026
:10312000E181013EF0D10A70019A1288002A00F074
:1031300041823B4903220B702A60FFF735B8394FB3
:103140003B78002B3FF49EA9374E307801F01CF9F4
:10315000364B1B78002B00F0918233887E2B00F2D7
:103160008D82334A0133108899B23180002800F0F3
:103170009582C9B2C0B22F4E03F0E6F93B783370A6
:10318000FFF712B83A6837E7DBB21846137003F05E
:10319000B9F9294B1B491A461F4B184600230B70DF
:1031A0003B7013700370FFF77FB80123FFF7BEB8C1
:1031B00080262249224B234A09881B8812680B4427
:1031C000B2EB630FBFF6F7A8164B1B78002B40F04D
:1031D000FE81B9F800301C4AB3423FF4ECA81B4B07
:1031E000168001221A70FFF7E6B8FDF74BFAB1E43A
:1031F000029BFF1FABAAAA2A6E9BFF1F6F9BFF1F9C
:103200000C9CFF1FFC9BFF1F8889FF1FE89AFF1F74
:103210006489FF1F829BFF1FC59AFF1F849BFF1FAE
:10322000F89BFF1FE69AFF1F109BFF1F729CFF1F5A
:10323000589BFF1FE29AFF1F389CFF1FAA9BFF1F8E
:10324000E09AFF1F149BFF1FC89BFF1FE79AFF1FF9
:103250006089FF1FC14B01931B88002B40F06C83DA
:10326000BF4B0393BF4B0293BF4E33786BB3DFF872
:103270001483DFF8F8A24FF0000B09E003F17300AC
:10328000C0B203F0B1F933780BF1010B5B451CDDE3
:1032900058F8043F99F800001844A0F17F038AFB16
:1032A0000321DA17C2EB610202EB42027F28A3EB93
:1032B0008203E3DCFDF7E6F9E2E7AA4B029303F0B1
:1032C00093F9009B1B78002BCED1039B1B78002B1E
:1032D0003FF4E6AB99F80030A3F10C007F2840F3EF
:1032E000A781A2488B3B80FB0320DA17C2EB60006A
:1032F00000EB4000A3EB800303F17300C0B203F0C6
:1033000073F9009B1B78002B00F08081964E337878
:10331000002B00F06582DFF86C82DFF850A24FF0DE
:10332000000B0AE003F17300C0B203F05DF93378DB
:103330000BF1010B5B457FF7B3AB58F8043F99F8ED
:1033400000001844A0F18B038AFB0321DA17C2EBBB
:1033500061020C3802EB42027F28A3EB8203E1DC1E
:10336000FDF790F9E0E75046FDF78CF9FFF781BBD8
:10337000FDF788F9FFF7DFB9002008707C4908786D
:1033800040B17C4900910978002900F0A981009F93
:10339000002139707849097800297FF448A8002E67
:1033A00067D1002865D1754E724F96F800E06C4EDB
:1033B00003966C4E02966A4E71493070694E0097C2
:1033C000087038703070BEF1000F7FF442A8FFF72C
:1033D00049B8634B1B78002B3FF4C5AC99F800301B
:1033E000A3F10C007F2840F3C281604A8B3B82FB33
:1033F0000321DA17C2EB610202EB4202A3EB820364
:1034000003F17300C0B203F0EFF8009B1B78002BB0
:103410003FF4A9AC544E3378002B3FF4A4AC594F81
:10342000DFF848814FF0000A0AE003F17300C0B2F0
:1034300003F0DAF833780AF1010A53457FF793ACC9
:1034400057F8043F99F800001844A0F18B0388FB5B
:103450000321DA17C2EB61020C3802EB42027F282B
:10346000A3EB8203E1DCFDF70DF9E0E7039800210F
:1034700001704249097800293EF4F4AF39490291BC
:103480000978002900F08881029800210170FEF778
:10349000E9BF039B1B78002B7FF446AB029B1B7894
:1034A000002B7FF441AB019B1988FFF743BB0B70E6
:1034B0003B681E44A6F118007F2840F301812B4B86
:1034C000973E83FB0632F317C3EB620303EB430320
:1034D000A6EB830606F173002B4BC0B2197803F0FC
:1034E0005BF864E50A707344A3F118007F2840F389
:1034F000F1801E4A973B82FB0321DA17C2EB61027F
:1035000002EB4202A3EB820303F17300C0B298F80E
:10351000001003F041F83B6806E6243B002BB9F8A5
:10352000000040F32F8198423EF41DAF9BB2174834
:10353000A9F8003001230370FEF715BFDFF84880BB
:10354000C0B298F8001003F027F8FFF707BB0E4B46
:103550003878197803F020F82EE500BF1C9BFF1F78
:10356000C59AFF1F849BFF1F8889FF1FABAAAA2A49
:10357000719CFF1F389CFF1F6D9CFF1FE69AFF1F69
:10358000FC9BFF1F6089FF1F6E9BFF1FE79AFF1FB9
:103590007F21402002F0D8FFB349B44A3B680B605A
:1035A0000021117034E5C0B298F8001002F0F4FF69
:1035B000FFF7C8B8D8B298F8001002F0EDFF3B68EA
:1035C000B7E5AB4BDFF8ECE21978FEF7CCBE4B2E3B
:1035D00040F3A9801836802EB9F80030A54AA8BF5C
:1035E0008026B3427FF4FBADFEF7E5BE99F80000FC
:1035F00002F0FAFF3188FFF79DBA9F4B01931B88B9
:10360000002B7FF45AAE9D4B029363E6029B1B781E
:10361000002B7FF449AA039B1B78002B7FF484AA1C
:1036200041E7002213460A70ACE4FDF72BF80EE4E4
:10363000FDF728F862E6FDF725F8FFE400221646BC
:103640000A7059E5FDF71EF8FFF767B98C4E307820
:1036500000F09AFE8B4B1B781BB133887E2B40F217
:10366000A780894B1B7823B13388854A002B40F013
:10367000AB80864E3B783370FEF796BD824B1B784D
:10368000002BF6D033887E4A002BF2D08049013BD4
:10369000088899B2118000287FF46BADC8B27B4EC8
:1036A00002F0C6FF3B783370FEF77EBD7F20FFF748
:1036B000CAB9FCF7E7FFFFF710BAFCF7E3FF53E4E2
:1036C000FCF7E0FF08E7FCF7DDFFFFF725BA7F20F6
:1036D000FFF7B7B8FCF7D6FF18E7FCF7D3FFFCE419
:1036E000664F6C4902974FF0000C81F800C0009FB4
:1036F00002994FF0010E87F800E081F800C049E61A
:103700000120FFF7A0B902F06FFFFFF70FB900210A
:10371000402002F019FFFFF76FBB99F8000002F09C
:1037200063FFFFF764BB243E002EB9F800303ADD9A
:10373000B3423EF440AEB6B2574BA9F80060012246
:103740001A70FEF738BE0120FFF77BB84A4B019391
:103750001B88002B7FF4B3ADFFF7A2B94F4A834219
:10376000A8BF03461360FEF7CFBF16462CE5FCF753
:1037700089FF47E6FCF786FFFFF712BBFCF782FFE5
:10378000FFF72DBB01283EF4EEAD0123CFE699F8FB
:10379000000002F029FF1AE44148009041483D49E9
:1037A0000390FEF756BE012B3EF405AE0126C3E79B
:1037B00001339BB23380D9B20520344E02F0C4FEEF
:1037C0003B783370FEF7F0BC013B9BB2D9B20520C9
:1037D0002E4E138002F0B8FE3B783370FEF7E4BC47
:1037E000029B1B78002B7FF45FA9FFF79DB92E4B3E
:1037F0001B782BB32D4B1B78002B7EF4DCAD2C4BB0
:103800001B78002B3EF4D7ADB9F8003022490A33BB
:10381000A9F800300A70FEF7CEBD244B1B78002BB0
:103820007EF4C9AD224B1B78002B3EF4C4ADB9F831
:1038300000301949013BA9F800300A70FEF7BBBD02
:103840001A4B1B78002B7FF411AA194B1B78002B05
:103850003EF4B1ADB9F800300F490133A9F800309A
:103860000A70FEF7A8BD00BFE89AFF1F8889FF1FF6
:10387000599CFF1FC89BFF1F1C9BFF1F849BFF1FA2
:10388000109BFF1F729CFF1F719CFF1FE29AFF1F7E
:10389000589BFF1FFC9BFF1FE79AFF1FC89AFF1F43
:1038A000389CFF1FC59AFF1F6E9CFF1F6F9CFF1F58
:1038B000709CFF1F319BFF1F224B00227F2107209E
:1038C0001A8002F041FE7F210B2002F03DFEFFF73F
:1038D00000BA1D4B01227F2107201A8002F034FE1E
:1038E0007F210B2002F030FEFFF7EBB9174B0422CB
:1038F0007F2107201A8002F027FE00210B2002F012
:1039000023FEFFF7D7B9114B02227F2107201A802F
:1039100002F01AFE7F210B2002F016FEFFF7C5B958
:103920000A4B002107201E8002F00EFE7F210B2093
:1039300002F00AFEFFF7B4B9054B0393054B02935F
:10394000BDE400BFE49AFF1F7A9BFF1FF09BFF1F9F
:10395000C59AFF1F849BFF1F38B506F04BFB0E482E
:1039600004F082FA0D4804F07FFA0D4804F07CFA66
:1039700000234FF07E5201210A48FCF777FD0A4BE5
:103980000A4A0B49802400251C7118461D60BDE8B9
:10399000384009F0F3BF00BFF89AFF1F249BFF1FB8
:1039A000809BFF1FCC9BFF1F409CFF1F1C89FF1F9C
:1039B0002906000043682A20198802F049BF00BF89
:1039C00010B5044622206368198802F041FFE368BD
:1039D00024201988BDE8104002F03ABF10B5044613
:1039E0000A206368198802F033FFE3680C20198805
:1039F000BDE8104002F02CBF10B5044606206368F5
:103A0000198802F025FFE36808201988BDE81040F6
:103A100002F01EBF10B5044602206368198802F048
:103A200017FFE36804201988BDE8104002F010BFBA
:103A300070B50E4C84B01225042201230646039073
:103A4000029320468DE824001423102105F010FC79
:103A5000062209230293039601952046009214231F
:103A6000102105F005FC04B070BD00BF909CFF1F45
:103A70002DE9F041224D82B0012602B284B20092BB
:103A8000284601967823192105F038FB04F10C0231
:103A900012B28DE844002846A7197823192104F1B1
:103AA000020805F02BFB3FB20FFA88F819233A46BB
:103AB000284619460196CDF8008005F01FFB7823B3
:103AC0003A4628461946CDF80080019604F10A07C7
:103AD0000B3405F013FB3FB224B278233A46284654
:103AE00019468DE8500005F009FB192300943A4669
:103AF00001962846194605F001FB02B0BDE8F081A9
:103B0000909CFF1F2DE9F0411E4682B01446002A0A
:103B10006AD0099B4D4A00EBC305012C6F892989A6
:103B20006868A7EB010382FB03E21A444FEAE373E0
:103B3000C3EBA21302887BD0042C38D112FA83F392
:103B4000994203DC9F423946A8BF1946089A018072
:103B5000B6F90030BDF920803D48971D4FF0000EAA
:103B60003FB2194642460097CDF804E005F0C6FA88
:103B700029896A896B68521A1B885C2AA3EB0103A6
:103B800059DD03EB43030132C3EB431393FBF2F321
:103B900003F11B0213B20120328019464246019004
:103BA00000972B4805F0AAFA2A4B00221A702A4BDC
:103BB000022CB3F9001045D0082C31D100221A8014
:103BC00091422DD0089AB6F90030214806320124DE
:103BD00012B2009219460194BDF9202005F08EFA28
:103BE000204602B0BDE8F0811C4D1D4A2B681268CA
:103BF000CB1A93420F4617D9164A338811781448C6
:103C0000012918BF01241470089A06321BB212B29F
:103C10008DE814001946BDF9202005F06FFA2F60D9
:103C2000012002B0BDE8F081204602B0BDE8F0817D
:103C30009BB2D31A84E75C2101FB03F393FBF2F2FE
:103C40001B32A7E74A1C12B21A80B9E7C94216B262
:103C5000909CFF1F099DFF1F809CFF1F049DFF1F5D
:103C600048F0000030B583B000230C4605B2009345
:103C700026225B231C210C4804F090FF29460123D7
:103C80002622094804F09AFA002C24B205DB2146CA
:103C900001232622044804F091FA044A044B1580BB
:103CA0001C8003B030BD00BF909CFF1F268AFF1F01
:103CB000288AFF1FF0B59B4C237883B01BB19A4B29
:103CC0004FF6FF721A80994BB3F90030C3B9984A86
:103CD000954B1068B3F9002080F30C005B2303FBC5
:103CE00000F000131C3082425ED04FF0FF31FFF72E
:103CF000B9FF904804F0B6FF0023237003B0F0BD75
:103D0000012B36D0022B6ED0032B53D0042BF3D1D2
:103D1000252200258DE8240076231C218548864E27
:103D2000864F05F0EBF917E0B0F5AF7FA8BF4FF471
:103D3000AF70323803FB00F387FB0321DB17C3EBC3
:103D400061111C3109B201231D442522794804F078
:103D500035FA0C2D00F08480E9B2794804F0ECF8D3
:103D600056F8042B801A31284FF05B03DCDC1C2151
:103D7000E9E7744B1A68B2F52F7F32DB41F25C231E
:103D80009342A8BF1346A3F52F735B226E4802FB34
:103D900003F380FB0320DB17C3EBA0201C30624B36
:103DA000B3F900308342A0D1684BB3F9003001333E
:103DB0009BD1A1E7664B1B68B3F5FA7F11DBB3F526
:103DC0007A6FA8BF4FF47A63A3F5FA7261485B2358
:103DD00003FB02F380FB0320DB17C3EB20201C3026
:103DE000DDE71C20DBE75C4B1B68B3F5FA7F33DBB8
:103DF000B3F57A6FA8BF4FF47A63A3F5FA7255480A
:103E00005B2303FB02F380FB0320DB17C3EB2020C3
:103E10001C30524B1B68B3F5FA7F1FDBB3F57A6F8A
:103E2000A8BF4FF47A63A3F5FA724A495B2303FBF8
:103E300002F381FB0321DB17C3EB21211C313A4B39
:103E4000B3F9003083427FF452AF404BB3F90030F6
:103E50008B427FF44CAF4FE71C20DAE71C21EEE7E2
:103E6000262200258DE8240076231C2131483C4E73
:103E7000324F05F043F916E0B0F5AF7FA8BF4FF41D
:103E8000AF70323803FB00F387FB0321DB17C3EB72
:103E900061111C3109B201231D442622254804F07A
:103EA0008DF90C2D0CD0E9B22E4804F045F856F8E7
:103EB000042B801A31284FF05B03DDDC1C21EAE77C
:103EC000272200258DE8240076231C211948264E40
:103ED0001A4F05F013F917E0B0F5AF7FA8BF4FF404
:103EE000AF70323803FB00F387FB0321DB17C3EB12
:103EF00061111C3109B201231D4427220D4804F031
:103F00005DF9062D3FF4F5AEE9B2184804F014F857
:103F100056F8042B801A31284FF05B03DCDC1C219F
:103F2000E9E700BF769CFF1F268AFF1F7C9CFF1FCE
:103F3000009CFF1F909CFF1FDC89FF1F4B48371B15
:103F4000249BFF1FD49AFF1FD3058541288AFF1F9A
:103F5000149BFF1F011FB812209BFF1F689CFF1FAF
:103F60003089FF1F809BFF1F0C8AFF1FF89AFF1FDD
:103F70002DE9F04FDFF8EC82B74CB8F900604D78CE
:103F800054F8264087B08246039305B10D78DFF8D8
:103F9000FCB2002A34D19BF800308BBBAF4EB6F98F
:103FA0000000002800F0CE80012800F024810120CC
:103FB00032232A46019000935146A94B2046FFF731
:103FC000A1FD00250746B6F90030022B40F3F4802E
:103FD00000233380B8F90030A24A002BC0F2F880E9
:103FE000042BC4BF00231380039B002B40F0F680FA
:103FF000002D0CBF38464FF0FF3007B0BDE8F08F02
:10400000964EE3682268984804930027059237800B
:104010008BF8007004F01AFD1120FFF729FD4FF016
:10402000010919232821CDF8049000912422194672
:104030008D4805F063F8782328212422CDF80490D8
:1040400000918948194605F059F84946864805F017
:10405000EBFB02221921844805F0E2FBDDF8149005
:1040600048460AF04DFA494602467F4805F072FD7F
:104070007D4805F085FD394614227B4805F0D0FBCC
:1040800003227A49784805F065FD774805F078FD08
:1040900039462322744805F0C3FB03227449724851
:1040A00005F058FD704805F06BFD049B002B72D1A4
:1040B0000123704A18461370FFF7BAFC2089638900
:1040C0006768191A5C293A885BDC131A5C2202FBC8
:1040D00003F292FBF1F31B33674A63481380012715
:1040E0001BB21A2219468DE88400142205F006F846
:1040F000049BDBB1218A638AE768581A5C283A88F6
:104100006FDD521A02EB4202C2EB4212431C92FBD9
:10411000F3F31B33524A54481380012738221BB251
:104120008DE884001946322204F0E8FF534A544BCC
:10413000B6F90000012111704FF6FF721A800028B5
:104140007FF432AFDFF848914E4AD9F80030126858
:10415000C3EB0A0393424CD9464B1A78012A18BF85
:10416000012018700127FFF763FCC9F800A0012D9A
:104170004ED0042D59D0022D60D0082D64D00025DA
:1041800021E7121A02EB4202C2EB42124B1C92FBD5
:10419000F3F31B33A0E72F20FFF76AFC39463222E6
:1041A000314805F03DFB032237492F4805F0D2FC8A
:1041B0002D4805F0E5FC7BE77FF40CAFE368002BAE
:1041C0003FF406AFB8F90030264A002BBFF608AF1F
:1041D00004231380039B002B3FF40AAFFFF76AFD13
:1041E00006E7511A5C2202FB01F292FBF0F31B334B
:1041F00090E70746BBE7002714238DE888002A468E
:1042000051461D4B2046FFF77DFC3D460746DAE64A
:10421000B8F800308BF800500133A8F8003063691B
:1042200083B1002520469847CDE6B8F8003001223A
:10423000013BA8F800308BF80020F0E70123338021
:104240000025C7E61D46BEE66369002232804FF0B6
:10425000FF35002BE6D1BDE62C8AFF1F809CFF1F97
:104260007A9CFF1F7C9CFF1F909CFF1FD8ED0000D5
:10427000DCED0000099DFF1F789CFF1F769CFF1F4F
:10428000268AFF1F48F00000E0ED00007E9CFF1F23
:10429000049DFF1F01210D2006F026BB00210D20EB
:1042A00006F022BB01460D2006F01EBB08B50D200E
:1042B00006F020FBB0FA80F149090D20BDE8084066
:1042C00006F012BB10B5002144080D2006F00CFBCF
:1042D000204606F045FB0D20012106F005FB204697
:1042E000BDE8104006F03CBB08B5214A214B1288BE
:1042F0001868824234DA204B1B88991A8342A8BF7F
:104300000346B1F5F87FA3EB020321DAC3EB0313F5
:1043100003EB431393FBF1F105310A2006F054F946
:10432000164B1978F1B1164B16491B6883F3070336
:10433000C3EB031303EB431381FB03211944DB1786
:10434000C3EBA11105310920BDE8084006F03CB9D6
:10435000C3EB43131B01013193FBF1F10531DCE7A2
:104360000021DAE70920BDE8084006F02DB900BFBA
:10437000829BFF1FC89AFF1F4C9CFF1F409BFF1F83
:104380003C9CFF1F090402817F2838B5A8BF7F200D
:104390000D4D4FF4FA7303FB00F485FB0423234413
:1043A000E117C1EBA3110A2006F00EF9A4F578403D
:1043B0000C3885FB00310144C017A0EBA111BDE80A
:1043C0003840092006F000B909040281024B4E2052
:1043D000198802F03DBA00BF1C9BFF1F024B44200E
:1043E000198802F035BA00BF029BFF1F024B102054
:1043F000198802F02DBA00BFB49BFF1F024B2C207E
:10440000198802F025BA00BFF49AFF1F024B1E2044
:10441000198802F01DBA00BFF09AFF1FC3680E2072
:10442000198802F015BA00BF024B2820198802F043
:104430000FBA00BF089CFF1F024B6420198802F0CE
:1044400007BA00BF049CFF1F024B5A20198802F0D4
:10445000FFB900BFDC9AFF1F024B1620198802F03B
:10446000F7B900BFE49AFF1F024B2E20198802F013
:10447000EFB900BF749BFF1F024B3020198802F078
:10448000E7B900BFD09AFF1F024B1820198802F02D
:10449000DFB900BF869BFF1F024B1A20198802F06C
:1044A000D7B900BF269BFF1F024B1C20198802F0C2
:1044B000CFB900BF1E9BFF1F024B6620198802F078
:1044C000C7B900BF369CFF1F024B2020198802F09D
:1044D000BFB900BF349CFF1F024B3220198802F085
:1044E000B7B900BF269CFF1F024B6820198802F055
:1044F000AFB900BF589BFF1F024B6C20198802F018
:10450000A7B900BFCC9AFF1F024B6E20198802F09A
:104510009FB900BF749CFF1F024B5220198802F004
:1045200097B900BF6089FF1F024B5020198802F025
:104530008FB900BFD489FF1F024B5420198802F0A5
:1045400087B900BFD689FF1F024B5C20198802F093
:104550007FB900BF248AFF1F024B5E20198802F03A
:1045600077B900BF2C89FF1F024B6020198802F029
:104570006FB900BFA69BFF1F024B5620198802F09F
:1045800067B900BF6C9BFF1F38B5094D4624204614
:1045900002F078F935F8021B00B28842204601D0BB
:1045A00002F056F90234A4B24E2CF0D138BD00BF4F
:1045B0000C9CFF1F064B074A10B41C88064B08468C
:1045C000002C14BF11461946042210BC0AF056B83C
:1045D000389BFF1F08F500000CF50000064B074A4A
:1045E00010B41C88064B0846002C14BF114619460F
:1045F000042210BC0AF042B8769BFF1F08F50000A9
:104600000CF50000064B074A10B41C88064B084600
:10461000002C14BF11461946042210BC0AF02EB813
:10462000069CFF1F08F500000CF50000064B074A2A
:1046300010B41C88064B0846002C14BF11461946BE
:10464000042210BC0AF01AB8FA9BFF1F08F50000FC
:104650000CF50000064B074A10B41C88064B0846B0
:10466000002C14BF11461946042210BC0AF006B8EB
:104670007A9BFF1F08F500000CF5000070B5284E6E
:1046800005460FCE86B06C460FC496E8030044F88A
:10469000040B2320218005F011FC40F6B83398422A
:1046A00030DC204B40F6F50219889B78ADF80D10F0
:1046B00090428DF80F302DDD00EB40001A4B1B4966
:1046C0001B4E00EB0010C21783FB0043C2EB6323B9
:1046D00081FB0314D917C1EBA40101EB810186FB17
:1046E0000040C2EB6030A3EB4103303030338DF833
:1046F00011008DF8133069462846162209F0BEFFD6
:1047000006B070BD0B4B1A889B78ADF80D208DF864
:104710000F30D1E7084B1868CDF81100EBE700BF68
:1047200020F5000010F50000976A3E2B676666666C
:104730008BAA30451CF5000014F50000F8B5174CA5
:10474000174E2278174D33782F888E46003218BFC7
:10475000012201467046FFF70BFC0023984233709C
:10476000237015DB14BF012000202B889F420ED040
:1047700040F23A72A3F5AF730B490C4C02FB03F302
:1047800081FB0312DB17A3EB621332332360F8BD06
:104790000749012218460A702270E6E7B88BFF1F0E
:1047A000269DFF1F489CFF1FB5814E1BC489FF1F1C
:1047B000889CFF1F014B187801F0E2BF1C9DFF1F72
:1047C000014B187801F0F6BF108DFF1F134BB3F9A2
:1047D000003030B583EAE374A4EBE374002BA0B29D
:1047E00018DB012300E0134603EB830252009442DE
:1047F000F9DA0B4D90FBF3F285FB03E403FB1200A7
:10480000DB173032D3EBA40380B201F8012BF1D1D6
:104810000B7030BD2D230B700131E2E7108DFF1FAF
:1048200067666666144BB3F9003070B583EAE375CA
:10483000A5EBE375002BACB21ADB012300E00346C5
:1048400003EB830040008542F9DA0C4E94FBF3F051
:1048500086FB03E503FB1044DB173030D3EBA503E5
:10486000A4B201F8010BF1D105480B70106070BDC6
:104870002D230B700131E0E7DC9AFF1F6766666647
:1048800038F50000134BB3F9003030B583EAE37418
:10489000A4EBE374002BA0B218DB012300E0134665
:1048A00003EB830252009442F9DA0B4D90FBF3F2D2
:1048B00085FB03E403FB1200DB173032D3EBA403C8
:1048C00080B201F8012BF1D10B7030BD2D230B709C
:1048D0000131E2E76089FF1F67666666134BB3F933
:1048E000003030B583EAE374A4EBE374002BA0B28C
:1048F00018DB012300E0134603EB830252009442CD
:10490000F9DA0B4D90FBF3F285FB03E403FB120095
:10491000DB173032D3EBA40380B201F8012BF1D1C5
:104920000B7030BD2D230B700131E2E7D489FF1FDE
:1049300067666666134BB3F9003030B583EAE374FB
:10494000A4EBE374002BA0B218DB012300E01346B4
:1049500003EB830252009442F9DA0B4D90FBF3F221
:1049600085FB03E403FB1200DB173032D3EBA40317
:1049700080B201F8012BF1D10B7030BD2D230B70EB
:104980000131E2E7D689FF1F67666666134BB3F90C
:10499000003030B583EAE374A4EBE374002BA0B2DB
:1049A00018DB012300E0134603EB8302520094421C
:1049B000F9DA0B4D90FBF3F285FB03E403FB1200E5
:1049C000DB173032D3EBA40380B201F8012BF1D115
:1049D0000B7030BD2D230B700131E2E7248AFF1FDD
:1049E00067666666134BB3F9003030B583EAE3744B
:1049F000A4EBE374002BA0B218DB012300E0134604
:104A000003EB830252009442F9DA0B4D90FBF3F270
:104A100085FB03E403FB1200DB173032D3EBA40366
:104A200080B201F8012BF1D10B7030BD2D230B703A
:104A30000131E2E72C89FF1F67666666054B1B881C
:104A40001BB9054B186808607047044B186808606C
:104A5000704700BF1C9BFF1F40F500003CF50000A5
:104A6000164B1B880BB31BB230B583EAE374A4EB7F
:104A7000E374002BA0B21CDB012300E0134603EB20
:104A8000830252009442F9DA0D4D90FBF3F285FB5C
:104A900003E403FB1200DB173032D3EBA40380B234
:104AA00001F8012BF1D10B7030BD064B186808607E
:104AB00070472D230B700131DEE700BFF09AFF1F16
:104AC000676666660CF50000164B1B880BB31BB2BD
:104AD00030B583EAE374A4EBE374002BA0B21CDBD3
:104AE000012300E0134603EB830252009442F9DAFB
:104AF0000D4D90FBF3F285FB03E403FB1200DB1783
:104B00003032D3EBA40380B201F8012BF1D10B704A
:104B100030BD064B1868086070472D230B700131BB
:104B2000DEE700BF2A9CFF1F676666660CF5000083
:104B3000164B1B880BB31BB230B583EAE374A4EBAE
:104B4000E374002BA0B21CDB012300E0134603EB4F
:104B5000830252009442F9DA0D4D90FBF3F285FB8B
:104B600003E403FB1200DB173032D3EBA40380B263
:104B700001F8012BF1D10B7030BD064B18680860AD
:104B800070472D230B700131DEE700BFE49AFF1F51
:104B90006766666644F50000174B1B881BB31BB2A3
:104BA00070B583EAE375A5EBE375002BACB21EDBB1
:104BB000012300E0034603EB830040008542F9DA5D
:104BC0000E4E94FBF3F086FB03E503FB1044DB176A
:104BD0003030D3EBA503A4B201F8010BF1D10848A2
:104BE0000B70106070BD074B1868086070472D236C
:104BF0000B700131DCE700BF749BFF1F67666666C0
:104C000018F500000CF50000164B1B880BB31BB207
:104C100030B583EAE374A4EBE374002BA0B21CDB91
:104C2000012300E0134603EB830252009442F9DAB9
:104C30000D4D90FBF3F285FB03E403FB1200DB1741
:104C40003032D3EBA40380B201F8012BF1D10B7009
:104C500030BD064B1868086070472D230B7001317A
:104C6000DEE700BFD09AFF1F676666660CF500009E
:104C7000164B1B880BB31BB230B583EAE374A4EB6D
:104C8000E374002BA0B21CDB012300E0134603EB0E
:104C9000830252009442F9DA0D4D90FBF3F285FB4A
:104CA00003E403FB1200DB173032D3EBA40380B222
:104CB00001F8012BF1D10B7030BD064B186808606C
:104CC00070472D230B700131DEE700BF369CFF1FBC
:104CD000676666660CF50000174B1B881BB31BB29A
:104CE00070B583EAE375A5EBE375002BACB21EDB70
:104CF000012300E0034603EB830040008542F9DA1C
:104D00000E4E94FBF3F086FB03E503FB1044DB1728
:104D10003030D3EBA503A4B201F8010BF1D1084860
:104D20000B70106070BD074B1868086070472D232A
:104D30000B700131DCE700BF349CFF1F67666666BD
:104D400048F500000CF50000074B1B88022B06D02D
:104D5000012B0CBF054B064B186808607047054BCC
:104D600018680860704700BFA69BFF1F50F5000041
:104D700054F500004CF50000054B1B881BB1054B9A
:104D8000186808607047044B18680860704700BFD7
:104D90006C9BFF1F5CF5000058F5000038B5FCF770
:104DA00061FD0D4B1B7833B90C4B1020198801F0B5
:104DB0004FFD012038BD0A4D0A4C2B782288B3FAEA
:104DC00083F382F008025B09114642202B70228097
:104DD00001F03EFD002038BDE69AFF1FB49BFF1F87
:104DE0009C9BFF1F009BFF1F184B1A8852B3184A49
:104DF000128830B50A80B3F90030002B83EAE374DF
:104E0000A4EBE374BCBF2D238B70A0B2ACBF023106
:104E10000331012300E0134603EB83025200944266
:104E2000F9DA0C4D90FBF3F285FB03E403FB12006F
:104E3000DB173032D3EBA40380B201F8012BF1D1A0
:104E40000B7030BD044B186808607047269BFF1F2D
:104E500060F50000676666660CF5000010B40A4B4A
:104E60000A4C0A4693E8030083B0238802AC04E9A5
:104E7000030004EB8303104653F8081C052203B01B
:104E800010BC09F0FBBB00BF68EE0000049CFF1FD4
:104E9000F0B40C4D0C4F0E460FCD8CB001AC0FC4CE
:104EA0000FCD0FC495E807003B8884E807000CAAE3
:104EB00002EB8303304653F82C1C04220CB0F0BCE8
:104EC00009F0DCBB70EE0000F09BFF1FF0B40A4D50
:104ED0000A4F0E460FCD86B001AC0FC42A683B883E
:104EE000226006AA02EB8303304653F8141C042206
:104EF00006B0F0BC09F0C2BB9CEE0000869BFF1F11
:104F0000F0B40A4D0A4F0E460FCD86B001AC0FC467
:104F10002A683B88226006AA02EB8303304653F8D6
:104F2000141C0C2206B0F0BC09F0A8BBB0EE0000C7
:104F30001E9BFF1F164B1B880BB31BB283EAE3704B
:104F4000A0EBE370002B30B584B21DDB012300E041
:104F5000134603EB830252009042F9DA0D4894FBAA
:104F6000F3F280FB03E503FB1244DB173032D3EB93
:104F7000A503A4B201F8012BF1D10B7030BD084696
:104F80000422054909F07ABB2D230B700131DDE7BE
:104F9000589BFF1F6766666664F50000F0B40A4D13
:104FA0000A4F0E460FCD86B001AC0FC42A683B886D
:104FB000226006AA02EB8303304653F8141C042235
:104FC00006B0F0BC09F05ABBC4EE0000CC9AFF1F3B
:104FD00070B53C4D2B780646002B35D11C467378B6
:104FE0000BB9204670BDFCF73DFC374A374B3848BB
:104FF000127831781B78007802EB43034A1E03EBEA
:1050000080030E2AEDD801A050F822F07550000060
:1050100097500000E34F000075500000E34F000080
:10502000E34F0000E34F000063500000E34F000037
:10503000E34F0000E34F0000E34F0000E34F0000A8
:10504000E34F00005F500000AE21224803F0AEFAAB
:10505000204803F0FBFC00232B700124BFE705F080
:1050600091FFAF211B4803F0A1FA1B4A01231370E3
:105070002B70B6E783B91948038804294FF6FF71EE
:1050800003F1FF320CBF01230B46134403F07F03EF
:10509000013303800FE073B1013B114A32F8133042
:1050A0004BB10E4E0F481049104A338001230026A1
:1050B00006700B701370084A0221012311702B70C7
:1050C000204670BDB88BFF1F399CFF1F3A9CFF1F05
:1050D0003B9CFF1F909CFF1F889CFF1FC89BFF1FCE
:1050E0008C9BFF1F509BFF1FE79AFF1FFC9CFF1F1D
:1050F00010B5064B064C1A882046012101F096FB9C
:1051000021884220BDE8104001F0A2BB389BFF1F60
:10511000009BFF1F10B5064B064C1A882046022143
:1051200001F084FB21884220BDE8104001F090BBD3
:10513000769BFF1F009BFF1F10B5064B064C1A887D
:105140002046052101F072FB21884220BDE8104075
:1051500001F07EBB069CFF1F009BFF1F10B5064B96
:10516000064C1A882046002101F060FB218842206D
:10517000BDE8104001F06CBBFA9BFF1F009BFF1FB6
:1051800008B5122001F07EFB054B1988884206D035
:10519000122001F05DFBBDE8084001F071BA08BDC6
:1051A000F09BFF1F08B5582001F06CFB054B1988D8
:1051B000884206D0582001F04BFBBDE8084001F0C2
:1051C0005FBA08BD2A9CFF1F08B5142001F05AFBE6
:1051D000054B1988884206D0142001F039FBBDE840
:1051E000084001F04DBA08BD7A9BFF1FF0B480EA79
:1051F000E075A5EBE0750028ACB21FDB1DBF2B23CB
:105200000B704E1C0E46012300E0134603EB830295
:1052100052009542F9DA0B4F94FBF3F287FB03053A
:1052200003FB1244DB173032D3EBA503A4B206F81C
:10523000012BF1D133700846F0BC70472D230B7061
:105240004E1CE0E767666666084B188828B10D2893
:1052500007D00D3800B2FFF7C9BF054A10680860D3
:105260007047044A10680860704700BF749CFF1FB5
:105270000CF5000068F50000144B18880C2811D0BC
:10528000192813D01A2815D01B2817D01C2819D07C
:105290001D2803D00C3800B2FFF7A8BF0C4A1068D5
:1052A000086070470B4A1068086070470A4A106827
:1052B00008607047094A106808607047084A10681B
:1052C00008607047074A106808607047269CFF1FF7
:1052D00080F500006CF5000070F5000074F500002A
:1052E00078F500007CF50000034B1888A0EB8000E7
:1052F000400000B2FFF77ABF1C9DFF1F024B1888C9
:10530000033800B2FFF772BF089CFF1F024B1888DA
:105310000C3800B2FFF76ABFDE9AFF1F024B1888F5
:10532000183800B2FFF762BF029BFF1FC3681888DE
:10533000183800B2FFF75ABF30B5134C85B00125BD
:105340002B463C2202212046009503F0A5F9204679
:1053500003F07CFB00224021802320460191009332
:1053600011460A4B029504F01FF8204603F07AFC20
:1053700007480849084A0023036083800B608B803C
:105380001360938005B030BD909CFF1F08F10000B2
:10539000F49CFF1F209DFF1F0C9DFF1F10B500EB0D
:1053A000C00000F10F02D2B293B284B09C1E981CD0
:1053B0003D2303918DE819003921024803F058FF7D
:1053C00004B010BD909CFF1F014B01221A70704762
:1053D000269DFF1FF0B585B05C4C5D4B02935D4A86
:1053E00001920423009320465B4B5C4F5C4E5D4D65
:1053F0004022802102F058FF20465B4A5B495C4C0A
:1054000008F0BCFA5B485C4987615C4FC7615C4F40
:105410008F615C4A5C4FCF615C4F97615C4B5D4F25
:10542000D7615D4F9F615D4FDF615D4FB7615D4F3C
:10543000F7615D4FAF615D4FEF615D4FA7615D4803
:105440005D4FE7615D4F87615D495E4FC7615E4FAC
:105450008F615E4A5E4FCF615E4F5F4B97615F4FDA
:10546000D7615F4F5F4E9F615F4FDF615F4F604D60
:10547000B761604FF761604F604CAF61604FEF61A3
:10548000604F6148A761614FE761614F6149876182
:10549000614FC761614F624A8F61624FCF61624F56
:1054A0009761624B624FD761624F9F61624E634F5B
:1054B000DF61634FB761634D634FF761634FAF6166
:1054C000634C644FEF61644FA7616448644FE761C8
:1054D000644F87616449654FC761654F8F61654A55
:1054E000654FCF61654F9761654B664FD761664FDA
:1054F0009F61664E664FDF61664F674DB761674FCC
:10550000F761674F674CAF61674F68486849EF6163
:10551000684F694DA761E561684F694D694CDFF8D7
:10552000C8E1694A694B8761C5618C61684E694F02
:10553000694D6A4CC1F81CE069486A499761D561B8
:105540009C61D861B16005B0F0BD00BF909CFF1FA9
:10555000A0860100801A0600AC8FFF1F0D530000CB
:10556000C88CFF1F988EFF1F1C89FF1F018300003E
:10557000288FFF1FEC8CFF1F948BFF1F1D44000022
:10558000FD520000D88BFF1F29440000B5450000E4
:10559000808DFF1FF1500000DD4500001551000017
:1055A00005460000395100005D4E000039440000FE
:1055B0002D460000888AFF1F5D510000E95200005F
:1055C000148DFF1FB5470000CD470000308EFF1F30
:1055D000C1470000914E0000388CFF1F8151000030
:1055E000C94A0000808CFF1FA5510000254800001B
:1055F000DC8AFF1F4944000055460000708FFF1FE2
:10560000C9510000314B00005C8CFF1F5944000061
:10561000994B0000008BFF1F69440000094C0000FB
:10562000BC8EFF1F79440000CD4E0000708BFF1F21
:1056300089440000E94D00005C8DFF1F9944000083
:10564000014F0000E08EFF1FA9440000714C0000D4
:10565000A48CFF1FB9440000D94C0000548EFF1FDA
:10566000C944000079520000048FFF1FD944000094
:10567000354F0000408AFF1FE94400009D4F0000A5
:10568000FC8BFF1FF944000049520000248BFF1FD0
:105690000945000085480000AC8AFF1F194500003D
:1056A000DD480000648AFF1F29450000E88DFF1FC8
:1056B0000C8EFF1F35490000394500008D49000060
:1056C00049450000E54900004C8FFF1F388DFF1F42
:1056D000D08AFF1F494D000069450000794D000048
:1056E00079450000595A0000594500002DE9F04F56
:1056F0002F4DDFF8CCB0DFF8C4A0DFF8C8900FCD95
:1057000091B003AC0FC40FCD0FC40FCD0FC42B68E5
:1057100023600025A8462F462E4600E09846BAF89A
:10572000003024495BF8232028461123FBF740F979
:1057300000EBC00400EB840089FB00340444C01774
:10574000C0EB6434C4F13C00C6F13C0207F14101F6
:10575000012600B208F1410300901BB2019612B27B
:1057600009B2154803F0CAFC08EB060305F211154F
:105770003C2B2646ADB24746D0D134226B210E4891
:1057800004F04EF800210C4804F04EF80B4B1B8837
:1057900010AA02EB830353F8344C204608F0B0FE05
:1057A00002460548214611B0BDE8F04F04F0D2B9D9
:1057B000D8EE000048EB0000909CFF1FF49AFF1FFA
:1057C00060EA0000090002802DE9F043804685B0C0
:1057D000002956D10121304804F026F82F4998F8C5
:1057E000062098F8083011F80290994522DA4FEA1D
:1057F00089064D460C24D8F80C3027489B595F6821
:1058000022B2002104F00CF8384608F079FE39463F
:105810000246214804F09EF91F4804F0B1F998F8B7
:10582000083001350934AB42A4B206F1040601DDAB
:10583000422CE0D1B9F1000F13D109F106099945C5
:105840000CDA3C2301213B22039102930093019245
:1058500039233F223A21104803F00AFD05B0BDE884
:10586000F0830F2301213B220391029300930192C5
:1058700039230C223A21084803F0FAFC98F8083042
:10588000DBE700213423009301913F230C220248DF
:1058900003F002FC9EE700BF909CFF1F209DFF1FAE
:1058A00010B5104C0121204603F0C4FF2046012111
:1058B00003F0BAFF20463422552103F0B1FF204601
:1058C0000222094904F046F920460522074904F05E
:1058D00041F9204604F054F92046BDE8104003F099
:1058E000C1B900BF909CFF1F84F5000088F500003F
:1058F00070B50D46064608F003FE00EB400084003C
:10590000002D36D0284608F0FBFD00EB400040009B
:1059100023185B1003F16001091A282209B2174805
:10592000C3F1600403F07CFF0121144803F07CFF05
:10593000284608F0E5FD29460246104804F00AF919
:105940000E4804F01DF902210C4803F06DFF21B24E
:1059500021220A4803F064FF304608F0D1FD3146A9
:105960000246064804F0F6F80448BDE8704004F02A
:1059700007B96410C4F16004E5E700BF909CFF1F05
:10598000214B70B5B3F9003083EAE374A4EBE37400
:10599000002B82B0A1B22FDB68466D46012300E0E8
:1059A000134603EB830252009442F9DA174E91FB3F
:1059B000F3F286FB03E403FB1211DB173032D3EB67
:1059C000A40389B205F8012BF1D119462B70FFF71A
:1059D0008FFF0F4B1B786BB101210E4803F024FFA2
:1059E000332274210B4803F01BFF01220A490948A6
:1059F00004F0B0F802B070BD2D238DF800300DF129
:105A000001056846CAE700BFB49BFF1F676666666C
:105A10009C9BFF1F909CFF1F78F8000010B50D4B5A
:105A20001B5C51F82340237884B013B1012004B0EB
:105A300010BD04AA01A942F8103D2046A369984769
:105A4000A38A9B07F2D401A80099FFF751FF012018
:105A500004B010BDF49CFF1FF8B51F4D287840B965
:105A60001E4B1B68994203D31D4A012313702B70F0
:105A7000F8BD0C4600261B48184F02F0E7FF04F65D
:105A8000B833324617483B6031212E7003F0C8FE10
:105A90000121144803F0CEFE3146124803F0C4FE43
:105AA000052211490F4804F055F80E4804F068F833
:105AB0000C2210210B4803F0B3FE0B220B490948BE
:105AC00004F048F805220A49064804F043F805485E
:105AD00004F056F80120F8BDB88BFF1FF09CFF1FA3
:105AE000889CFF1F909CFF1F90F5000098F5000018
:105AF00088F5000010B5424C424882B002F0A6FF83
:105B00002378C3B906213F4803F08EFE2378012B8A
:105B100037D90A22022B11463A486BD003F080FE97
:105B200039490322374804F015F8364802B0BDE879
:105B3000104004F025B8354B1A7801210523002ABE
:105B400035D10191009311462E4803F027FB304BCD
:105B50001A78002A36D005230122019200930022F0
:105B60000A21284803F098FA2A4B1A78002A35D1DE
:105B700001210523019100931421224803F00EFB1B
:105B8000C0E7254C2388092B32D9632B8CBF0A210F
:105B90001F210A221B4803F043FE2188194804F004
:105BA0003FF8184802B0BDE8104003F0E9BF0022FA
:105BB000019100931146134803F06EFA144B1A78C2
:105BC000002AC8D105230121019100930A210D4823
:105BD00003F0E4FA0F4B1A78002AC9D001220523FA
:105BE0000192009300221421064803F055FA89E738
:105BF0003021CEE703F014FE0322084992E700BFEC
:105C0000FC9CFF1F909CFF1FA8F50000399CFF1F04
:105C10003A9CFF1F3B9CFF1FC89BFF1FA4F5000081
:105C20002DE9F041754C2278002A05460F4614BF35
:105C30004FF001084FF000084ED1714E3368CB1A77
:105C4000B3F5FA6F04D86B78A3B94046BDE8F0818C
:105C50006C4B6D486D49DFF8D0E11A700123037079
:105C60000988237026208EF8002000F0F1FD6B7863
:105C7000002BEAD03760FBF7F5FD654A654B6649B6
:105C8000127828781B78097802EB4303421E03EB55
:105C900081030E2AD9D801A151F822F08D5D0000B0
:105CA000595D00004B5C00008D5D00004B5C000006
:105CB0004B5C00004B5C0000415D00004B5C000051
:105CC000F35C00004B5C00004B5C00004B5C000090
:105CD0004B5C0000EF5C0000AF215048484E02F0E2
:105CE00065FCFFF707FF002337602370ABE705F083
:105CF00049F94A4802F0AAFE0221484803F094FDFF
:105D00000F222321454803F08BFD052244494348D7
:105D100003F020FF414803F033FF1E2223213F48B8
:105D200003F07EFD05223F493C4803F013FF3B484A
:105D300003F026FF394802F095FF00F0ADFC84E740
:105D4000394D2B78012B50D9304B2620198800F083
:105D50007FFD00232B7078E7002B3FF476AF013BEB
:105D6000324A32F81330002B3FF46FAF274C3048E3
:105D700025492D4A23804FF001080023037081F844
:105D8000008082F80080FFF7B5FE5EE793B1013B2B
:105D9000264A32F8131019B31C4B254D1A4C224ACF
:105DA00019800026012326202E702370137000F026
:105DB0004FFD15E0154C1E4922880B7004284FF644
:105DC000FF7002F1FF310CBF012202460A440E4E61
:105DD000154D02F07F0201320121228031702B70BB
:105DE000FFF788FE4FF001082FE70649064A012316
:105DF0000020087013702370A6E700BFB88BFF1F48
:105E0000189DFF1F889CFF1FE79AFF1FC89BFF1F5D
:105E1000399CFF1F3A9CFF1F3B9CFF1F909CFF1F5C
:105E2000ACF50000B4F50000FC9CFF1F8C9BFF1F2D
:105E3000509BFF1F2DE9F04F05468BB00F46AD4834
:105E40000121164603F0F6FCAA8812F0010440F086
:105E5000B080DFF8CC8298F80030002B7DD1AB7990
:105E6000A54AD15CA1B9DFF8BCA279781AF80390F1
:105E700041B339780139072900F2B780DFE811F022
:105E8000F1005401B5006C01B500B500B500E900A2
:105E90007C78002C00F0CA800139EC68387854F81E
:105EA0002170FC68411EB4F80080072900F2A78029
:105EB000DFE811F074015901A5006C01A500A500EF
:105EC000A5009F00DFF854A2DAF80020B21AB2F55C
:105ED000967F75D9894A107801281ABF0120107061
:105EE0001170874A18BF0146D05CC0EB0900C0B2F0
:105EF000FFF754FA0124CAF80060AB889B0770D5FD
:105F00007B78002B6DD0FBF7ADFC7E4B7E4A7F4843
:105F10001B78127839780078022515FB02330A299C
:105F200003EB800300F04E810C295AD1002B58D08E
:105F300003F11900764E774A013B0021400080B200
:105F400026F813100123157088F8003000F080FC4B
:105F5000714B032220461A702FE0664802F076FD4E
:105F60000121644803F060FC62482246214603F0A8
:105F700057FCAB88580725D42C68204608F0C0FA97
:105F8000214602465B4803F0E5FD5A4803F0F8FD60
:105F9000092201238DE80C0000217F23554803F0DE
:105FA000ADF800212846FFF70FFC002388F80030E9
:105FB00055E7AB683146384698470BB0BDE8F08FDF
:105FC0000846FAE72B6804A8984704A808F098FA4E
:105FD00004A90246474803F0BDFD464803F0D0FD42
:105FE000D6E720460BB0BDE8F08F00240AF80390F6
:105FF00083E70021D1543846FB699847FC68A4F830
:106000000080002725223C238DE8840041211822AE
:10601000384803F041F8E968A879FFF7FFFC374AF0
:106020003E4B17701E600BB0BDE8F08F3B490A680D
:10603000B21AB2F5967FD4D9304F0E603E78012E59
:1060400000F0B480E968184601233B70FFF7E6FCD6
:10605000B3E7304AE9791170012288F80020002462
:10606000C4E72A7A013A4A45BFDD09F10104E4B2E6
:10607000A145BAD0224E16F803B0CBEB0900C0B24E
:106080000021FFF78BF92B7A052BD9461BD9CBEBD7
:106090000402042A40F3AE80A4F1040BBBF1000F0C
:1060A000C0F2B080063B5B45A8BF5B465FFA83F950
:1060B000AA791348B15C994205D000F802900121F9
:1060C0002846FFF781FBC9EB0400C0B201210B4E4B
:1060D000FFF764F9002134230191009305483170E2
:1060E00040230B223F21A14602F0D6FF0124AB79C9
:1060F0007CE700BF909CFF1F0C9DFF1F099DFF1FA9
:10610000209DFF1F399CFF1F3A9CFF1F3B9CFF1FD8
:106110008C9BFF1F889CFF1FFC9CFF1F049DFF1F83
:10612000B88BFF1FF49CFF1F0FFA89F1E868604CE1
:1061300050F821602168049134785E490498086021
:10614000002C71D0012C7FF450AF5B4A317A88F873
:1061500000401170002449E7B9F1000F50D009F157
:10616000FF34E4B284E7B98A01F0040189B200295E
:106170003FF440AF3B6A03929847039A00283FF4EC
:106180003DAFAB79FC680021D15438E77B8A4345A9
:106190003CD908F101081FFA88F830E73B8A4345EB
:1061A0003BD208F1FF381FFA88F828E725238DE84D
:1061B000180042483C703C231822412102F06CFF39
:1061C0003046FAE6002B3FF40CAF3D4A3D4E1188B5
:1061D000394A03F11900013B400080B226F8131040
:1061E000012388F80030157000F032FB364B204652
:1061F0001D70E2E6002A3FF755AF04F1FF3B4DE783
:106200004C46F3E64FF000094B4651E7BB8ADA07EC
:106210007FF5F5AEB7F81080F1E6BB8AD9077FF5B8
:10622000EEAEB7F81280EAE62849C85CC0EB090078
:1062300009F1010EC0B201214FF0340B02F803E066
:10624000FFF7ACF8B6681D48019440230B223F21AC
:106250000124CDF800B002F01FFF40230B223F21A4
:106260001648CDF800B0019402F098FF214613487B
:1062700003F0DAFA304608F043F9A0EB800000F1B1
:106280005F0109B20F220D4803F0CAFA304608F048
:1062900037F931460246094803F05CFC074803F031
:1062A0006FFCE968A879FFF7B9FBAB799EE600BF00
:1062B0005C9DFF1F049DFF1F889CFF1F909CFF1F7C
:1062C000C89BFF1F8C9BFF1FFC9CFF1F209DFF1F77
:1062D0002DE9F047DFF808926D4B99F800601B68D4
:1062E000DFF800A282B0003601934FF0030018BF20
:1062F0000126019F9AF8008004F0FCFA054604206C
:1063000004F0F8FA0446052004F0F4FA800040EAAC
:106310004404062004F0EEFA2C4364B25D4944EADA
:10632000C0000A7880F00F03DBB29A425A4A3CD090
:106330001760002259480B7003788DF800808DF8A3
:10634000012053B3564A12684EF66021BA1A8A42A7
:1063500019D8022B59D0012B5FD0062B48D0032B24
:1063600063D0042B69D0052B77D0072B7DD0082B69
:1063700000F08380092B68D016B14A4802F072FC05
:1063800002B0BDE8F087484A484C00230121237041
:1063900003701360938089F800103A4669464448B8
:1063A000FFF748FD3043C6B2E6E71268BA1A1E2A64
:1063B0006BD99AF80020934222D0394C3D488AF894
:1063C0000030012B276082EA030207609846B1D0B3
:1063D000042BAFD137480068381AB0F5C87FA9D967
:1063E000354C2068381A3228A4D927601A46A1E70C
:1063F0003A4669463148FFF71DFD3043C6B2BBE758
:10640000012B4FF00002E3D1E4E73A4669462C48FD
:10641000FFF710FD3043C6B2AEE73A466946294859
:10642000FFF708FD3043C6B2A6E73A46694626485C
:10643000FFF700FD3043C6B29EE73A46694623485F
:10644000FFF7F8FC3043C6B296E73A466946204863
:10645000FFF7F0FC3043C6B28EE73A4669461D4866
:10646000FFF7E8FC3043C6B286E73A4669461A4869
:10647000FFF7E0FC3043C6B27EE73A46694617486C
:10648000FFF7D8FC3043C6B276E7002252E700BFE0
:106490005C9DFF1F089DFF1F849CFF1F889CFF1FA2
:1064A000009DFF1F909CFF1F0C9DFF1FFA9CFF1F6C
:1064B000FCF00000149DFF1F8C9CFF1F5CF000008F
:1064C0006CF000004CF000000CF0000094F00000B4
:1064D00078F0000018EF0000C8F00000D08AFF1F1D
:1064E000B88BFF1FFB9CFF1F28B11028044BA8BFCF
:1064F000102018607047024B01201860704700BFE1
:10650000289DFF1F38B50F4D2B78013B01381B022A
:10651000C4B203F47063200443F4404343F00C031B
:1065200000F4FE00184305F04DFB2868013860F0C8
:106530003F00C0B204F074FB2046BDE8384004F0D0
:106540006FBB00BF289DFF1F70B5124D2B78013B1C
:106550001B0203F47063064643F43043080632041A
:1065600000F0FE4043F00B03034302F4FE00184327
:106570000C4605F027FB2868013860F04F00C0B2D8
:1065800004F04EFB304604F04BFB2046BDE8704063
:1065900004F046BB289DFF1F70B5124D2B78013BC0
:1065A0001B0203F47063064643F4104308063204EA
:1065B00000F0FE4043F00903034302F4FE001843D9
:1065C0000C4605F0FFFA2868013860F06F00C0B291
:1065D00004F026FB304604F023FB2046BDE8704063
:1065E00004F01EBB289DFF1F38B5104D2B78013BD2
:1065F0001B0203F47063044643F41043000443F0A9
:10660000090300F4FE00184305F0DCFA286801389D
:1066100060F06F00C0B204F003FB204604F000FB02
:106620000020BDE8384004F0FBBA00BF289DFF1FE2
:1066300038B50E4D2B78013B1B0203F47063044602
:1066400043F45043000443F00D0300F4FE001843EC
:1066500005F0B8FA2868013860F02F00C0B204F0E5
:10666000DFFA2046BDE8384004F0DABA289DFF1F63
:1066700008B5002005F070FB0028FAD108BD00BF66
:1066800008B564210720FFF75FFF7F210B20BDE8DD
:106690000840FFF759BF00BF10B500217B20FFF76E
:1066A00053FF0024E0B2FFF79FFF0134022004F003
:1066B00057F9802CF6D110BD10B504464FF4406058
:1066C00004F05EFA04F0B6FA2CB1102C044BA8BF0B
:1066D00010241C6010BD024B01241C6010BD00BFC3
:1066E000289DFF1F10B5044641F0E00004F098FA21
:1066F00004F07F0004F094FAC4F3C610BDE8104023
:1067000004F08EBA38B5134D2B78044641F6FF726B
:10671000A0F50050824203F1FF33A8BF02461B02DE
:1067200002F5005203F47063100443F4604343F035
:106730000E0300F4FE005204184302F0FE42104320
:1067400005F040FA296801392046C9B2BDE8384051
:10675000FFF7C8BF289DFF1F38B504460D46F0203F
:1067600004F05EFA35B1254414F8010B04F058FA30
:10677000AC42F9D1F720BDE8384004F051BA00BF6F
:1067800000B50B4B83B00246998818680090032A25
:10679000ADF8041002D903B05DF804FB6846062189
:1067A0008DF80520FFF7D8FF03B05DF804FB00BFAC
:1067B000D0F8000000B50B4B024683B018689988EA
:1067C0000090131F4C2BADF8041002D903B05DF8F4
:1067D00004FB684606218DF80520FFF7BDFF03B0D6
:1067E0005DF804FBD8F80000030203F4FE43C0F395
:1067F000C6101843704700BF03784078DB0103F4EC
:106800007E5300F07F001843704700BF82B002AA99
:10681000114642F8040D002012F8013B03F07F03FB
:10682000914243EA0020F7D102B07047003210B421
:1068300003884FF0010404FA01F418BF012202FAA0
:1068400001F123EA04020A43028010BC704700BF32
:1068500070B5CEB20C46054603F014FC864203D058
:106860003146284603F028FC0135284603F00AFC8F
:10687000240A844205D021462846BDE8704003F032
:106880001BBC70BD38B5054603F0FCFB4FF000049F
:1068900060F30704681C03F0F5FB60F30F24A0B25B
:1068A00038BD00BFF8B504460020FFF7EBFF002C11
:1068B00000F0A6834FF4AF610220FFF7C9FF4FF449
:1068C0007A610420FFF7C4FF4FF496610620FFF7BA
:1068D000BFFF4FF4FA610820FFF7BAFF4FF4AF6132
:1068E0000A20FFF7B5FF40F6FC010C20FFF7B0FFD0
:1068F0004FF496612220FFF7ABFF4FF4166124207E
:10690000FFF7A6FF7D212A20FFF7A2FF0C210E2012
:10691000FFF79EFF01211020FFF79AFF02211220AE
:10692000FFF796FF00211420FFF792FF00211620A9
:10693000FFF78EFF02211820FFF78AFF01211A209E
:10694000FFF786FF02211C20FFF782FF04211E2093
:10695000FFF77EFF14212020FFF77AFF0121262078
:10696000FFF776FF03212820FFF772FF04212C2078
:10697000FFF76EFF0F212E20FFF76AFF0021302066
:10698000FFF766FF0C213220FFF762FF0021342061
:10699000FFF75EFF00213620FFF75AFF0021382065
:1069A000FFF756FF00213A20FFF752FF00213C205D
:1069B000FFF74EFF00213E20FFF74AFF0021402055
:1069C000FFF746FF00214220FFF742FF1F2144202E
:1069D000FFF73EFF13214620FFF73AFF0E21482024
:1069E000FFF736FF11214A20FFF732FF0A214C2022
:1069F000FFF72EFF00214E20FFF72AFF062150202F
:106A0000FFF726FF02215220FFF722FF0C2154201E
:106A1000FFF71EFF00215620FFF71AFF0021582024
:106A2000FFF716FF01215A20FFF712FF03215C2018
:106A3000FFF70EFF0A215E20FFF70AFF002160200A
:106A4000FFF706FF04216220FFF702FF0121642007
:106A5000FFF7FEFE00216620FFF7FAFE0B216820FB
:106A6000FFF7F6FE7F216A20FFF7F2FE00216C207F
:106A7000FFF7EEFE00216E20FFF7EAFE2221002044
:106A8000FFF7E6FE0220FFF7FDFEB0F5805F03464C
:106A900080F0DA83D24A04201380FFF7F3FEB0F5CA
:106AA000805F034680F0C883CE4A06201380FFF73C
:106AB000E9FEA0F52F739BB2B3F57A6F024606D9B3
:106AC00040F628210620FFF7C3FE40F62822C64BD9
:106AD00008201A80FFF7D6FEA0F52F739BB2B3F5FE
:106AE0007A6F024606D940F6E4410820FFF7B0FE6F
:106AF00040F6E442BD4B0A201A80FFF7C3FEA0F522
:106B0000FA739BB240F6AC518B42024606D94FF461
:106B1000AF610A20FFF79CFE4FF4AF62B44B0C202C
:106B20001A80FFF7AFFEA0F5FA739BB240F6AC51A6
:106B30008B42024606D940F6FC010C20FFF788FE86
:106B400040F6FC02AB4B0E201A80FFF79BFE182884
:106B5000034600F26B83A84A10201380FFF792FED1
:106B6000431E9BB20F2B024604D901211020FFF7D0
:106B70006FFE0122A14B12201A80FFF783FE0A2824
:106B8000034600F24D839E4A14201380FFF77AFEDD
:106B90000128034604D900211420FFF759FE0023E1
:106BA000984A16201380FFF76DFE7F28034600F2F7
:106BB0003183954A18201380FFF764FE04280346AA
:106BC00000F22283914A1A201380FFF75BFE0C2803
:106BD000034600F2E4828E4A1C201380FFF752FE27
:106BE0000428034600F2D5828A4A1E201380FFF74C
:106BF00049FE0928034600F2C682874A20201380F6
:106C0000FFF740FE4628034600F2B782834A22205F
:106C10001380FFF737FEA0F5FA739BB240F6AC5134
:106C20008B42024606D94FF496612220FFF710FEF0
:106C30004FF496627A4B24201A80FFF723FEA0F5CA
:106C4000FA739BB240F6AC518B42024606D94FF420
:106C500016612420FFF7FCFD4FF41662714B2620CD
:106C60001A80FFF70FFE7F28034600F280826E4AEB
:106C700028201380FFF706FE0628034600F27182E3
:106C80006A4A2A201380FFF7FDFDA0F132039BB270
:106C9000B3F5967F024604D97D212A20FFF7D8FD5F
:106CA0007D22634B2C201A80FFF7ECFD0C28034655
:106CB00000F251825F4A2E201380FFF7E3FD1E2869
:106CC000034600F242825C4A30201380FFF7DAFD6F
:106CD0000928034600F23382584A32201380FFF716
:106CE000D1FD1D28034600F22482554A342013802A
:106CF000FFF7C8FD7F28034600F21582514C36206D
:106D00002380FFF7BFFD7F28034600F2068238206C
:106D10006380FFF7B7FD7F28034600F2F8813A2031
:106D2000A380FFF7AFFD7F28034600F2EA813C20F5
:106D3000E380FFF7A7FD7F28034600F2DC813E20B9
:106D40002381FFF79FFD7F28034600F2CE8140207C
:106D50006381FFF797FD7F28034600F2C081422040
:106D6000A381FFF78FFD384D28804420FFF78AFD6F
:106D70003028034600F2AD81344A46201380FFF7E5
:106D800081FD3028034600F29E81314C482023804B
:106D9000FFF778FD3028034600F28F814A20638098
:106DA000FFF770FD3028034600F281814C20A3805C
:106DB000FFF768FD3028034600F273814E20E38020
:106DC000FFF760FD0128034604D900214E20FFF79C
:106DD0003FFD00231F4A50201380FFF753FD3BE087
:106DE000829BFF1F4C9CFF1F3A9BFF1F249CFF1F91
:106DF000FE9BFF1F089BFF1FDE9AFF1FB49BFF1F18
:106E0000F09BFF1F7A9BFF1FE49AFF1F869BFF1FCB
:106E1000269BFF1F1E9BFF1FF09AFF1F349CFF1F26
:106E2000E09AFF1FAA9BFF1FC89BFF1F089CFF1F24
:106E3000489CFF1FF49AFF1F749BFF1FD09AFF1FEF
:106E4000269CFF1F8C9BFF1F009BFF1F029BFF1FA9
:106E50000C9CFF1F1C9BFF1F431E9BB20B2B02466B
:106E600004D906215020FFF7F3FC0622CF4B522015
:106E70001A80FFF707FD0428034600F20C81CC4A74
:106E800054201380FFF7FEFC431E9BB21D2B0246CD
:106E900004D90C215420FFF7DBFC0C22C54B5620F3
:106EA0001A80FFF7EFFC0128034604D90021562081
:106EB000FFF7CEFC0023C04A58201380FFF7E2FC06
:106EC0007F28034600F2E180BC4A5A201380FFF776
:106ED000D9FC431E9BB2092B024604D901215A203A
:106EE000FFF7B6FC0122B64B5C201A80FFF7CAFC04
:106EF000431E9BB2102B024604D903215C20FFF7EE
:106F0000A7FC0322AF4B5E201A80FFF7BBFC431E99
:106F10009BB21D2B024604D90A215E20FFF798FC84
:106F20000A22A94B60201A80FFF7ACFC0228034616
:106F300000F2A580A54A64201380FFF7A3FC012876
:106F4000034604D901216420FFF782FC0123A04AF3
:106F500062201380FFF796FCC31E9BB2012B0246F2
:106F600004D904216220FFF773FC0422994B6620A8
:106F70001A80FFF787FC7F2803467AD8964A682054
:106F80001380FFF77FFC7F2803466CD8934A6A2062
:106F90001380FFF777FC7F2803465ED8904A6C2069
:106FA0001380FFF76FFC0428034650D88D4A6E20EB
:106FB0001380FFF767FC192843D82B88DFF844E2D9
:106FC000894F8A4A8A4D8B4E8B4C8C4903F0010CB9
:106FD000AEF800C0C3F3400EA7F800E0C3F380078B
:106FE0001780C3F3C007864A2F70C3F30017C3F39B
:106FF0004015C3F38013378025800B801080F8BDC7
:107000004FF6FF7398423FF455AC22283FF43AAD57
:1070100017287FF64FAC19287FF6B8AC1B287FF6EF
:10702000D5AC1C283FF4EAAC1E287FF6EFAC1F2835
:107030003FF4F4AC20283FF40DAD21287FF41EADC1
:1070400014E56E200021FFF703FC0020B5E70021C6
:107050006C20FFF7FDFB0023A8E77F216A20FFF7E4
:10706000F7FB7F239AE70B216820FFF7F1FB0B2347
:107070008CE700216620FFF7EBFB00237EE7002171
:107080006020FFF7E5FB002354E700215820FFF7BD
:10709000DFFB002318E702215220FFF7D9FB022370
:1070A000EDE60A214C20FFF7D3FB0A2386E61121E7
:1070B0004A20FFF7CDFB112378E60E214820FFF789
:1070C000C7FB0E236AE613214620FFF7C1FB1323FB
:1070D0005BE61F214420FFF7BBFB1F234CE600218A
:1070E0004020FFF7B5FB002339E600213E20FFF7E3
:1070F000AFFB00232BE600213C20FFF7A9FB002378
:107100001DE600213A20FFF7A3FB00230FE6002134
:107110003820FFF79DFB002301E600213620FFF712
:1071200097FB0023F3E500213420FFF791FB0023B8
:10713000E4E50C213220FFF78BFB0C23D5E5002181
:107140003020FFF785FB0023C6E50F212E20FFF737
:107150007FFB0F23B7E504212C20FFF779FB0423E5
:10716000A8E503212820FFF773FB032388E501210D
:107170002620FFF76DFB012379E514212020FFF77E
:1071800067FB142342E504211E20FFF761FB042363
:1071900033E502211C20FFF75BFB022324E50121DC
:1071A0001A20FFF755FB012315E500BFD489FF1F07
:1071B0006089FF1FD689FF1F6C9BFF1F2A9CFF1F42
:1071C000DC9AFF1F248AFF1F2C89FF1FA69BFF1F2D
:1071D000049CFF1F289BFF1F369CFF1F589BFF1F0F
:1071E000109BFF1FCC9AFF1F389BFF1F769BFF1F32
:1071F0009C9BFF1FA89BFF1F069CFF1FBC9BFF1FA4
:10720000749CFF1FFA9BFF1F02211820FFF720FB31
:107210000223D7E400211620FFF71AFB0023C8E45D
:1072200002211220FFF714FB0223ACE40C210E20F4
:10723000FFF70EFB0C238EE44FF47A610420FFF776
:1072400007FB4FF47A632FE44FF4AF610220FFF79E
:10725000FFFA4FF4AF631DE4F8B5812006F0C8FBD8
:10726000204B214A054603CB1368C5F803001A0CCE
:107270007020C5F807102B80AA70FFF7B5FA2E46CC
:10728000002426F80B0FA0B2FFF7FCFAFFF7ACFAC8
:107290000234702C26F8020FF5D16C1E05F17C0625
:1072A0004FF0FF3014F8013F082758400F4B40F3D0
:1072B00000017A1E0B4012F0FF0783EA5000F5D15F
:1072C000B442EFD1C043FFF7A1FA3A46C5F87D00BA
:1072D0008121284604F0C4FC2846BDE8F84006F0A9
:1072E0008FBB00BFE4F80000E0F800002083B8ED99
:1072F000F0B50E4B0E4C054693E8070085B02468A8
:107300002E88AD7801AB83E80700270C18460022D1
:107310000B21ADF804408DF80670ADF80C608DF8C7
:107320000E5004F09DFC05B0F0BD00BFF0F8000069
:10733000E0F80000F0B5124B124D1E68124F0FCD51
:1073400087B06C460FC495E8030044F8040B386816
:107350003B79CDF80D00320C222021808DF80220DF
:107360008DF81130ADF80060FFF73EFA0022ADF85D
:107370000B001221684604F073FC07B0F0BD00BF9B
:10738000E0F80000FCF8000088F50000002004F0A0
:10739000E3BC00BF02F02EBE70B5124C82B00025D7
:1073A000402306462946204600930195802320224B
:1073B00001F072FE20222946204602F031FA2046D2
:1073C000012102F037FA304607F09AF831460246BA
:1073D000204602F0BFFB204602B0BDE8704001F03D
:1073E00041BC00BF909CFF1FF0B5802983B075D9C8
:1073F0000546441E00F17C064FF0FF3014F8012FC3
:1074000008275040404A40F300017B1E0A4013F019
:10741000FF0782EA5000F5D1B442EFD1C043FFF735
:10742000F5F90146D5F87D000190019A914202D00C
:10743000B2F17F2F0BD105F10B00FFF7DDF97028BA
:107440000BD03248FFF7A8FF002003B0F0BD304852
:10745000FFF7A2FF384603B0F0BD05F10D00FFF7BE
:10746000CBF9222840D1002440F6AC5613E0042882
:107470001AD0062821D008281FD00A2828D00C2886
:1074800022D1A1F5FA7292B2B24201D8FFF7E0F927
:107490000234702C0ED004F10D002844FFF7ACF933
:1074A000022C0146A0B2E2D1B1F5805FEED30234E6
:1074B000702CF0D1012003B0F0BDA1F52F7292B273
:1074C000B2F57A6FE4D8E1E7222801D0242811D15F
:1074D000A1F5FA7292B2B242DAD8D7E70D48FFF7B7
:1074E0005BFF002003B0F0BD0B48FFF755FF002005
:1074F00003B0F0BD2A28C9D1A1F1320292B2B2F58F
:10750000967FC5D8C2E700BF2083B8ED40F90000E0
:107510002CF9000014F9000054F9000003290CD9DB
:1075200070B5461C82B005460C46304603222A49F7
:1075300007F054F810B102B070BD70470B2C05D99C
:1075400005222649281D07F049F840B12448FFF7D5
:1075500023FF244802B0BDE87040FFF7C9BE05F123
:107560000901032201A807F089F801A803221E4996
:1075700007F034F8D8B103221C4901A807F02EF80F
:1075800008B301A803221A4907F028F8B0B919482E
:10759000FFF702FFA11E89B23046FFF725FF002842
:1075A000C9D0154802B0BDE87040FFF7F5BE1348DA
:1075B000FFF7F2FEFFF750FE1148F3E71148FFF71F
:1075C000EBFE1148C6E71148FFF7E6FE02B0BDE842
:1075D0007040FFF7AFBE00BFE0F800006CF900009C
:1075E00074F9000088F900008CF90000B4F900007B
:1075F000CCF90000D0F90000E4F9000090F9000097
:10760000A4F90000F8F900000CFA0000B8F9000035
:107610002DE9F043174D2B6883B081460F46904605
:10762000F3B1154E34880A1992B2184611463280C9
:1076300006F05CFD28603A464946204402F06CFDA5
:10764000B8F1000F09D031882868FFF767FF286874
:1076500006F0D6F900232B60338003B0BDE8F08339
:10766000054E01930846318006F0C2F9019B28605F
:107670001C46E0E7309DFF1F2C9DFF1F10B51F4CDF
:107680004FF4FA70FCF71EFE204601F0DFF90022ED
:107690001146204602F0C4F82046012102F0CAF843
:1076A0002046002102F0C0F80B221549204602F0C6
:1076B00051FA204602F064FA0F221249204602F0E5
:1076C00049FA204602F05CFA0F490722204602F0F0
:1076D00041FA204602F054FA204601F0C3FA0B4B5F
:1076E0000B4A1A604FF4FA70FCF7ECFDFFF722FE2C
:1076F0000848BDE81040FFF74FBE00BF909CFF1F39
:1077000010FA00001CFA00002CFA0000E89EFF1F8F
:107710001176000034FA00000020704790F83920FC
:1077200090F83800101A704790F8383090F83920E7
:107730009A4205D95A1C034480F83820187E7047B5
:107740004FF0FF30704700BF90F8383090F8392084
:107750009A4286BF1B18187E4FF0FF30704700BF5B
:10776000704700BF38B50546B0F85E0090B195F897
:107770005D301446C3F1210294420CD805F13B0060
:107780001844224602F0C8FC95F85D30234485F881
:107790005D30204638BD012014462871EEE700BF59
:1077A000B0F85E306BB190F85D30202B07D8C2186E
:1077B000013380F85D30012082F83B1070470123CF
:1077C00003710020704700BF0023426980F8383001
:1077D00080F8393080F85C3080F85D3080F85E30B9
:1077E00080F85F3006CA30B40D68046943662A43E6
:1077F00083660A60A370426990F861301649146884
:1078000013441D7A5B7B01EBC5051B026D6803F415
:10781000E06343F064032B6090F8623013449D7C76
:10782000DB7D01EBC5011B02496803F4E06343F013
:1078300064030B6021685368194205D0036927224D
:107840005A70036904229A71036920225A710369EC
:1078500080229A7030BC70476805010043690CCBE8
:1078600012681A420CD0094B99420AD9084B994226
:10787000036994BF1A220D225A70036904229A7177
:107880007047036927225A70F7E700BF7F1A060086
:107890003F420F0010B50269D378DBB2D906044627
:1078A0003DD510215806D17038D503F0040303F0FC
:1078B000FF02002B51D03D49626E00230B7084F80B
:1078C0005D30002A5BD0904794F85D30002B56D095
:1078D0002369D0229A70236994F83B201A71236996
:1078E000012284F85C200222DA7010BD304B84F84B
:1078F00060009C424AD02F4B9C4252D094F83910E1
:1079000013791F29DBB207D82848007820B1601806
:10791000013184F8391003760223D37010BD590663
:10792000C3D4917801F0100101F0FF000029DDD0EF
:1079300013F001031ED194F85C1094F85D008842A6
:1079400081BF4B1C091984F85C3091F83B301371EE
:107950002369D0229A702269DEE7236984F83920EE
:10796000C0229A702369114A1979012111700222EB
:10797000DA7010BDC023937022691379CCE701221D
:10798000002384F85D2084F83B30A1E7626994F815
:107990006130094913440322187A02F043FD226939
:1079A000ACE7626994F861300449F3E7349DFF1F46
:1079B000AC8FFF1F1890FF1F1D7A0000297A00006E
:1079C0000369DB7803F0200373B190F86030013372
:1079D000DBB2012B80F860301AD9426990F861302F
:1079E0001344187A02F09ABD70B5426903F0FF059E
:1079F00090F8613013440446187A02F08FFDA36EAC
:107A00005BB184F8385094F83900BDE870401847ED
:107A100090F85F30002BE0D0704770BD0148FFF751
:107A2000CFBF00BFAC8FFF1F0148FFF7C9BF00BF2A
:107A30001890FF1F2DE9F047374FDFF8E0903B68C3
:107A4000026982B006460093DDF800800021A0257F
:107A5000D3789B065BD53B680193019BC8EB03037E
:107A60000F2BF5D949B1102BF2D00020907033695B
:107A700080229A7002B0BDE8F087726996F8613092
:107A800013440521187A02F043FF726996F86130B9
:107A90001344012193F812A0504602F039FF092443
:107AA0000021504602F020FF2B46013BFDD1012171
:107AB000504602F019FF2B46013BFDD1013CEFD1AE
:107AC000706996F8611001444FF4A0720C7A4B7BF8
:107AD00009EBC4011B02496803F4E06343F064034B
:107AE0000B6096F862300344997CDB7D09EBC101A1
:107AF0001B02496803F4E06343F064030B60013A3E
:107B0000FDD13269D3789B064FF00101A3D4012047
:107B100002B0BDE8F08700BF5C9DFF1F6805010053
:107B2000F0B503691222DA700269937803F020033A
:107B300085B004460D46002B5ED0B42393703C49BB
:107B400022690B680093009E05E00B680193019B7E
:107B50009B1B042B42D8D37803F0200303F0FF00D3
:107B6000002BF2D094F85D30002B31D04FF0000E96
:107B70004FF0020C04EB0E0393F83B3013710B68CB
:107B80000393039F206907E09B060DD50B680293C2
:107B9000029BDB1B052B28D8C378DBB203F0020263
:107BA00002F0FF06002AEFD080F803C02669F378C0
:107BB000DBB2DF0632462DD49F062BD5DB0731D44E
:107BC0000EF1010E94F85D305FFA8EFE7345D1D848
:107BD00000201DBB002384F85E3004E09070236910
:107BE00080229A70042005B0F0BD8670236980223F
:107BF00004209A7005B0F0BD03F0FF06FFF71AFFEE
:107C000010B9042005B0F0BD236984F85F60B0228C
:107C10009A7094E78023B3700420DAE72669802302
:107C2000B370D7E7BEF1000F0CBF02200320F6E7C8
:107C30005C9DFF1F2DE9F04106690025122780F8A1
:107C4000385080F83950F770D0F810C09CF802E036
:107C50000EF0200E88B00446884615461E46BEF13A
:107C6000000F49D0B4238CF80230784B21691A6890
:107C70000092DDF800E006E01A6801920198CEEB70
:107C80000000042830D8C87800F0200000F0FF077A
:107C90000028F1D04FEA480242F00102D2B20A7144
:107CA0001A680292DDF808E0206906E01A6803927B
:107CB0000399CEEB010105292AD8C17801F0020110
:107CC00001F0FF070029F1D04FF0020C80F803C04B
:107CD0002269D17811F0110722D12DBB002E0CBFE3
:107CE000A0238023937003E08F70236980229A7011
:107CF000384608B0BDE8F0810EF0FF07FFF79AFEA6
:107D00000028F5D0236984F85F70B0229A70ACE740
:107D100087702369802238469A7008B0BDE8F081E8
:107D2000802393700027E3E7012D75D0A021917087
:107D300021690A79BE4667464FF0A80C1A6804927A
:107D4000049805E01A680592059A121A052A4AD87D
:107D5000CA7802F0020202F0FF08002AF2D0CF70C7
:107D60002169CA78D2B212F0100F08465AD1920691
:107D700058D5013DEDB2012D49D0BEF11F0F3BD9C1
:107D80000A79012DDAD11A680692069D05E01A6873
:107D90000792079A521B052A46D8C27802F00202BF
:107DA00002F0FF01002AF2D00223C3702269D378C7
:107DB000DBB2D9063AD49B0634D5B023BEF11F0FEF
:107DC00093703FD8226904EB0E0312791A760EF1F4
:107DD000010E5FFA8EFE16B1236980229A7084F834
:107DE00039E0774684E781F80280236980229A701F
:107DF000774684F839E07BE704EB0E0291F80480C3
:107E000082F818800EF1010E5FFA8EFEB9E781F854
:107E100002C021690846B0E7A82191702069BE46DA
:107E20000279B0E7774663E78170DEE71021A0238F
:107E3000D170013BFDD12269937803F0F7037746B7
:107E4000937055E723691B79C5E700BF5C9DFF1F51
:107E50000148FFF71FBD00BFAC8FFF1F0148FFF7B0
:107E600019BD00BF1890FF1F704700BF38B5144CF4
:107E7000037801225B000546204684F83B3084F8F5
:107E80005E2084F85D20FFF78BFC20460021FFF781
:107E900047FE0B4C2978012320461A46FFF7CAFEFD
:107EA0000128F6D194F8383094F839209A4205D94F
:107EB000E218013384F83830107E38BDFF2038BD19
:107EC000AC8FFF1F38B51B4C037801225B000546C1
:107ED000204684F83B3084F85E2084F85D20FFF76C
:107EE0005FFC20460021FFF71BFE124C297820463C
:107EF00001230222FFF79EFE0228F6D194F83820D3
:107F000094F839108A420FD2531CDBB2A018994260
:107F100084F83830007E0AD9234402321B7E84F86C
:107F2000382040EA032038BD4FF6FF7038BD40F4DA
:107F30007F4038BDAC8FFF1F0C2901D9002070474E
:107F40000231490001F0FE01FFF7BCBF70B50C4CD7
:107F50000378164601255B00204684F83B3084F800
:107F60005E5084F85D50FFF71BFC31462046FFF75A
:107F700017FC29462046BDE87040FFF7D1BD00BF81
:107F8000AC8FFF1FF8B505460F4616464124214623
:107F90003A462846FFF7DAFF611C0234C9B232467E
:107FA0002846E4B2FFF7D2FF592CF0D1F8BD00BF4C
:107FB00038B504460D463548FFF706FC632280219C
:107FC00020462570FFF7C2FF012002F0C9FC2046C1
:107FD00000225E21FFF7BAFF20465D21FFF746FF32
:107FE000242801D0002038BD204606220C21FFF7AE
:107FF000C9FF204601222B21FFF7A8FF20460122BE
:108000002C21FFF7A3FF20460E222D21FFF79EFF14
:10801000204600222E21FFF799FF204601222F2122
:10802000FFF794FF204605223021FFF78FFF2046FF
:1080300001223121FFF78AFF204600223221FFF77B
:1080400085FF204600223321FFF780FF20460022D3
:108050003421FFF77BFF204600223521FFF776FF12
:10806000204600225B21FFF771FF204610225C2191
:10807000FFF76CFF204620225D21FFF767FF2046B7
:108080008F225E21FFF762FF012038BDAC8FFF1FFA
:1080900010B4047F4160022CC26002D010BC01F019
:1080A000D7BB836810BC184790E80C00F0B41C687C
:1080B00059682568164F174E29432160164D1749F8
:1080C0001760D66015611160417A154A5C180A3153
:1080D00094F8244053F8215002EBC40149680D6024
:1080E000017A5C1803EB8101247ECD6902EBC401A7
:1080F00049680D60817A581803EB810390F83000CD
:10810000596B02EBC002F0BC53681960704700BFA6
:1081100001401F00011000380110007800001F808E
:1081200068050100704700BFF0B50C1EBDF8146073
:1081300034DBB0F906701919B942C4BF3B1B1BB23E
:10814000002BA6461CDD002A1146B8BFD11D02F047
:108150000705CC10826A012007FB04E1A840012E2C
:108160000A44C0B21ED00CD3022E09D1013B12FA30
:1081700083F3013A12F8011F41409A421170F9D17C
:10818000F0BDC043013B12FA83F3C0B2013A12F8CA
:10819000011F014093421170F9D1F0BD23441BB27D
:1081A0000024C6E7013B12FA83F3013A12F8011FDB
:1081B00001439A421170F9D1F0BD00BFF8B50D1E10
:1081C0000EDB14461F46064601F03AFBA84207DDC7
:1081D000002C05DB304601F037FBA04201DCF8BD86
:1081E000F8BD304601F02AFB022853D003284BD0BB
:1081F000012806D16540F3886C406540013B5D1B5A
:108200002DB2012F03D02AD3022F14D0F8BD002C99
:108210002246B6F90630B06AB8BFE21D42F3CF027B
:1082200002FB035504F00704435D012101FA04F445
:108230001C434455F8BD002C2246B6F90630B06AFE
:10824000B8BFE21D42F3CF0202FB035504F007045E
:10825000435D012101FA04F45C404455F8BD002C53
:108260002246B6F90630B06AB8BFE21D42F3CF022B
:1082700002FB035504F00704435D012101FA04F4F5
:1082800023EA04044455F8BD3389013B591B2546B4
:108290000CB2B6E7F18832890139013A4D1B141B43
:1082A0002DB224B2ADE700BF2DE9F041079E9DF944
:1082B0001880089D04461F4600F0C0FF0D4B0E4875
:1082C0000E4984F83380FF22002F08BF1F4684F830
:1082D0002F20002384F8302084F8312084F83220C5
:1082E0002060A665E565676261652362A36220463A
:1082F000BDE8F081AC8FFF1FC0FA0000011001380B
:1083000010B50446806A034B236008B105F078FB82
:10831000204610BDC0FA0000F8B5436ADBB190F802
:108320002C200125AA4083F83B2083F85E5083F877
:108330005D500446406A03680E461B68002198475A
:10834000606A036831461B6898472946606ABDE841
:10835000F840FFF7E5BBC26BC56C1368046A23EAFB
:10836000050313604CB122684FF00043D3625163A0
:10837000D36A002BFCDA936BF8BD836B466B082540
:10838000802410E03768426C3A4332601F68826C88
:108390003A431A601A68876C013D22EA07024FEAE5
:1083A00054041A6007D02142ECD13268476C22EAAB
:1083B00007023260EAE7F8BD70B50446406A0D4630
:1083C00000282BD0A16DFFF749FA002D20460CBFE5
:1083D000A621A721FFF7A0FF606A20B1E16DBDE8EB
:1083E0007040FFF73BBA216C226D0868236A024394
:1083F0000A6093B1DA7A82B1D00703D5224A99692B
:108400001160DA7A910703D5204AD9691160DA7AC6
:10841000520702D51E4A1B6A136070BD236A002BE7
:108420002BD0D97A626DE1B172B6D97ACE0706D572
:108430001848D9680668314099610160D97A88077F
:1084400006D51548196906683140D9610160D97AA5
:108450004E0705D511485969066831401962016017
:1084600062B61B68D968914207D00D4818600D4963
:10847000DA6042F0804018611960226C216D136847
:1084800023EA01031360A0E700E100E004E100E05B
:1084900008E100E080E100E084E100E088E100E044
:1084A00001403F0000003F80436A2DE9F04105464E
:1084B0000E469046002B3ED090F82C100124A1408F
:1084C00083F83B1083F85E4083F85D40406A0368A0
:1084D00000211B6808F1FF379847FFB2B8F1000F81
:1084E00023D03744A046013E686A16F8011F03688E
:1084F0001B6898470134B742E4B216D0202CF3D160
:108500000121686AFFF70CFB95F82C206B6A52007A
:1085100083F83B2083F85E8083F85D80686A036897
:1085200000211B6898470124DEE7686A0121BDE845
:10853000F041FFF7F5BAC26BC16C136823EA01037F
:1085400006EB080413604FF00048A6420ED02B6AD9
:1085500016F801EB63B11A68C2F82C80C2F834E057
:10856000D36A002BFCDAA642936BF0D1BDE8F08110
:10857000AB6BD5F834C008208021DCF800206F6C8C
:108580001EEA010F14BF3A43BA43CCF800201A6820
:10859000AF6C3A431A601A68AF6C013822EA0702DE
:1085A0004FEA51011A60E8D1CFE700BF70B5044629
:1085B000406A0D46002828D0A16DFFF74FF92046EC
:1085C0002946FFF7A9FE606A20B1E16DBDE8704061
:1085D000FFF744B9216C226D0868236A02430A60E0
:1085E00093B1DA7A82B1D00703D5234A9969116031
:1085F000DA7A910703D5214AD9691160DA7A5207EC
:1086000002D51F4A1B6A136070BD236A002B2BD052
:10861000D97A626DE1B172B6D97ACE0706D519481A
:10862000D9680668314099610160D97A880706D512
:108630001548196906683140D9610160D97A4E0739
:1086400005D512485969066831401962016062B661
:108650001B68D968914207D00D4818600D49DA604F
:1086600042F0804018611960226C216D136823EA82
:1086700001031360A3E700BF00E100E004E100E0B4
:1086800008E100E080E100E084E100E088E100E052
:1086900001403F0000003F802DE9F041044686B0D4
:1086A000806A9DF830801E460F461546B4F90830A2
:1086B000002800F04281DA1D48BF03F10E02B4F930
:1086C0000630D21003FB02F2002105F0BDFCB4F924
:1086D0000820202A00F39280B4F90610A34B012051
:1086E000203A733902EBD27201EBD1714FF0200EB8
:1086F000029073208DE8014042F34F0241F34F0195
:10870000204600F051FE606A84F82D70002800F0C9
:108710004D81002D40F08A80B4F90830202B14BF21
:108720003D253C2584F82C50B8F1000F40F08580A1
:1087300006B394F93300002818DBC0B2012102F01F
:10874000E7F8012194F8330002F0CEF8012002F09E
:1087500007F9002194F8330002F0C6F80A2002F06D
:10876000FFF8012194F8330002F0BEF8606A002897
:1087700000F08280A16DFFF771F804227C49204649
:10878000FFF792FE217A0139C9B22046FFF7C4FDF6
:10879000784904222046FFF787FE94F92D30012BFB
:1087A00014BF142110212046FFF7B6FD04227249A0
:1087B0002046FFF779FEB4F90630802B00F0928056
:1087C000602B00F0A680D9212046FFF7A5FD94F983
:1087D0002D30012B14BFF12122212046FFF79CFDF3
:1087E000204606226549FFF75FFE606A50B3E16DDF
:1087F000FFF734F8012006B0BDE8F081B4F90610A7
:108800005F4B0120403A52394FF0400E029002EB8C
:10881000D272522001EBD1718DE8014042F34F0238
:1088200041F34F01204600F0BFFD6CE76DB284F8C4
:108830002C50B8F1000F3FF47BAFFEF7C5FF002EC0
:1088400094D076E7216C226D0868236A02430A609F
:1088500073B1DA7A62B1D00703D54A4A99691160D7
:10886000DA7A91077CD4520702D5474A1B6A136013
:10887000012006B0BDE8F081236A002B2BD0D97A05
:10888000626DE1B172B6D97ACF0706D53F48D96893
:108890000568294099610160D97A8E0706D53C4860
:1088A000196905682940D9610160D97A4D0705D554
:1088B00038485969056829401962016062B61B6829
:1088C000D968914207D0344818603449DA6042F0E0
:1088D000804018611960226C216D136823EA01033E
:1088E00013604AE7B4F90830202B00F08680402B53
:1088F0007FF469AF2A4920460322FFF7D5FD94F99A
:108900002D30012B14BFCF219F212046FFF704FDFE
:1089100059E7B4F90830102B7FF455AF21492046B0
:108920000322FFF7C1FD94F92D30012B14BFAF21B5
:1089300010212046FFF7F0FC45E7DA1D48BF03F1A0
:108940000E02B4F90630D21003FB02F21046059273
:1089500005F04EF8A06200283FF44DAF059AB3E64B
:10896000114AD9691160DA7A7DE700BF18FB00006F
:10897000F8FC0000FCFC000000FD000004FD00000D
:108980000CFD000000E100E008E100E080E100E013
:1089900084E100E088E100E001403F0000003F800A
:1089A00014FB0000CCFF000004E100E0012194F87A
:1089B0003100244F01F0ACFF94F83200012101F0A6
:1089C000A7FF94F9312094F9323057F83220E2634E
:1089D00057F83330206A23640125E56425651A6859
:1089E0002A431A6078B1B8F1000F3FF428AFFFF7BF
:1089F0005BFB002E3FF4BAAE9BE6042212492046F0
:108A0000FFF752FDDFE6294694F82F0001F080FFC2
:108A1000294694F8300001F07BFF94F92F2094F957
:108A2000303057F83220626357F833306564A564FC
:108A30001A68A36322F001021A60002E3FF496AE7A
:108A400077E600BF6805010010FB0000B0F90820C0
:108A5000D31D48BF02F10E03B0F90620806ADB1077
:108A600002FB03F2002105F0EFBA00BFF0B50029C8
:108A7000BDF814502EDBB0F90660B1422ADA002AA4
:108A800059DBB0F9087014461C44BC42C4BFBB1A81
:108A90001BB2002B1EDDD2B2D408D0F828E016FBA2
:108AA000041112F00702DBB20EEB010421D0C2F177
:108AB0000807FAB2374F9342BF5C0CD2C3EB020CEB
:108AC000FF2646FA0CF6012D07EA06073FD005D32C
:108AD000022D36D0F0BD012D39D030D21EF8016004
:108AE00026EA07070EF801709342F3D3B0F9061097
:108AF0000C449A1AD2B2072A10D9022D36D0002D72
:108B000014BFFF26002613462670083BB0F9061056
:108B1000DBB2072B0C44F7D802F00702002AD9D0A9
:108B20001D4B012D9B5C1DD017D3022DD2D1227875
:108B300053402370F0BD13441BB20022A1E7022D65
:108B400025D11EF8016077400EF80170CCE71EF8C1
:108B5000016037430EF80170C6E7227822EA03036A
:108B60002370F0BD227813432370F0BD11462378A3
:108B7000DB4323700839B0F90630C9B207291C4419
:108B8000F5D812F00702A5D0034B9B5CCFE7344425
:108B9000AFE700BFB0FA0000A0FA000070B4C47DD7
:108BA000BDF80C50022C18D0032C1FD0012C0BD078
:108BB000002A03DBB0F90840944201DC70BC704726
:108BC000039570BCFFF7B0BAC4880395013CA41AA2
:108BD0000A4621B270BCFFF749BF0689C488013E2E
:108BE000641AB21AE41A12B221B2E1E704890395B9
:108BF000E41A641A114622B270BCFFF737BF00BFF7
:108C000070B4C57DBDF80C60022D1AD0032D12D0B2
:108C1000012D03D0039670BCFFF728BFC488E41A67
:108C2000A41A0A4621B2002A03DBB0F90840944294
:108C300013DC70BC70470489013C641A114622B2EF
:108C4000F1E7C48805890396013CAD1AED1A621A52
:108C500011B22AB270BCFFF709BF039670BCFFF7D0
:108C600063BA00BF2DE9F8430446406A002863D088
:108C7000A16DFEF7F3FD052274492046FFF714FCB1
:108C8000A1790139C9B22046FFF746FBB4F90820A3
:108C9000E588A66AD31D48BF02F10E03DB10626AA5
:108CA00015FB03F51FFA85F8002A7BD094F82C30C9
:108CB0000125AB4082F83B3082F85E5082F85D506F
:108CC000606A036840211B6808F1FF379847BFB20C
:108CD000B8F1000F23D03744A846013E606A16F869
:108CE000011F03681B6898470135B742EDB216D0E3
:108CF000202DF3D10121606AFEF712FF94F82C2099
:108D0000636A520083F83B2083F85E8083F85D80BD
:108D1000606A036840211B6898470125DEE701214E
:108D2000606AFEF7FDFE606A002800F08D80E16D4C
:108D3000BDE8F843FEF792BD236A002B2BD0D97A09
:108D4000626DE1B172B6D97ACE0706D54048D968CE
:108D50000568294099610160D97A8D0706D53D489B
:108D6000196905682940D9610160D97A480705D594
:108D700039485969056829401962016062B61B6863
:108D8000D968914207D0354818603549DA6042F019
:108D9000804018611960226C216D136823EA010379
:108DA000136068E7E26BE36C1168276A0B4306EB1C
:108DB000080913604FF0004E4E450DD016F801CB58
:108DC0002FB33A68C2F82CE0C2F834C0D36A002B43
:108DD000FCDA4E45936BF1D1226C236D11680B4385
:108DE000136097B1FB7A83B1D90703D51D4BBA69DC
:108DF0001A60FB7A9A0703D51B4BFA691A60FB7A53
:108E00005B0702D5194B3A6A1A60BDE8F883A36B79
:108E1000D4F8348008208021D8F80020656C1CEA42
:108E2000010F14BF2A43AA43C8F800201A68A56C92
:108E30002A431A601A68A56C013822EA05024FEA33
:108E400051011A60E8D1B7E7276AC5E7A8FA000020
:108E500080E100E084E100E088E100E001403F00C3
:108E600000003F8000E100E004E100E008E100E0F4
:108E70002DE9F04F85B09946BDF93870BDF83CA09A
:108E8000BB1AC1EB090B002BB8BF5B42BBF1000F53
:108E9000B8BFCBF1000B5B450D46164600938046EC
:108EA00048DC4D453A4633464CDC194613460A46E3
:108EB000C5EB09019B1A89B2002B0CB2B8BF5B420B
:108EC00004EBD474BE42ACBF4FF0FF3201224D45DB
:108ED000039102924FEA640429DC9BB201930DE0F6
:108EE000D8F80070BF69B847019BE41AA3B21CB25E
:108EF0000135002C2DB211DBA94518DB009B5B4529
:108F00002A46534631464046EADCD8F8002053460C
:108F10009769294632464046B847E5E7029A164423
:108F2000039AA94502EB030436B224B2E6DA05B08F
:108F3000BDE8F08F4A462B46B94635464D451746A3
:108F40001E46B2DD304629463E464D460746894616
:108F5000AEE700BF10B404682469A44610BC6047A3
:108F600030B40468BDF808500295A46BA44630BC28
:108F7000604700BF30B40468BDF808500295E46B48
:108F8000A44630BC604700BF70B40468BDF90C60F3
:108F9000BDF8105003960495246CA44670BC60473D
:108FA000704700BF10B582B0B0F90C200191016884
:108FB000009200220C6CB0F90A301146A04702B0B2
:108FC00010BD00BF704700BF01F003010129C1754A
:108FD00006D0032904D0C288038942818381704767
:108FE0000289C38842818381704700BF2DE9F04127
:108FF0000568134E6F6986B0B7420446BDF83080ED
:1090000010D1013B13441BB20093CDF804800B46F2
:10901000AD6A2046A8472368DB6AB3420AD106B08E
:10902000BDE8F081059304920391B84703A9256830
:109030000EC9E6E7204606B0BDE8F041184700BF7C
:10904000A18F00002DE9F0410568124E6F6986B0CE
:10905000B7420446BDF830800FD1013BCDF8048003
:109060000B4400921BB2AD6A2046A8472368DB6A16
:10907000B3420AD106B0BDE8F08105930492039192
:10908000B84703A925680EC9E7E7204606B0BDE842
:10909000F0411847A18F00002DE9F04F0568DFF877
:1090A00058B06F6985B05F450646BDF93890BDF888
:1090B0003CA00C46904615D11F19BC420CDACDF8E5
:1090C00000A0214601342D6A4B464246304624B268
:1090D000A847BC423568F2DBEB6A5B4507D105B0B7
:1090E000BDE8F08F0393B8473568039BE4E730464B
:1090F00005B0BDE8F04F1847A18F00002DE9F043FF
:1091000087B099420546BDF93840BDF83C6025D08E
:10911000A24212D00768DFF88080D7F81490C145CA
:1091200032D18DE850002846BC6AA0472B68DB6A24
:10913000434524D107B0BDE8F083994202DD0846DB
:109140001946034628680E96C46B01335B1A1BB29E
:109150002846A44607B0BDE8F0436047A24202DDBE
:10916000134622461C4628680E96631C846B9B1A85
:109170001BB22846A44607B0BDE8F0436047284626
:1091800007B0BDE8F0431847059304920391C84720
:1091900003A92F680EC9C4E7A18F00002DE9F04F85
:1091A000D0F800E0DFF89090DEF814B083B0CB4543
:1091B0000446BDF93080BDF834A00D4617461E4662
:1091C00031D1CDF800A0DEF824B0294633463A4626
:1091D0002046D8472368CDF800A008F1FF323A4472
:1091E000D3F824B0294612B233462046D847236824
:1091F000CDF800A02946D3F820B03A464346204691
:10920000D8472068CDF800A0711E29444346056A5E
:1092100009B23A462046A8472368DB6A4B4506D187
:1092200003B0BDE8F08FD847D4F800E0C9E7204686
:1092300003B0BDE8F04F1847A18F0000F0B4002440
:1092400001264FF6FF75094F07600471C475C4818C
:1092500004824476C4618675067685824582C18023
:10926000028141818281F0BC704700BFD8FF0000BD
:109270002DE9F04F85B00668BDF84450BDF938803F
:10928000CDF8008004460195D6F848B00392BDF9A8
:109290003C60BDF9407089469A46D84723680195DD
:1092A000009742465146D3F8488020463346C0478F
:1092B0002068039B0E930F95856C4B463A463146CA
:1092C0002046AC4605B0BDE8F04F60472DE9F04FB1
:1092D00087B01746BDF9404000912546E91D05932A
:1092E00044BF2B4603F10E010268BDF84860536984
:1092F0000294C91003912B49BDF9444001968B4259
:10930000824645D1002C3CDD029B3C445E1EB6B239
:109310004FF0000923B2049301364D46029B002B07
:1093200028DD059B002403EB090806E0EDB22B06BF
:1093300004F1010411D4A6421CD0A1B211F0070F10
:1093400023B24FEA4505F1D1002BB8BF0733DB103C
:10935000013418F803502B06EDD5009BD2F818B055
:1093600019443A4609B2019B5046D847A642DAF85A
:109370000020E2D1039B01379944049B3FB2BB42DA
:10938000CCD1D36A074A934206D107B0BDE8F08F2B
:109390009847DAF80020B5E7504607B0BDE8F04F2F
:1093A000184700BFA18F000070B4BDF90C60BDF973
:1093B0001050BDF8144003960495059470BCFFF757
:1093C00085BF00BF2DE9F04F93B090460591C1696C
:1093D0001090BDF870000790BDF874909DF878A0CB
:1093E0000493002900F0CD800A7A0AC989460499BD
:1093F0008A1AD2B203EBC203BAF1010FDA780B92E8
:1094000093F905201E8893F802B00F9293F9064055
:1094100079D913B2099323B20C93109B1A68A94B04
:109420001193194653698B4240F0A6800B9B002B89
:1094300055D01FFA88F300210D93C8462344DDF868
:10944000409006910E930F460C46BBF1000F3FD0A3
:10945000BDF818100C9B03971FFA8AF0CB1813FB6A
:1094600000F304900E9801440D98034409B21BB216
:109470000A910893002505E00135EBB264009B4595
:10948000E4B222D9039B2B44590703D1731C18F86B
:1094900006409EB22306EFD5099BBDF81000E918DF
:1094A00011FB00F10598BAF1010F0FFA8AF301449C
:1094B0001CD0079801900093D26909B2174648461C
:1094C000089AB847D9F80020D6E7039F5F44FFB257
:1094D000069B0B9901330693DBB29942B5D8D36A48
:1094E000119A934243D113B0BDE8F08F0F9B191826
:1094F00093690A9A29441F4609B2079B4846B84710
:10950000D9F80020B8E700230C93099385E70A9A5D
:109510000D9B0132013B52B213F0FF030A920D93EF
:109520006FD1DDF81890079BDDF83C80DDF820A0B6
:109530004B4517D0BAF1010F00F0C8800B9A109D6F
:10954000CDF804900BEB8B014FEACB030A44009358
:109550001146DEF81C405346424609B22846A04751
:10956000D5F800E0DEF82C30119A9342BBD0109869
:1095700013B0BDE8F04F1847109D284698472A6859
:1095800054E7109A0598B2F90A308342ABDDB2F97C
:109590000C304345A7DD062313FB0A03002BA2DD95
:1095A00008EBCA03002B9EDD537E2BB9049BAF2B27
:1095B00002D90133DBB20493109BD3F800E0414B96
:1095C00011931A46DEF81430934240F08E801FFA51
:1095D00088F30E9308339BB2BDF81420059305233E
:1095E0000D9300230A93CDF83C800FFA8AF3DDF83F
:1095F0004080CDF818900B921FFA8AFBCDF820A07E
:1096000099460A9ABDF810000B9C0E9D0523194639
:1096100011FB00232C481146C75C039702FB0B4249
:1096200014FA81F312B21BB209920C932C462E4607
:109630001CE0089B0999012B2AB24B4640462DD0CD
:10964000079F0197CDF80090DEF81CA0D047D8F80E
:1096500000E0039B5B0801340393059BA4B25D44C7
:109660005E44A342ADB2B6B23FF451AF039BD807FC
:10967000DFD4079B069A9342EBD0089B012B16D0B0
:10968000069B0193CDF80090DEF81CA009994B468B
:1096900032B24046D047D8F800E0DAE7DEF818A04A
:1096A000079B0C9922B2D047D8F800E0D1E7DEF84A
:1096B00018A00C991346404622B2D047D8F800E0D3
:1096C000C7E700BFA18F0000280001000B99109D83
:1096D000CDF800900531DEF8204009B2424608235B
:1096E0002846A047D5F800E03CE7109C2046984764
:1096F000D4F800E06BE700BFF0B5C36985B004465D
:109700002BB30A2968D00D294AD01A7A914247D33F
:10971000587A884244D35D688A1A05EBC205AA7854
:10972000002A50D0E87800284DD0207E00283AD07A
:1097300095F905E0B4F90E00A67DB4F90A707244FB
:1097400006FB0202BA4262DCB4F9102030E00A29BA
:1097500056D00D2924D0027E002A4BD0B0F90E003D
:10976000A57DB4F90A60062212FB0502B2423EDD75
:10977000228AE38102EBC50212B218462282A78A2E
:10978000668A02950B468DE8C00001462046FFF729
:1097900019FEA37DE28903EB430302EB4303E3815C
:1097A000012005B0F0BDA67DB4F90E00B4F910207B
:1097B000B4F814E0678A02960B468DE880400146B3
:1097C0002046FFF7FFFD2979E389A27D012001FBF7
:1097D0000233E38105B0F0BD0022C2819A7A817D17
:1097E000038A01FB02330382012005B0F0BDB4F906
:1097F0001020C4E7857DB4F91020B0F90E00BEE753
:10980000028A817DC38102EBC1030382C8E7002085
:10981000E0819B7A228A03FB062212B22282C7E7EA
:10982000C1810282704700BF002908BF01218175F4
:10983000704700BF81824182704700BFC07D704782
:10984000B0F90A00704700BFB0F90C00704700BFC4
:1098500010B4EFF3108272B6437F33B9017F012950
:1098600007D003290FD00123437702B962B610BC99
:109870007047124C2168A1B1114943610B688361A3
:1098800008605861EFE70F4C216881B10E494361D0
:109890000B688361086058610C4B4FF08051196070
:1098A000E1E7074B4161816120601860DBE7064B0F
:1098B0004161816120601860EEE700BF489DFF1F95
:1098C000449DFF1F389DFF1F3C9DFF1F04ED00E0DE
:1098D00070B5EFF3108272B60C4C206880B10C4E5C
:1098E00000254369236073B19D6102B962B6457773
:1098F00083689847EFF3108272B620680028F0D191
:1099000002B962B670BD3360EFE700BF389DFF1F3C
:109910003C9DFF1FFFF7DCBF184A30B41468002CD1
:1099200027D0036821688B420ED2CB1A00218460B5
:10993000C1602360E06010600223037530BC704793
:1099400011688B42144608D3A2685B1A0360002A90
:10995000F6D18260C460A060EEE7D268C260846025
:10996000E060C568CB1A0222A8602360027530BC93
:1099700070478460C4601060DEE700BF409DFF1F39
:10998000F8B5224E34682CB32368002B3AD1204F0F
:109990001D4604E03468ECB12368002B32D1A36883
:1099A00003B1DD6020693360036825751B68BB4225
:1099B00021D1037F4560022BC46020D0FFF748FF10
:1099C0006368002BE6D023602046FFF7A5FF3468CC
:1099D000002CE1D1EFF3108372B60E4A002110681B
:1099E000116003B962B628B18468FFF795FF20467D
:1099F0000028F9D1F8BD224600219847E0E78368A6
:109A00009847DDE7013B2360E4E700BF409DFF1F6F
:109A100091800000509DFF1F024A136801331360BC
:109A2000FFF7AEBF5C9DFF1F704700BF0368F0B437
:109A3000FBB1002501249D60DC601B4C1A601C44B6
:109A4000241104F144056A11032692009E60174F09
:109A50000679174B47F8241002F1604202F5614283
:109A600005F01F05012000FA05F5E6541560F0BC6D
:109A70007047104C236843F40003236000BF0E4B73
:109A80000E4DA4F58734A4F59E7401261E6023466E
:109A900004609C68002CD0D01033AB420360F8D136
:109AA000002303601846E2E7008FFCBF8490FF1F8D
:109AB00044E400E03C8004400070034040710340F7
:109AC0000168A9B10B4BF0B40B441B110A4E0B4FAC
:109AD0000B4D46F8237003F1440202F01F040123EA
:109AE0005211A340002445F822308C600460F0BC81
:109AF000704700BF008FFCBF8490FF1F299A0000B1
:109B000080E100E0024A034B012111601B68184705
:109B10000C7103408490FF1F024A034B0121116026
:109B20005B6818471C7103408490FF1F024A034B77
:109B3000012111609B6818472C7103408490FF1F1E
:109B4000024A034B01211160DB6818473C71034056
:109B50008490FF1FF8B50E4671B17AB107461446DE
:109B600000253B6816F8011B1B6838469847013CE6
:109B70000544F6D12846F8BD0846F8BD1046F8BDA4
:109B800000B5064A036812885B6883B001A9ADF886
:109B900004200222984703B05DF804FB2805010069
:109BA000F0B507468BB0002A33D0012A08BF0A223D
:109BB00051B3212400E0F4B2B1FBF2F502FB151120
:109BC000C8B2092900F1300198BFC8B20AA988BFFC
:109BD0003730214488BFC0B201F8240C661E2946E4
:109BE000002DE8D133B1013CE4B20AAB23442D226D
:109BF00003F8242C3B6801AA11195B683846C4F1AC
:109C0000220298470BB0F0BD30228DF82520212488
:109C1000E8E70368C9B21B6898470BB0F0BD00BF06
:109C20000029BABF49422D2300230A22FFF7B8BFFB
:109C3000374A384913681B06FCD40B6813F08003BD
:109C4000F8D172B634490A78002A5FD0334A3448D2
:109C5000F0B4344C176806682568D4680C303E446C
:109C6000143200681268304F35442C4420440244BA
:109C7000C2F34E022D4E2E482E4D2F4C42F4004280
:109C80003A60376806682D682C4A24680C303E44D8
:109C9000006812682A4F35442C4420440244C2F321
:109CA0004E02284E2848294D294C42F400423A6081
:109CB000376806682D68274A24680C303E440068DF
:109CC0001268254F35442C4420440244C2F34E020E
:109CD000224E2348234D244C42F400423A60376818
:109CE00006682D68214A24680C303E4400681268DA
:109CF00035442C4420440244C2F34E021C4842F432
:109D0000004202600B7062B6F0BC704762B67047EA
:109D100024B0034024B00B40559DFF1F38B00340D2
:109D20003CB0034040B003402CB0034058B0034067
:109D30005CB0034060B0034064B003406CB00340CB
:109D400030B0034038B00B403CB00B4040B00B404B
:109D500044B00B404CB00B402CB00B4058B00B4003
:109D60005CB00B4060B00B4064B00B406CB00B407B
:109D700030B00B4030B42948294A2A4B2A4D602480
:109D8000E121047011701B78284C082B30D00A2B6D
:109D90002748284937D00C2B0CBF35223D221223EF
:109DA0002A60236002600B60234B24491B78244AFD
:109DB000BBB101230B601360224B23491B78234A5C
:109DC000012B26D9042B0FD9082B1ED9102B94BF99
:109DD000862387230B6013601D4B01221A7030BC51
:109DE00070470B601360E7E784230B601360F3E7B1
:109DF00000F58E200F490830012213232A602360CA
:109E000002600B60D0E73922F7E785230B6013600F
:109E1000E2E780230B601360DEE700BF00400740ED
:109E2000014007409490FF1F08B003400CB003406E
:109E300008B00B400CB00B40589DFF1F20B00340F2
:109E400020B00B409590FF1F24B0034024B00B407E
:109E5000559DFF1F0C2830B417D91023984228BFF6
:109E600018461C46104A114D1178181A8C42287059
:109E700018D00F4913700B7823B10E490E4A0023F6
:109E80000B60136030BCFFF775BF0A2802D90C23A2
:109E90001C46E7E7082802D90A231C46E2E7082304
:109EA0001C46DFE730BC70479490FF1F549DFF1F96
:109EB000559DFF1F24B0034024B00B4028282FD805
:109EC000334B2DE9F0411E5CFF2E2BD0314B1B781C
:109ED000002B2AD132062CD472B62F4D2F4C2F4690
:109EE000012326602B7062B672B623681B060CD461
:109EF0003B781BB9F4E72B78002BF1D062B602F067
:109F00009BF972B623681806F5D5254B1B6800220D
:109F10002A7062B6234A107843FA00F0BDE8F08157
:109F2000002070470020BDE8F081FFF781FE320677
:109F3000D2D572B61C4DDFF87C801C4C06F0400771
:109F4000FFB206F03F06D8F80030DFB123F010036F
:109F5000C8F8003001232660134A2B7062B672B62F
:109F6000236819060CD413781BB9ECE72B78002B67
:109F7000E9D062B602F060F972B623681B06F5D527
:109F80000B4BC3E743F01003C8F80030E2E700BF13
:109F90002C050100559DFF1F579DFF1F00B003407A
:109FA00010B00340549DFF1F569DFF1F00B00B4093
:109FB00010B00B400CB00B400A4A0B49136843F435
:109FC000805313600B7843B9084BC0221A70084BBA
:109FD00080F30C0000B218807047044B80221A7086
:109FE000F5E700BF2C800440589DFF1F21C00C40A6
:109FF00000C00C40F0B51B4B1B4E596818689A689E
:10A00000DB6885B06C460FC4337899071DD5174AB5
:10A01000174C1378174913F0700318BF1370164AC2
:10A02000164B8027177000263320032226706D46BA
:10A0300008701A7072B6043C45F001052046A84726
:10A0400062B6237813F0700309D10D4B064901E085
:10A05000013B02D00A78D207FAD505B0F0BD2370D3
:10A0600005B0F0BD580501000100024000000240AB
:10A07000040002400B000240070002400A000240B8
:10A08000410D0300B0F5006F0AD210B5094B1B78E3
:10A09000DB07044606D504F1A0500078C0B210BD1D
:10A0A00000207047FFF7A6FF04F1A0500078C0B26F
:10A0B00010BD00BF01000240B0F5006F17D238B5E7
:10A0C0000F4B1B78DA070D46044611D504F1A0505A
:10A0D0000378AB420AD00B4A137813F0700318BF11
:10A0E0001370074A05701378DB07FCD538BD70473D
:10A0F000FFF780FF04F1A0500378AB42EBD1F5E706
:10A10000010002400000024008B5F6F7CDFAF8F76A
:10A1100025F802F091F8FAE7844641EA000313F0CB
:10A1200003036DD1403A41D351F8043B40F8043B5E
:10A1300051F8043B40F8043B51F8043B40F8043B21
:10A1400051F8043B40F8043B51F8043B40F8043B11
:10A1500051F8043B40F8043B51F8043B40F8043B01
:10A1600051F8043B40F8043B51F8043B40F8043BF1
:10A1700051F8043B40F8043B51F8043B40F8043BE1
:10A1800051F8043B40F8043B51F8043B40F8043BD1
:10A1900051F8043B40F8043B51F8043B40F8043BC1
:10A1A00051F8043B40F8043B403ABDD2303211D361
:10A1B00051F8043B40F8043B51F8043B40F8043BA1
:10A1C00051F8043B40F8043B51F8043B40F8043B91
:10A1D000103AEDD20C3205D351F8043B40F8043B61
:10A1E000043AF9D2043208D0D2071CBF11F8013B5F
:10A1F00000F8013B01D30B8803806046704700BF25
:10A20000082A13D38B078DD010F003038AD0C3F133
:10A210000403D21ADB071CBF11F8013B00F8013B15
:10A2200080D331F8023B20F8023B7BE7043AD9D3D4
:10A23000013A11F8013B00F8013BF9D20B780370A9
:10A240004B7843708B7883706046704708B5104C2C
:10A2500008E0236859050DD423681A050FD4236834
:10A26000DB0411D423685803F3D500F08DFE236876
:10A270005905F1D502F044F823681A05EFD502F02C
:10A28000D5F82368DB04EDD500F0F0FCEAE700BF69
:10A290003480044008B5FFF7D9FF00BF014B1022FE
:10A2A0001A80704700200540704700BF094908B573
:10A2B0000B6830B16A461844A2F58052904202D22F
:10A2C0000860184608BD03F065FB0C2303604FF0DF
:10A2D000FF3008BD9890FF1FFEE700BFEFF313802B
:10A2E00070B9EFF310836BB9EFF305825AB94FF4ED
:10A2F0008070EFF311832BB1984228BF1846704746
:10A300004FF0FF3070470F2A01D81846F1E7014B94
:10A31000D05CEEE7F0E300E0F0B44D1E2E460024E2
:10A3200000E00134B0FBF2F302FB1300092800F156
:10A3300030078ABF3730F8B2C0B206F8010F1846AE
:10A34000002BEED10A1953704CB1107815F8016F3B
:10A3500028700133E01A834202F80169F5DB0846F0
:10A36000F0BC7047704700BF10B40F4B53F830205B
:10A3700092F880422CB1012369B182F8803010BC80
:10A38000704703EBC0035B681A6841B922F0020210
:10A390001A6010BC704782F8003110BC704742F060
:10A3A00003021A6010BC7047680501001C4A02EBEA
:10A3B000C00301295B6811D004291BD052F830007A
:10A3C000002280F8802229B1022920D0032922D03E
:10A3D0001A6070474FF480721A60704752F830006C
:10A3E0004FF4A27280F880121A601A6822F02002DC
:10A3F0001A60704752F830104FF4A272012081F8B1
:10A4000080021A601A6842F020021A60704740F217
:10A4100003121A6070474FF481721A60704700BFD0
:10A4200068050100212848D8F8B5042A44D8DFE897
:10A4300002F0484B4E0345004FF410262B4B03EB24
:10A44000C0030D465C68216811F4E06148D0284BD8
:10A45000284A2949C3F89C2104F140422748C3F8FF
:10A46000A411A2F59221264FC3F8A0017C2925480A
:10A47000C3F8A871C3F8AC012CD9A2F594237C2BA6
:10A480002AD9A2F596237C2B28D9A2F598237C2BD8
:10A4900029D9A2F59A227C2A27D81B4872B62368AC
:10A4A00023F4702343F08072C4F3840116432360C5
:10A4B00040F82150266062B6F8BD70474FF4302650
:10A4C000BCE74FF40026B9E74FF44026B6E74FF457
:10A4D0002026B3E70D48E1E70D48DFE70D48DDE74B
:10A4E000FFF764FFB3E70C48D8E7F8BD6805010043
:10A4F0000082FF1FF188FF1F9988FF1FC588FF1F7B
:10A500006D88FF1F4188FF1F7491FF1F9C90FF1FE4
:10A51000D490FF1F2491FF1F5491FF1F1A4B03EB90
:10A52000C00010B4426802F14043A3F592217C2997
:10A5300023D9A3F594217C290DD9A3F596217C2953
:10A540001FD9A3F598217C2919D9A3F59A237C2B2F
:10A5500011D80E4C00E00E4C72B613680D4823F073
:10A560008773C2F3840123F4803343F08073136054
:10A5700044F8210062B610BC7047074CECE7074C6A
:10A58000EAE7074CE8E700BF680501007491FF1F88
:10A59000D490FF1F65A300009C90FF1F5491FF1FE4
:10A5A0002491FF1F30B4054B054D064C00221021AD
:10A5B0001A602A602060196030BC704714D00340D4
:10A5C00004D0034000D00340282838B52ED00029FD
:10A5D00004464FDD5F4B1B78012505FA03F28A42E2
:10A5E00002D8212837D938BD0338C2B2012A3AD956
:10A5F000202C4AD0192C48D0574A126802FB01126D
:10A6000022FA03F31D2800F29B80DFE800F0928B12
:10A61000847D9999766F9999999999999999996859
:10A62000615A53994C99999999999945494B1B7835
:10A630000B2B08D90C2B1CBF0C3B19410846BDE85D
:10A640003840FFF7B9BCC3F10C0399400846BDE898
:10A650003840FFF7B1BC2946FFF786FE2946BDE822
:10A660003840FFF7A3BE3D4A126802FB011222FAEE
:10A6700003F3C7E72128B6D80021FFF775FE20466F
:10A680000121BDE83840FFF791BE354A126802FB50
:10A69000011222FA03F3B5E73249334A0B604FF453
:10A6A0005173136038BD3149314A0B604FF4517317
:10A6B000136038BD2F49304A0B6040F244431360A9
:10A6C00038BD2E492E4A0B6040F24443136038BD1A
:10A6D0002C492D4A0B6040F24443136038BD2B498E
:10A6E0002B4A0B6040F24443136038BD29492A4A83
:10A6F0000B6040F24443136038BD2849284A0B6080
:10A7000040F24443136038BD2649274A0B6040F2AB
:10A710004443136038BD2549254A0B6040F2444349
:10A72000136038BD2349244A0B604FF45173136002
:10A7300038BD2249224A0B604FF45173136038BD73
:10A74000212C3FF650AF7F29D4BF002101212046A4
:10A7500093E700BF7C91FF1F0880034008900340EF
:10A7600008800B4010800B4048A0044018800B402C
:10A770004CA004401880034008B0044010800340FF
:10A7800004B004404080034018C0044038800340B7
:10A7900014C004402880034010B0044020800340CF
:10A7A0000CB004403080034010C004404880034097
:10A7B0001CC00440189003403490044010900340A3
:10A7C0003090044038B1102828BF1020044AC3B28A
:10A7D000107813707047024A012310781370704785
:10A7E0007C91FF1F2DE9F8430E4680463249334DD8
:10A7F000304603F055F847F6122300281ABF1D46CD
:10A800004FF002094FF00109002425FA04F002F08C
:10A8100051FE4FF05E51074602F0A4FE014630465D
:10A8200003F052F830B90134072CEED1E80902F0F8
:10A8300041FE07463146384602F048FF4FF07C5152
:10A8400002F086FD03F07AF84FF6FF729042A8F10D
:10A85000030328BF1046012B29D9B8F1170F17D8C9
:10A86000174B23FA08F303F0010383F0010223B925
:10A87000B8F1190F0FD0BDE8F883124B124D1349F0
:10A880001A6044EAC9042A6008601C60BDE8F883C5
:10A89000B8F1200FECD10E4B0E4D0F49002244EAC7
:10A8A000C9041A602A6008601C60BDE8F8830B4B7D
:10A8B0000B4D0C49F2E700BF001BB740006CDC02F7
:10A8C0006006F000008003400480034008800340DD
:10A8D00000800B4004800B4008800B400090034038
:10A8E0000490034008900340212801D8FFF73CBDA5
:10A8F000704700BF212806D8044B53F8303093F836
:10A900000002C0B270470020704700BF6805010018
:10A91000212801D8FFF74ABD704700BF72B60C4925
:10A920000C4B0D4A1B680868126862B6520102D5CA
:10A93000322B88BF01300949C3F5BB334FF47A721B
:10A94000FF33A1FB031302FB00F000EB93107047F1
:10A950005C9DFF1F18E000E004ED00E0ABAAAAAA8E
:10A960002DE9F843054672B6204F214B214A1B685A
:10A970003C68126862B6520102D5322B88BF01349E
:10A9800095B3C3F5BB331C4EDFF86490DFF86480E9
:10A99000FF334FF47A72A6FB031302FB04F404EBBB
:10A9A000931472B6D9F800103A68D8F800E062B68D
:10A9B000C1F5BB33FF33A6FB03031EF0806FC4EB6E
:10A9C00093134FF47A7002D0322988BF013200FB12
:10A9D0000233B3F57A7F04D3013D05D004F57A74D0
:10A9E000DFE701F029FCDCE7BDE8F8835C9DFF1F91
:10A9F00018E000E004ED00E0ABAAAAAAF8B52D4BE0
:10AA00002D49DFF8D0E0DFF8D0C02C4E2C4D2D4C76
:10AA10002D4A2E4F4FF4000018604FF080701860E0
:10AA20004FF0007018604FF0806018604FF00060C9
:10AA300018600020086028234BF6FF71CCF8001046
:10AA4000CEF80030336013602B6023603B60B3624C
:10AA50009362092245F8242CC4F8D80F05F57F65C8
:10AA6000C7F8D41F07F5FF2707F5FA67C6F8F83FC0
:10AA70002B6006F5FF26C4F8D42F05F5FD2504F557
:10AA8000FF24386006F2F4761148316005F5FF6561
:10AA900004F5FD642B6023600260FFF76BF9192059
:10AAA000FFF75EFF00F0B6FF40F21310BDE8F8407C
:10AAB000FFF756BF08E100E0048003401480034024
:10AAC000248003402C8003401C80034034800340DA
:10AAD00000800B400C800340088003402DE9F84FB4
:10AAE000214B1B6807460BB101221A70DFF88890D2
:10AAF0001E4D99F80040DFF884801D4E0134272C4C
:10AB00008ABF4FF0000A5FFA84FA5446AB462B78AE
:10AB1000A34216D1FFF7E2FB40281FDC33791B0666
:10AB2000F5D59BF800300133272B86BF0022134652
:10AB3000DAB218F80330DBB2F3712A702B78A34233
:10AB4000E8D00C490A4BFFB208F804700120AC228F
:10AB5000087089F800A0DA70BDE8F88FFF28D6DD0C
:10AB600001F06AFBD3E700BFD49DFF1FD19DFF1FFB
:10AB700000C00640D09DFF1FD89DFF1F689DFF1F8E
:10AB80001C4BDFF894C01A681B49F0B542F48052A0
:10AB90001A4D1A60DFF884E0194F1A4E1A4C002340
:10ABA0008CF800304FF451722B701F2840F213358F
:10ABB0008EF800303B70337025600A6012D8194659
:10ABC0000124124A124D11701248547000212C2792
:10ABD000402693724FF4003491701174D7702E7028
:10ABE0000460F0BDC0F34431C0F3471400F01F030C
:10ABF000E7E700BF348004400CC00440659DFF1FA0
:10AC0000D19DFF1FD09DFF1F08C0044000C006401B
:10AC100031E400E004E100E0649DFF1FD89DFF1FC8
:10AC2000034B1B68DB0401D5FFF758BF704700BF1B
:10AC30003480044010B5044C237823B101F0FCFAB1
:10AC40002378002BFAD110BDD09DFF1F054A064B7B
:10AC500010781B78C0B2DBB2984238BF4030C01ABF
:10AC6000704700BF649DFF1F659DFF1F30B42B4BD5
:10AC70001A7994061FD52A48DA79037829490133CD
:10AC80003F2B0978C8BF00238B42D2B203D0264C99
:10AC9000D9B2E2540170254A116861B1244A127890
:10ACA000D2B2934236BFC2F140029B1A9B18272BA7
:10ACB000C4BF01230B70194AD378DBB2180611D434
:10ACC0005A060DD5154B1B795B0609D5194B1A4948
:10ACD0001B6800220A7003B11A70104B2C22DA7024
:10ACE00030BC704711790906EAD5144910480C7830
:10ACF0000178C9B28C420DD04A1C272A84BF00219A
:10AD00000A460F4D054C98BFD1B2AA5CD2B2E2718F
:10AD10000170D5E76C21D170D2E700BF00C00640BA
:10AD2000649DFF1F659DFF1F909DFF1F609DFF1F7E
:10AD3000D19DFF1FD49DFF1FD09DFF1FD89DFF1FDA
:10AD4000689DFF1F21282FD8184B195CFF292BD095
:10AD5000174B184ADFF870C003EBC000F0B543682A
:10AD6000DFF868E0144F154D154E00241C60DEF826
:10AD70000030012043F020038840CEF800301460FA
:10AD80004FF4A07338602E60C2F800C0013BFDD1C3
:10AD900013689B05FCD42023013BFDD1094B09B26C
:10ADA00033F8110080B2F0BD002070477806010032
:10ADB000680501000050044008500440045004405D
:10ADC000000002030051044080014A003880044022
:10ADD000431E032B14D872B60A4951F8230068B1F8
:10ADE00070B4094C058834F81320466841F8236094
:10ADF000521B24F8132062B670BC704762B67047CD
:10AE000000207047349EFF1F78A0FF1F01380328E1
:10AE10000BD872B6074B53F8203043B100205B6863
:10AE20000130002BFBD162B67047002070471846F6
:10AE3000F9E700BF889EFF1F30B472B62B4A137823
:10AE40001D0706D52A4B196A002936D0996A0029B0
:10AE500041D053781C0706D5254B196C00293ED0EC
:10AE6000996C002939D09378190705D5204B196EB4
:10AE7000002936D0996E89B1D3781B0707D51C4BB2
:10AE8000D3F880207AB3D3F8882011213AB162B682
:10AE9000184B00221A7030BC00F04ABE0D21154C30
:10AEA000154D227843F8315003EBC1030830013AC5
:10AEB0005860227062B630BC704704220D4C0F4DB2
:10AEC000217843F8325003EBC20308304A1E586021
:10AED000227062B6EFE70521E1E70921DFE70822EA
:10AEE000ECE70C22EAE71022E8E700BF9C0601002D
:10AEF0000080FF1FB19EFF1FC80040008800400077
:10AF0000431E032B1DD81B4A400140F0100030B4F3
:10AF1000104472B6184CE25C032A1BD8DFE802F03A
:10AF20000212151703220D88E25410F0080F14BF07
:10AF3000C823882343EA054308310360416062B6B1
:10AF400030BC704708300222EDE70522EBE70830FD
:10AF50000422E8E7094A52F8230038B1084A52F8B7
:10AF60002300416042F8231062B6E9E742F823105B
:10AF7000034AF7E70080FF1FC09EFF1F889EFF1F48
:10AF8000989EFF1F00BE70472DE9F04FDFF818B301
:10AF9000DFF818A387B044E0AD4F4FEA930807EB02
:10AFA000C809013ED9F8042003F00803F6B2A2F163
:10AFB000080003F0FF04002B40F0018157F83830FF
:10AFC0001B0C99B222F8081C002B00F0EF80A14B5B
:10AFD00022F8064C42F8044C53F82620002A00F0D0
:10AFE000CF819D4D55F8263058609C4C45F8260081
:10AFF00034F81630194424F8161000F079FD0028B2
:10B0000000F0C281964A974B19F0080F00F1080032
:10B0100018BF1346C9F8040047F8383008238BF8E6
:10B0200000309BF80040E4B265071CD58E4B1B78BE
:10B03000B3B18E490A7802F0FF0322B1013BDBB2C3
:10B040000B7003B900BE8A490A7802F0FF032AB1E7
:10B05000013BDBB20B70002B00F0688100F066FE54
:10B0600004238BF8003004F0080303F0FF02002BE8
:10B0700000F0C9809AF80030DBB21E098CD19A0822
:10B08000DFF8CC9159F8321009EBC200C1F383010B
:10B09000013940680C2900F28580DFE801F07A7AF6
:10B0A0008383838383834683838307000168714D91
:10B0B0004068714F714E6860296088B240F28161CA
:10B0C0000024674B49F832304FF0010E88423C6053
:10B0D000C9F81040C9F8184086F800E05C4A00F250
:10B0E000E780B0F5D06F80F01B82B0F5817F00F073
:10B0F000D98100F26981802800F02A82822840F0FC
:10B10000D781A98801F07F01042900F2D1815C4830
:10B110005C4A890008441470547001788C0740F12F
:10B12000608382F800E0022173E1534F3A682AB34A
:10B13000554B524E554819883478057840298E462B
:10B1400045F0020828BF4FF0400E002C84F00104A7
:10B150003470CEEB01010CBF8824C82409EBC8066B
:10B1600089B285F0010544EA0E447260198049F8FD
:10B17000384072440570002965D03A603D4B1A880A
:10B18000B2F5A06F0ED100219A785970404B1A7019
:10B1900008E038493F4C0D68A54200F098803049DE
:10B1A00049F832103C4A0123137037E72C4A2D4BE3
:10B1B00019F0080F18BF134647F838302EE700F093
:10B1C000B7FC364A364952F82630002B00F0E380AF
:10B1D00058688C5D42F8260003F10802C9F8042083
:10B1E000032C05D8DFE804F02C02292602228A5518
:10B1F0001A8819F0080F0CBF8823C82343EA0243BA
:10B2000047F838300AE7E00700F19380210600F1A3
:10B21000D180A20706D5234A234913780220DBB246
:10B2200013700870E30602D51F4B10221A7007B086
:10B23000BDE8F08F04228A55DAE705228A55D7E760
:10B2400003228A55D4E7BEF1400F18BF002294E7CD
:10B250000080FF1F349EFF1FE09DFF1F78A0FF1F8F
:10B26000C800400088004000BC9EFF1F459EFF1F95
:10B27000309FFF1FA89EFF1FDC9DFF1F449EFF1FE6
:10B28000C0200740B49EFF1FF09DFF1FB09EFF1F10
:10B29000982007402109000394200740889EFF1F43
:10B2A000C09EFF1F88200740802007409020074055
:10B2B000B0F5106F00F07C8140F2A38040F62112BF
:10B2C000904240F07B82A54A012313706AE74C68E4
:10B2D000A3498C427FF463AF0178A9297FF45FAF63
:10B2E000417845297FF45BAF8178C2297FF457AF5D
:10B2F000C1786B297FF453AF9A489B4E017834781C
:10B3000081F00105002C41F0020105700CBF88207E
:10B31000C82084F0010449F8310009EBC1019348C9
:10B320003470002505244D60047038E700F064FF98
:10B3300094E68F4B89488B491A614FF0020E80F8D2
:10B3400000E08C4F0A708C49196099608B4E8C4DCF
:10B350008C4C9A610D213970FF213170DFF84CE27D
:10B3600029702270884D894A8EF800109F27012489
:10B3700006F8047C5D600470DA6007B0BDE8F08F09
:10B3800043F82600824D30E6824A47F838001378A9
:10B390000133137042E68B5D032B00F2BA8001A2E9
:10B3A00052F823F01DB000001DB00000FDB30000F6
:10B3B000F7B300006F49724B80220D2008701A709D
:10B3C000A2077FF52FAF26E740F20232904240F00D
:10B3D000ED81AA8802F07F02042A69D86D88002DC9
:10B3E00066D16449CDF804E0920011440A7842F035
:10B3F00002020A70C1E101238B550FE600238B5531
:10B400000CE6B0F5086F53D16349644A09781170AE
:10B410007146ED888D4280F0E88252480478402DD4
:10B42000AE4644F0020C28BF4FF0400E02EB0E0374
:10B4300009EBCC01029301234A604FEA0E48CEEBA0
:10B44000050101930025C82242EA080384F00102A5
:10B4500049F83C3035700270DFF814C1424BDFF818
:10B46000048149BBBEF1400F7FF42DAF42F0020CC6
:10B4700009EBCC03029ADFF8F8E05A608DBB0D04AB
:10B4800045F088059DF804304EF83C500A4433706E
:10B490000470134640297FF416AF0021404A3B60F8
:10B4A000118010E7AA8802F07F02042A40F28B8103
:10B4B000304A0F23137006E74029D7D942F0020221
:10B4C0000CEBC200029E4660BDB19DF804503548A9
:10B4D0001D703346403988F8004040334CF8320044
:10B4E000DCE79DF8043033700D04029B047045F0D6
:10B4F000C8050B444EF83C50CCE79DF804501D7035
:10B50000029B1D4888F80040403940334CF8320017
:10B51000C4E719F0080F0CBF022303238B557DE508
:10B5200021494A68002AC3D06C88B5F804E003E0DA
:10B530000C314A68002ABBD00B88A342F8D14B8853
:10B540007345F5D1240A032C0CBF1178098960E7F3
:10B55000124A0221147054705BE700BF9420074028
:10B5600001000400B09EFF1F449EFF1F459EFF1F69
:10B570000080FF1FC020074088004000882007404F
:10B580008020074098200740F49DFF1F489EFF1F22
:10B59000E09DFF1FB19EFF1FBC9EFF1FB49EFF1FBB
:10B5A000F09DFF1FC8004000A00601008C2007404E
:10B5B000B248116AAC7804700C0600F19881D9F891
:10B5C0002820AF49100600F1DB81D9F83020AC49C2
:10B5D000120600F1D081D9F83820A949130600F1EC
:10B5E000C581D9F84020A649150600F1BA81D9F8DD
:10B5F0004820A349140600F1AF81D9F85020A04992
:10B60000100600F1A481D9F858209D49120600F1D6
:10B610009981D9F860209A49130600F18E81D9F8F2
:10B6200068209749150600F18381D9F87020944964
:10B63000140600F17881D9F878209149100600F1BC
:10B640006D81D9F880208E49120600F16181D9F808
:10B6500088208B49130600F15581D9F8902088493C
:10B66000150600F14981D9F898208549140600F1A2
:10B67000FF808448844A854901908548854D864CE1
:10B68000049700230596029580460F4616461D46F0
:10B690000394306828B1446800F04AFA2046002C30
:10B6A000F9D100233360029B38681A46002342F820
:10B6B000253028B1446800F03BFA2046002CF9D12F
:10B6C00000223A60019A98F800301146002241F8B1
:10B6D000042B039A0191023B4FF0000122F8151050
:10B6E000032B07D8DFE803F05D025D024FF0010392
:10B6F00088F800300135042D06F1040607F104072F
:10B7000008F10108C5D1654C654D2278654B049F51
:10B71000059E0021100729701A7000F1928062497D
:10B7200062780A700021C9F83010C9F83810110782
:10B73000DFF84C816ED4A2785C49DFF844810A704E
:10B7400000211207C9F85010C9F858104BD4E278FC
:10B7500057494B4C0A7013074FF00001C9F870109D
:10B76000C9F8781000F1AE8033780193002283F09D
:10B770000105C9F89020C9F8982000210291884657
:10B780008E460A464B48047844F0020C09EBCC0381
:10B790000393019B002B039B5A600CBF8822C82295
:10B7A00052E64FF0000388F80030A3E7B0F5A06F31
:10B7B0007FF47EAE012300250193DEE740F62122CF
:10B7C0009042F7D074E66D88002D7FF471AE3A494F
:10B7D000CDF804E0920011440A7822F002020A70C7
:10B7E000CBE7022115E600F083F9002800F0EB809A
:10B7F0000830324AC8F86400C8F8602000F078F9D0
:10B80000002800F0DA8008302D4AC9F86C00C9F829
:10B8100068209CE700F06CF9002800F0E080083018
:10B82000264AC8F84400C8F8402000F061F9002812
:10B8300000F0CF800830224AC9F84C00C9F84820EF
:10B8400079E700F055F9002800F0A58008301B4A80
:10B85000C9F82400C9F8202000F04AF9002800F0B7
:10B8600094800830164AC9F82C00C9F8282056E7F9
:10B87000D1F89C00083800F05BF9FAE6BC9EFF1F87
:10B880000080FF1F989EFF1F349EFF1F889EFF1F92
:10B89000C09EFF1FE09DFF1F78A0FF1F9C060100B8
:10B8A000B19EFF1FC4200740C8200740CC2007409E
:10B8B000D0200740B09EFF1FC020074088004000F6
:10B8C000C800400000F014F9002870D008304F4A3A
:10B8D000C4F88400C4F8802000F00AF9002860D081
:10B8E00008304B4AC9F88C00C9F888203CE7506AF8
:10B8F000083800F01DF962E6D1F89400083800F02D
:10B9000017F9B0E6D1F88C00083800F011F9A4E678
:10B91000D1F88400083800F00BF998E6C86F0838B1
:10B9200000F006F98DE6486F083800F001F982E66C
:10B93000C86E083800F0FCF877E6486E083800F06A
:10B94000F7F86CE6C86D083800F0F2F861E6486D6B
:10B95000083800F0EDF856E6C86C083800F0E8F852
:10B960004BE6486C083800F0E3F840E6C86B08384E
:10B9700000F0DEF835E6486B083800F0D9F82AE622
:10B98000C86A083800F0D4F81FE62A78C9F82800F9
:10B9900001322A70C3E62A78C9F8200001322A70E1
:10B9A0005AE72A78C9F8880001322A70DCE62A783A
:10B9B000C4F8800001322A708EE72A78C9F868003E
:10B9C00001322A70C3E62A78C8F8600001322A7072
:10B9D00014E72A78C9F8480001322A70ABE62A78C1
:10B9E000C8F8400001322A701FE740298E4628BF60
:10B9F0004FF0400E02EB0E0302930123CEEB010148
:10BA00004FEA0E4800250193BCE600BF88004000C5
:10BA1000C8004000F8B500F08FFD294B29482A4C9A
:10BA20002A4F2B4DDFF8BCC0DFF8BCE0294E0022C6
:10BA30001A605A609A60DA601A615A619A61DA6132
:10BA40001A625A629A62DA621A635A639A63DA6312
:10BA50001A645A649A64DA641A655A659A65DA65F2
:10BA60001A665A669A66DA661A675A679A67DA67D2
:10BA7000C3F880200168C3F8842041F4802101606C
:10BA8000C3F307212170C3F30740134938701B0E1D
:10BA90002B70FF238CF80030104D8EF800301048CA
:10BAA0000B700123337084F8642070264FF4007407
:10BAB000102207F82C3C2E70046081F8F820F8BDA5
:10BAC0000080FF1F348004409C200740B0200740C6
:10BAD000B4200740942007401020074049E400E0CC
:10BAE00008E100E08020074088200740704700BF41
:10BAF00072B60D480268B2FA82F30F2B10DC4FF0D9
:10BB00000041D94022EA0102026062B6074803EB15
:10BB1000C303DB00C2180021C150104651607047BA
:10BB200062B60020704700BF8091FF1FBC83FF1FDB
:10BB30000D4B0E4AC31AA2FB03231B090F2B0CD873
:10BB40000B4A127852B972B60A484FF000410268A7
:10BB500021FA03F31A43026062B67047064A12786C
:10BB6000002AF0D0FFF768B9BC83FF1F398EE33895
:10BB7000B19EFF1F8091FF1FBC9EFF1F38B50E4B6B
:10BB80000E4C1B68218805468BB1B1F5917F05D21B
:10BB90000B4A4B1C55549BB2238038BD00220848E9
:10BBA00098470021064A55540123238038BDB1F53A
:10BBB000917FEDD338BD00BFE89EFF1F82A0FF1F1D
:10BBC00088A0FF1F2DE9F843214E224F3168012341
:10BBD00080463B70B1B1204D4B8801EB83020133AD
:10BBE00000240F2BC2F808802C7004D84B8000234F
:10BBF0003B70BDE8F88340230B800320FFF780F9FA
:10BC00003460F4E7DFF8549099F80030002BF0D05E
:10BC1000114D45F6215408E0013C12D02B7883B930
:10BC200000F00AFB99F800307BB10320FFF7EEF833
:10BC30000528F1D8FFF75CFF014630600028EBD003
:10BC4000CAE701232B70BDE8F883BDE8F88300BF85
:10BC5000049FFF1FD89EFF1F089FFF1FBC9EFF1F52
:10BC60001201F8B5D5B2A1B3012943D043780446F7
:10BC700000781B0643EA004040F4704045F004069B
:10BC80008F1E3043FFF79EFF022F04F1020314D9E9
:10BC9000053414F8023C14F8032C14F8010C1B04AE
:10BCA00043EA0223334343EA0060033FFFF78AFF7E
:10BCB000022F234604F10304EBD8022F23D0012FD7
:10BCC0000DD045F4774040F00500BDE8F840FFF79F
:10BCD00079BF14482843BDE8F840FFF773BF1878D0
:10BCE00045F4770545F0060545EA0020BDE8F84033
:10BCF000FFF768BF03780C4845EA03452843BDE8D1
:10BD0000F840FFF75FBF1A78587845F0774545F05F
:10BD1000070545EA022545EA0040BDE8F840FFF77F
:10BD200051BF00BF06F0F70007F000F738B5084B29
:10BD30001C7824B9074D296809B14B8803B938BD6F
:10BD40009B000B800320FFF7DBF82C6038BD00BFA1
:10BD5000D89EFF1F049FFF1F2DE9F041AD4E3368B1
:10BD60000746002B00F092801D885A88910803EB4B
:10BD700081010432AA428C6842D25A8004F00F0634
:10BD80004FEA1428A449A6F1080208F00F00C4F3F2
:10BD90000313062A00F101050B701AD9B31E012BFB
:10BDA0005FFA88F04ED9052E48D0042E00F0A48109
:10BDB000731F022B7FD90F2E0ED1F72842D8F028FF
:10BDC00002D0964B1B883BB1FFF7D8FE0020BDE8A0
:10BDD000F08127B1BD4202D00020BDE8F081082EDD
:10BDE000C4F3033300F08780092E11D00A2E40F0EF
:10BDF00094800A2BF0D18A4B8A4A1B68A02181E0EB
:10BE00001846FFF795FE0420FEF7E2FF3060B5E725
:10BE1000092BE1D1270E00F07B81834B814A1B68FF
:10BE20009021C4F307461170EDB2FCB2002B00F074
:10BE30009D80224631462846984797E0F02843D90E
:10BE4000F72841D0F1380E28C6D801A353F820F0C6
:10BE500007C00000EBBF0000D9BF0000D9BD000043
:10BE6000D9BD0000CBBF0000D9BD0000ABC00000B1
:10BE7000D9BD000075C000008FC00000B3BF000036
:10BE8000D9BD00009BBF00007FBF0000674B1B783F
:10BE9000002BA1D00420FEF79BFF03463060002852
:10BEA0009AD00588002D7FF460AFFFF741FE356022
:10BEB0002846BDE8F081FFF761FEC4F30740FFF7B5
:10BEC0005DFE072E02D1200EFFF758FE534B584A55
:10BED000198858481468584D524A017000270E0AB4
:10BEE000F0201F802E7010700CB301225348A04721
:10BEF0000120BDE8F081082B7FF46EAF504B494A1A
:10BF00001B688021C4F307461170EDB2240E6BB399
:10BF1000284622463146984728E00B2E11D10B2B9C
:10BF20007FF45AAF474B3F4A1B68B021EAE7464BC4
:10BF30001B68002B00F0FB80404898470120BDE8BB
:10BF4000F0810C2E40F000810C2B7FF445AF3F4B6D
:10BF5000344A1B68C0211170EDB2C4F30746002BB0
:10BF600000F0C88028463146240E98473849314AA7
:10BF7000314B0D7016701C700120BDE8F081354BFF
:10BF80001B68002B00F0D6809847C4F30746254B6A
:10BF9000EDB2240E83F80080E8E72F4B1B68002BDE
:10BFA000F2D12E4B1B68A3B1FE209847C4F307467D
:10BFB000EDE72B4B1B68002BE6D1284B1B6843B1E8
:10BFC000FC209847C4F30746E1E7264B1B68002B8B
:10BFD000DAD1C4F30746DAE7234B1B68C4F30746FC
:10BFE000002BD4D030469847D1E7204B1A68002A5E
:10BFF000EFD0260C630C06F07F0003F47E53184349
:10C00000F6B29047C3E71A4B1B68C4F30746002BF0
:10C01000E8D1BCE7109FFF1F86A0FF1F82A0FF1F73
:10C02000EC9EFF1F80A0FF1F209FFF1FBC9EFF1FD5
:10C03000E89EFF1F84A0FF1F85A0FF1F88A0FF1F91
:10C04000189FFF1F1C9FFF1F009FFF1FDC9EFF1FED
:10C0500087A0FF1FC89EFF1FCC9EFF1FD09EFF1F03
:10C060000C9FFF1FFC9EFF1F149FFF1FE49EFF1FDE
:10C07000F89EFF1F3F4B1B68002B85D13E4B1B6872
:10C08000002BA6D0FA209847C4F307467FE73B4B26
:10C090001B68002B7FF478AF374B1B68002B98D0C0
:10C0A000FB209847C4F3074671E7354B1B68002B0C
:10C0B0007FF46AAF304B1B68002B8AD0F82098477A
:10C0C000C4F3074663E70E2B7FF486AE2D4A2E4B52
:10C0D0001268E0211970002A47D0260C610C06F086
:10C0E0007F0301F47E511943EDB2A1F500512846BA
:10C0F0009047F6B2240E39E7FFF740FDC4F307403E
:10C10000FFF73CFD200EFFF739FD0020BDE8F08170
:10C110001E4B1D4A1B6880211170EDB2C4F3074607
:10C1200083B1314628463A4698473C461EE70120EF
:10C13000BDE8F081104B1B68002B3FF44AAFFF2095
:10C14000984746E71C4611E70D2EBCD10D2B7FF416
:10C1500043AE0F4B0C4A1B68D0211170EDB2C4F3F3
:10C160000746002B7FF4FEAEC4E7C4F30746EDB2EA
:10C17000240EFBE6F49EFF1FD09EFF1FD49EFF1FE0
:10C18000C49EFF1FE09EFF1F80A0FF1F189FFF1F80
:10C19000F09EFF1F38B5164D2868E0B1018844882D
:10C1A000A14213DD03191B7A83B104F10803C218FD
:10C1B0000C1B002302E012F8011F21B10133A3423E
:10C1C000F9D1204638BD1C46204638BDFFF7B0FCEB
:10C1D0000020286038BD074B1B780BB9002038BD04
:10C1E0000220FEF7F5FD28600028D7D1F6E700BF52
:10C1F0002C9FFF1FBC9EFF1F0D4B1B78BBB910B5BA
:10C200000C4C216803F0FF024B883F2B07DC0733FF
:10C210000B4401F1470003F8012F8342FBD1402377
:10C220000B800120FEF76CFE0023236010BD7047D9
:10C23000249FFF1F289FFF1F38B5224C237803B18E
:10C2400038BD01232370FFF7A5FF70BB00F048F84D
:10C2500040BB00F0DBF810BBFEF7F8FCE0B90023B0
:10C260002370EFF30583002BEAD1EFF3108172B650
:10C27000154B1868E0B1154C2278CAB945691D60A4
:10C2800001232370C5B1AA6101B962B600254577C3
:10C29000836898472570D3E700F020F8DFE700F0C7
:10C2A0001BF8D9E700F016F8D3E7FFF71FFCCDE73E
:10C2B0000029C5D162B638BD054B1D600029E5D106
:10C2C000E3E700BF319FFF1F489DFF1F4C9DFF1FED
:10C2D000449DFF1F704700BF704700BF704700BFFD
:10C2E000054A064B10781B78C0B2DBB2984238BFC3
:10C2F0004030C01A704700BF389FFF1F399FFF1F93
:10C30000F0B4384B1A7912F0300F2CD072B6997DF8
:10C3100001F0FF0200293DD062B6334F334938782F
:10C320000D78334E1C46C0B2EDB2431C402BE17970
:10C3300028BF0023AB4202F1FF32C9B21CBFF15447
:10C34000184612F0FF02F0D12A4B1B68C2B23A70B5
:10C350004BB1A84236BFC5F14005401B4019272804
:10C36000C4BF01221A701F49CA78D2B2150616D46A
:10C3700052060DD51B4B1B795B0609D51E4B1F4979
:10C380001B6800220A7003B11A70164B3C22DA7047
:10C39000F0BC70474022D9795A7462B6E3E70B7952
:10C3A0001C06E5D5164B174E1C783378E4B2DBB289
:10C3B0009C420ED0144D01E0A3420AD00133402B21
:10C3C00028BF00230879E85CC0B2C871087D07283F
:10C3D000F2D9DBB2034933700B79180644BF7C23D2
:10C3E000CB70C5E700A00640389FFF1F399FFF1F95
:10C3F0007C9FFF1F349FFF1FC09FFF1FBC9FFF1F1D
:10C40000C49FFF1FBD9FFF1F3C9FFF1F054A064B98
:10C4100010781B78C0B2DBB2984238BF4030C01AE7
:10C42000704700BF38A0FF1FCD9FFF1FF0B4384BEF
:10C430001A7912F0300F2CD072B6997D01F0FF02FC
:10C4400000293DD062B6334F334938780D78334EEA
:10C450001C46C0B2EDB2431C402BE17928BF00233B
:10C46000AB4202F1FF32C9B21CBFF154184612F0C0
:10C47000FF02F0D12A4B1B68C2B23A704BB1A842FE
:10C4800036BFC5F14005401B40192728C4BF012213
:10C490001A701F49CA78D2B2150616D452060DD5A5
:10C4A0001B4B1B795B0609D51E4B1F491B680022DD
:10C4B0000A7003B11A70164B3C22DA70F0BC704758
:10C4C0004022D9795A7462B6E3E70B791C06E5D5A8
:10C4D000164B174E1C783378E4B2DBB29C420ED078
:10C4E000144D01E0A3420AD00133282B28BF0023BA
:10C4F0000879E85CC0B2C871087D0728F2D9DBB2C0
:10C50000034933700B79180644BF7C23CB70C5E711
:10C5100000B0064038A0FF1FCD9FFF1FF89FFF1FF0
:10C52000C89FFF1F3CA0FF1FCC9FFF1F40A0FF1F05
:10C5300039A0FF1FD09FFF1F70B584B072B6194B92
:10C54000194D1A48702241260F2480211A702E702E
:10C550001A460470197013781B06FCD5144B186822
:10C5600062B6144B144C984298BF00EB800001A9AE
:10C5700098BF40000A22FDF7CFFE01A92046002304
:10C5800011F8012B01333AB10A2B20F8022FF7D111
:10C590001623237004B070BD5B00DBB2237004B0BF
:10C5A00070BD00BF000002400700024006000240CC
:10C5B000080002407F9698004C92FF1FFFFFFFFF8C
:10C5C0002DE9F043DFF8EC808BB006460F4600F013
:10C5D00073F898F90030013304460D4637D03046E1
:10C5E000394600F0DFF9002831D02BA3D3E900232E
:10C5F0003046394600F026FE814668BB28A3D3E9C1
:10C6000000233046394600F0FFFD00B398F90030B2
:10C61000254ACDF82090042400200021022BCDE9EA
:10C620000467CDE9026700940192CDE906012CD0A0
:10C63000684600F0BDF940B3089B1BB101F0AAF9B0
:10C64000089B0360DDE906010BB0BDE8F0832046DE
:10C6500029460BB0BDE8F083134A98F900300192E7
:10C6600003210022CDE90467CDE902670091089219
:10C670002BB90E4B4FF06042CDE90623D8E70C49A9
:10C680000020022BCDE90601D2D101F083F922234B
:10C690000360D1E7AFF30080EF39FAFE422E864007
:10C6A00051302DD5104987C00C070100FFFFEF471F
:10C6B0000000F07F6292FF1F2DE9F04FB04F21F094
:10C6C0000042BA4283B00C464FEAD17605460DD9F6
:10C6D000AC4FBA4225D9C1F31303034340F0EF80B6
:10C6E0000EB10020014603B0BDE8F08FA64B9A4280
:10C6F00000F2CC80A54B9A4200F2DE808AA3D3E9F7
:10C70000002300F05DF90022A14B00F09BFD002802
:10C7100000F005812846214600229D4B00F050F98B
:10C72000E1E783A3D3E9002300F08CFD002840F06B
:10C73000CB802846214680A3D3E9002300F064FD86
:10C740000028CED1934B284603EBC60821467CA394
:10C75000D3E9002300F0E6FAD8E9002300F030F92D
:10C7600000F07AFD804600F077FA77A3D3E9002342
:10C7700006460F4600F0D6FA02460B4628462146EA
:10C7800000F01CF972A3D3E90023CDE90001304683
:10C79000394600F0C7FA82468B4652465B46DDE9D1
:10C7A000000100F00BF905460C462A4623462846B0
:10C7B000214600F0B7FA68A3D3E9002306460F46E6
:10C7C00000F0B0FA66A3D3E9002300F0F7F8324690
:10C7D0003B4600F0A7FA64A3D3E9002300F0F0F889
:10C7E00032463B4600F09EFA61A3D3E9002300F0F5
:10C7F000E5F832463B4600F095FA5FA3D3E9002303
:10C8000000F0DEF832463B4600F08CFA02460B465A
:10C810002846214600F0D2F806460F462846214613
:10C8200032463B46B8F1000F56D000F07BFA324654
:10C8300004460D463B4600204FF0804100F0BEF814
:10C8400002460B462046294600F096FB02460B4660
:10C850005046594600F0B2F8DDE9002300F0AEF88A
:10C860000B4602464A49002000F0A8F86FF47F7397
:10C8700098454FDA08F57A7801EB085100224FF01D
:10C88000B87300F04FFA03B0BDE8F08F424B9A4204
:10C890003FF658AF414BF4002344D3E9002300F0A6
:10C8A0008DF83F4BC6F101081C44CDE90001D4E9E5
:10C8B00000ABC6EB080870E74FF0000875E70246CA
:10C8C0000B4600F07DF80EE717A3D3E900231046CE
:10C8D000194600F027FA06E700F024FA0022804605
:10C8E00089464FF080433046394600F067F80246EB
:10C8F0000B464046494600F03FFB2A46234600F0DF
:10C900005DF802460B460020214900F057F803B0BD
:10C91000BDE8F08F01EB085103B0BDE8F08F804611
:10C9200043E700BFAFF300809C7500883CE4377E8E
:10C93000EF39FAFE422E864051302DD5104987C07E
:10C94000FE822B654715F73F0000E0FE422EE63FD2
:10C95000763C7935EF39EA3DD0A4BE726937663E40
:10C96000F16BD2C541BDBB3E2CDE25AF6A56113FEF
:10C9700093BDBE166CC1663F3E5555555555C53FD6
:10C98000412E8640FFFFEF7F422ED63FFFFF2F3E16
:10C990000000F03F10070100B1A2F03F3007010096
:10C9A0002007010041F0004101F58010C00F7047E1
:10C9B0000020704781F0004102E000BF83F0004397
:10C9C00030B54FEA41044FEA430594EA050F08BF2A
:10C9D00090EA020F1FBF54EA000C55EA020C7FEAEE
:10C9E000645C7FEA655C00F0E2804FEA5454D4EB6B
:10C9F0005555B8BF6D420CDD2C4480EA020281EA35
:10CA0000030382EA000083EA010180EA020281EA6C
:10CA10000303362D88BF30BD11F0004F4FEA0131BE
:10CA20004FF4801C4CEA113102D0404261EB4101CD
:10CA300013F0004F4FEA03334CEA133302D0524253
:10CA400063EB430394EA050F00F0A780A4F101040F
:10CA5000D5F1200E0DDB02FA0EFC22FA05F2801849
:10CA600041F1000103FA0EF2801843FA05F359412F
:10CA70000EE0A5F120050EF1200E012A03FA0EFCAE
:10CA800028BF4CF0020C43FA05F3C01851EBE371D8
:10CA900001F0004507D54FF0000EDCF1000C7EEBF5
:10CAA00000006EEB0101B1F5801F1BD3B1F5001F33
:10CAB0000CD349085FEA30004FEA3C0C04F1010452
:10CAC0004FEA445212F5800F80F09A80BCF1004F7B
:10CAD00008BF5FEA500C50F1000041EB045141EAFD
:10CAE000050130BD5FEA4C0C404141EB010111F4FE
:10CAF000801FA4F10104E9D191F0000F04BF0146A9
:10CB00000020B1FA81F308BF2033A3F10B03B3F186
:10CB100020020CDA0C3208DD02F1140CC2F10C0216
:10CB200001FA0CF021FA02F10CE002F11402D8BF74
:10CB3000C2F1200C01FA02F120FA0CFCDCBF41EA40
:10CB40000C019040E41AA2BF01EB0451294330BD0F
:10CB50006FEA04041F3C1CDA0C340EDC04F11404EC
:10CB6000C4F1200220FA04F001FA02F340EA0300C3
:10CB700021FA04F345EA030130BDC4F10C04C4F109
:10CB8000200220FA02F001FA04F340EA03002946E9
:10CB900030BD21FA04F0294630BD94F0000F83F433
:10CBA000801306BF81F480110134013D4EE77FEA16
:10CBB000645C18BF7FEA655C29D094EA050F08BF62
:10CBC00090EA020F05D054EA000C04BF1946104643
:10CBD00030BD91EA030F1EBF0021002030BD5FEA87
:10CBE000545C05D14000494128BF41F0004130BDAF
:10CBF00014F580043CBF01F5801130BD01F0004503
:10CC000045F0FE4141F470014FF0000030BD7FEA75
:10CC1000645C1ABF194610467FEA655C1CBF0B4670
:10CC2000024650EA013406BF52EA033591EA030F87
:10CC300041F4002130BD00BF90F0000F04BF00217F
:10CC4000704730B54FF4806404F132044FF00005B2
:10CC50004FF0000150E700BF90F0000F04BF00212B
:10CC6000704730B54FF4806404F1320410F0004591
:10CC700048BF40424FF000013EE700BF42004FEA8C
:10CC8000E2014FEA31014FEA02701FBF12F07F4309
:10CC900093F07F4F81F06051704792F0000F14BF06
:10CCA00093F07F4F704730B54FF4607401F000454A
:10CCB00021F0004120E700BF50EA010208BF7047A1
:10CCC00030B54FF000050AE050EA010208BF704796
:10CCD00030B511F0004502D5404261EB41014FF4FF
:10CCE000806404F132045FEA915C3FF4DCAE4FF003
:10CCF00003025FEADC0C18BF03325FEADC0C18BFEA
:10CD0000033202EBDC02C2F1200300FA03FC20FA3A
:10CD100002F001FA03FE40EA0E0021FA02F1144487
:10CD2000C1E600BF70B54FF0FF0C4CF4E06C1CEA9C
:10CD300011541DBF1CEA135594EA0C0F95EA0C0F11
:10CD400000F0DEF82C4481EA030621EA4C5123EA84
:10CD50004C5350EA013518BF52EA033541F48011B3
:10CD600043F4801338D0A0FB02CE4FF00005E1FB66
:10CD700002E506F00042E0FB03E54FF00006E1FBB0
:10CD800003569CF0000F18BF4EF0010EA4F1FF04F3
:10CD9000B6F5007F64F5407404D25FEA4E0E6D4133
:10CDA00046EB060642EAC62141EA55514FEAC52044
:10CDB00040EA5E504FEACE2EB4F1FD0C88BFBCF5C0
:10CDC000E06F1ED8BEF1004F08BF5FEA500E50F171
:10CDD000000041EB045170BD06F0004646EA010137
:10CDE00040EA020081EA0301B4EB5C04C2BFD4EB69
:10CDF0000C0541EA045170BD41F480114FF0000E62
:10CE0000013C00F3AB8014F1360FDEBF002001F0CF
:10CE1000004170BDC4F10004203C35DA0C341BDC49
:10CE200004F11404C4F1200500FA05F320FA04F01B
:10CE300001FA05F240EA020001F0004221F000414F
:10CE400010EBD37021FA04F642EB06015EEA430EC2
:10CE500008BF20EAD37070BDC4F10C04C4F12005F2
:10CE600000FA04F320FA05F001FA04F240EA0200A5
:10CE700001F0004110EBD37041F100015EEA430E76
:10CE800008BF20EAD37070BDC4F1200500FA05F296
:10CE90004EEA020E20FA04F301FA05F243EA020315
:10CEA00021FA04F001F0004121FA04F220EA020024
:10CEB00000EBD3705EEA430E08BF20EAD37070BD6A
:10CEC00094F0000F0FD101F00046400041EB01014A
:10CED00011F4801F08BF013CF7D041EA060195F02C
:10CEE000000F18BF704703F00046520043EB0303E6
:10CEF00013F4801F08BF013DF7D043EA06037047D3
:10CF000094EA0C0F0CEA135518BF95EA0C0F0CD0DD
:10CF100050EA410618BF52EA4306D1D181EA030123
:10CF200001F000414FF0000070BD50EA410606BF1D
:10CF30001046194652EA430619D094EA0C0F02D162
:10CF400050EA013613D195EA0C0F05D152EA0336A7
:10CF50001CBF104619460AD181EA030101F00041C5
:10CF600041F0FE4141F470014FF0000070BD41F00E
:10CF7000FE4141F4780170BD70B54FF0FF0C4CF4E8
:10CF8000E06C1CEA11541DBF1CEA135594EA0C0F07
:10CF900095EA0C0F00F0A7F8A4EB050481EA030E54
:10CFA00052EA03354FEA013100F088804FEA03333B
:10CFB0004FF0805545EA131343EA12634FEA022209
:10CFC00045EA111545EA10654FEA00260EF00041CA
:10CFD0009D4208BF964244F1FD0404F5407402D21C
:10CFE0005B084FEA3202B61A65EB03055B084FEAAD
:10CFF00032024FF480104FF4002CB6EB020E75EBAA
:10D00000030E22BFB61A754640EA0C005B084FEAD1
:10D010003202B6EB020E75EB030E22BFB61A75464E
:10D0200040EA5C005B084FEA3202B6EB020E75EB99
:10D03000030E22BFB61A754640EA9C005B084FEA11
:10D040003202B6EB020E75EB030E22BFB61A75461E
:10D0500040EADC0055EA060E18D04FEA051545EA0D
:10D0600016754FEA06164FEAC30343EA52734FEAB6
:10D07000C2025FEA1C1CC0D111F4801F0BD141EA2F
:10D0800000014FF000004FF0004CB6E711F4801F94
:10D0900004BF01430020B4F1FD0C88BFBCF5E06F74
:10D0A0003FF6AFAEB5EB030C04BFB6EB020C5FEA84
:10D0B000500C50F1000041EB045170BD0EF0004ED9
:10D0C0004EEA113114EB5C04C2BFD4EB0C0541EA0B
:10D0D000045170BD41F480114FF0000E013C90E608
:10D0E00045EA060E8DE60CEA135594EA0C0F08BFCC
:10D0F00095EA0C0F3FF43BAF94EA0C0F0AD150EACB
:10D1000001347FF434AF95EA0C0F7FF425AF10465D
:10D1100019462CE795EA0C0F06D152EA03353FF485
:10D12000FDAE1046194622E750EA410618BF52EA02
:10D1300043067FF4C5AE50EA41047FF40DAF52EAD6
:10D1400043057FF4EBAE12E74FF0FF3C06E000BF73
:10D150004FF0010C02E000BF4FF0010C4DF804CD80
:10D160004FEA410C7FEA6C5C4FEA430C18BF7FEA40
:10D170006C5C1BD001B050EA410C0CBF52EA430C6E
:10D1800091EA030F02BF90EA020F0020704710F1EE
:10D19000000F91EA030F58BF994208BF90422CBF7D
:10D1A000D8176FEAE37040F0010070474FEA410C76
:10D1B0007FEA6C5C02D150EA013C07D14FEA430C94
:10D1C0007FEA6C5CD6D152EA033CD3D05DF8040B05
:10D1D000704700BF8446104662468C461946634637
:10D1E00000E000BF01B5FFF7B7FF002848BF10F10E
:10D1F000000F01BD4DF808EDFFF7F4FF0CBF012053
:10D2000000205DF808FB00BF4DF808EDFFF7EAFFCE
:10D2100034BF012000205DF808FB00BF4DF808ED89
:10D22000FFF7E0FF94BF012000205DF808FB00BF7E
:10D230004DF808EDFFF7CEFF94BF012000205DF808
:10D2400008FB00BF4DF808EDFFF7C4FF34BF012015
:10D2500000205DF808FB00BF4FEA410212F5001202
:10D2600015D211D56FF47873B3EB625212D94FEA2D
:10D27000C12343F0004343EA505311F0004F23FA17
:10D2800002F018BF404270474FF00000704750EA6C
:10D29000013005D111F0004008BF6FF00040704729
:10D2A0004FF00000704700BF4FEA4102B2F1E04387
:10D2B00024BFB3F5001CDCF1FE5C0DD901F0004C7D
:10D2C0004FEAC0024CEA5070B2F1004F40EB8300CD
:10D2D00008BF20F00100704711F0804F21D113F1F9
:10D2E0003872BCBF01F00040704741F480114FEA32
:10D2F0005252C2F11802C2F1200C10FA0CF320FABB
:10D3000002F018BF40F001004FEAC1234FEAD323D7
:10D3100003FA0CFC40EA0C0023FA02F34FEA430341
:10D32000CCE77FEA625307D150EA01331EBF4FF0CA
:10D33000FE4040F44000704701F0004040F0FE40E5
:10D3400040F40000704700BF80F0004002E000BFE2
:10D3500081F0004142001FBF5FEA410392EA030FE0
:10D360007FEA226C7FEA236C6AD04FEA1262D2EB2A
:10D370001363C1BFD218414048404140B8BF5B422F
:10D38000192B88BF704710F0004F40F4000020F0C8
:10D390007F4018BF404211F0004F41F4000121F0DE
:10D3A0007F4118BF494292EA030F3FD0A2F1010228
:10D3B00041FA03FC10EB0C00C3F1200301FA03F166
:10D3C00000F0004302D5494260EB4000B0F5000F89
:10D3D00013D3B0F1807F06D340084FEA310102F148
:10D3E0000102FE2A51D2B1F1004F40EBC25008BFFA
:10D3F00020F0010040EA03007047490040EB0000C4
:10D4000010F4000FA2F10102EDD1B0FA80FCACF1F2
:10D41000080CB2EB0C0200FA0CF0AABF00EBC250F1
:10D4200052421843BCBFD0401843704792F0000FDF
:10D4300081F4000106BF80F400000132013BB5E732
:10D440004FEA41037FEA226C18BF7FEA236C21D0A8
:10D4500092EA030F04D092F0000F08BF084670470D
:10D4600090EA010F1CBF0020704712F07F4F04D1DB
:10D47000400028BF40F00040704712F100723CBFEE
:10D4800000F50000704700F0004343F0FE4040F418
:10D49000000070477FEA226216BF08467FEA2363D6
:10D4A0000146420206BF5FEA412390EA010F40F4C1
:10D4B000800070474FF0000304E000BF10F000430D
:10D4C00048BF40425FEA000C08BF704743F09643F4
:10D4D00001464FF000001CE050EA010208BF70470F
:10D4E0004FF000030AE000BF50EA010208BF704796
:10D4F00011F0004302D5404261EB41015FEA010CAB
:10D5000002BF84460146002043F0B64308BFA3F1A2
:10D510008053A3F50003BCFA8CF2083AA3EBC25384
:10D5200010DB01FA02FC634400FA02FCC2F12002A3
:10D53000BCF1004F20FA02F243EB020008BF20F0DA
:10D540000100704702F1200201FA02FCC2F1200240
:10D5500050EA4C0021FA02F243EB020008BF20EA35
:10D56000DC7070474FF0FF0C1CEAD0521EBF1CEA63
:10D57000D15392EA0C0F93EA0C0F6FD01A4480EA51
:10D58000010C400218BF5FEA41211ED04FF000633A
:10D5900043EA501043EA5111A0FB01310CF0004066
:10D5A000B1F5000F3EBF490041EAD3715B0040EA8C
:10D5B000010062F17F02FD2A1DD8B3F1004F40EB5C
:10D5C000C25008BF20F00100704790F0000F0CF02F
:10D5D000004C08BF49024CEA502040EA51207F3AF3
:10D5E000C2BFD2F1FF0340EAC250704740F40000CE
:10D5F0004FF00003013A5DDC12F1190FDCBF00F0BF
:10D6000000407047C2F10002410021FA02F1C2F16C
:10D61000200200FA02FC5FEA310040F1000053EA08
:10D620004C0308BF20EADC70704792F0000F00F056
:10D63000004C02BF400010F4000F013AF9D040EA5C
:10D640000C0093F0000F01F0004C02BF490011F4F0
:10D65000000F013BF9D041EA0C018FE70CEAD153EE
:10D6600092EA0C0F18BF93EA0C0F0AD030F0004C6E
:10D6700018BF31F0004CD8D180EA010000F0004022
:10D68000704790F0000F17BF90F0004F084691F0E0
:10D69000000F91F0004F14D092EA0C0F01D142021A
:10D6A0000FD193EA0C0F03D14B0218BF084608D1E3
:10D6B00080EA010000F0004040F0FE4040F400002D
:10D6C000704740F0FE4040F4400070474FF0FF0CC0
:10D6D0001CEAD0521EBF1CEAD15392EA0C0F93EA07
:10D6E0000C0F69D0A2EB030280EA010C49024FEA59
:10D6F000402037D04FF0805343EA111143EA101312
:10D700000CF000408B4238BF5B0042F17D024FF4C9
:10D71000000C8B4224BF5B1A40EA0C00B3EB510FA4
:10D7200024BFA3EB510340EA5C00B3EB910F24BF8D
:10D73000A3EB910340EA9C00B3EBD10F24BFA3EB12
:10D74000D10340EADC001B0118BF5FEA1C1CE0D1DA
:10D75000FD2A3FF650AF8B4240EBC25008BF20F08D
:10D76000010070470CF0004C4CEA50207F32C2BFE1
:10D77000D2F1FF0340EAC250704740F400004FF07E
:10D780000003013A37E792F0000F00F0004C02BFAF
:10D79000400010F4000F013AF9D040EA0C0093F079
:10D7A000000F01F0004C02BF490011F4000F013BD3
:10D7B000F9D041EA0C0195E70CEAD15392EA0C0F3B
:10D7C00008D142027FF47DAF93EA0C0F7FF470AF73
:10D7D000084676E793EA0C0F04D14B023FF44CAFB6
:10D7E00008466EE730F0004C18BF31F0004CCAD14B
:10D7F00030F000427FF45CAF31F000437FF43CAF87
:10D800005FE700BF4FF0FF3C06E000BF4FF0010CA8
:10D8100002E000BF4FF0010C4DF804CD4FEA40028A
:10D820004FEA41037FEA226C18BF7FEA236C11D0D4
:10D8300001B052EA530C18BF90EA010F58BFB2EB87
:10D84000030088BFC81738BF6FEAE17018BF40F007
:10D85000010070477FEA226C02D15FEA402C05D1BB
:10D860007FEA236CE4D15FEA412CE1D05DF8040B40
:10D87000704700BF844608466146FFE70FB5FFF7D3
:10D88000C9FF002848BF10F1000F0FBD4DF808ED8B
:10D89000FFF7F4FF0CBF012000205DF808FB00BF7C
:10D8A0004DF808EDFFF7EAFF34BF012000205DF8D6
:10D8B00008FB00BF4DF808EDFFF7E0FF94BF012023
:10D8C00000205DF808FB00BF4DF808EDFFF7D2FF20
:10D8D00094BF012000205DF808FB00BF4DF808ED63
:10D8E000FFF7C8FF34BF012000205DF808FB00BF30
:10D8F0004FEA4002B2F1FE4F0FD34FF09E03B3EB5D
:10D9000012620DD94FEA002343F0004310F0004F9C
:10D9100023FA02F018BF404270474FF000007047F2
:10D9200012F1610F01D1420205D110F0004008BF91
:10D930006FF0004070474FF00000704742000ED279
:10D94000B2F1FE4F0BD34FF09E03B3EB126209D43A
:10D950004FEA002343F0004323FA02F070474FF0F0
:10D960000000704712F1610F01D1420202D14FF065
:10D97000FF3070474FF00000704700BF0B46014674
:10D98000184600F001B800BF13460A4601460220BF
:10D9900000F0A8BE014B1868704700BF9096FF1FAB
:10D9A00070B50F4E0F4D761BB61018BF002405D072
:10D9B000013455F8043B9847A642F9D10A4E0B4D65
:10D9C000761B02F0BFFEB61018BF002406D001344B
:10D9D00055F8043B9847A642F9D170BD70BD00BF11
:10D9E00050070100500701006407010050070100C3
:10D9F000024B0146186800F00BB800BF9096FF1F5D
:10DA0000024B0146186800F031BF00BF9096FF1F1F
:10DA10002DE9F04F01F10B05162D83B0064640F2BB
:10DA20009F8035F0070500F1BF80A94200F2BC805D
:10DA300000F058FBB5F5FC7FC0F09C826B0A00F04B
:10DA4000BA80042B00F28381A80900F1390E4FEA55
:10DA50004E033830C44F07EB8303A3F108015C6821
:10DA6000A14207D1ACE0002A80F2AC80E468A14278
:10DA700000F0A680636823F003035A1B0F2AF2DD2F
:10DA8000B9493C6901F1080E744500F0B38163683F
:10DA900023F003035A1B0F2A00F39981002AC1F8CF
:10DAA00014E0C1F810E080F29E80B3F5007F80F0B2
:10DAB0006781DB0803F1010C01229B1002FA03F3DA
:10DAC0004A6851F83C80C4F8088001EBCC091A433D
:10DAD000A9F10803E3604A6041F83C40C8F80C40F3
:10DAE000831001249C40944200F28A80144206D1A3
:10DAF00020F003006400144200F10400FAD007EBA8
:10DB0000C009CC468046DCF80C108C4507D173E187
:10DB1000002A80F28181C9688C4500F06D814B68D4
:10DB200023F003035A1B0F2AF2DD0C46D1F80CC078
:10DB300054F8088F4B1945F001054D6042F0010182
:10DB4000C8F80CC03046CCF808807B613B61C3F854
:10DB50000CE0C3F808E059609A5000F0C5FA1FE0E5
:10DB6000102921D800F0BEFA1025062302207E4F8E
:10DB700007EB8303A3F108025C68944200F045813F
:10DB80006368E168A56823F00303234430465A68BC
:10DB9000E96042F001028D605A6000F0A5FA083495
:10DBA000204603B0BDE8F08F00240C2320463360EC
:10DBB00003B0BDE8F08F80234FF0400E3F2049E7CF
:10DBC00070465DE72344E1685A68A56842F00102A7
:10DBD000E96030468D605A6000F086FA08342046CD
:10DBE00003B0BDE8F08F234430465A6842F001028A
:10DBF0005A6000F079FA0834204603B0BDE8F08F8F
:10DC0000BC68636823F00308A84504D3C5EB080388
:10DC10000F2B00F38C80554BDFF860911A68D9F810
:10DC2000003001332A4404EB080A00F0608102F559
:10DC300080520F3222F47F6222F00F0211463046EA
:10DC4000019200F04BFCB0F1FF3F8346019A00F0D7
:10DC50005881824500F2FC80454B1968DA45114431
:10DC6000196000F05381D9F80000DFF810E10130AD
:10DC70001BBFCAEB0B0A5144CEF800B019601BF071
:10DC8000070100F01781C1F10800C1F580518344FC
:10DC900008315A44C2F30B02C2EB0109494630462F
:10DCA000019300F01BFC431C019B00F03F81CBEB78
:10DCB00000024A4442F001021968C7F808B049441A
:10DCC000BC42CBF804201960DFF8A49016D0B8F15C
:10DCD0000F0F40F2FD806268A8F10C0323F00703E8
:10DCE000E01802F001024FF0050E1A430F2B62609C
:10DCF000C0F804E0C0F808E000F21C811D4BBC68CD
:10DD00001A68914288BF19601B4B1A689142626879
:10DD100088BF196022F003029542A2EB050301D8E7
:10DD20000F2B04DC304600F0DFF9002438E76219DD
:10DD300043F0010345F0010565603046BA60536069
:10DD400000F0D2F90834204603B0BDE8F08F142B60
:10DD500071D9542B00F2A480280B00F16F0E4FEA0A
:10DD60004E036E3076E600BF9496FF1F4CA0FF1F57
:10DD700050A0FF1F48A0FF1F44A0FF1FA09AFF1F35
:10DD80005A0A042A5ED9142A00F2B38002F15C0117
:10DD900049005B3207EB810C57F82110DFF8DC817A
:10DDA000ACF1080C8C4500F088804A6822F0030230
:10DDB000934202D289688C45F7D1D1F80CC07A68B9
:10DDC000C4F80CC0A160CCF80840CC6088E66319A8
:10DDD00042F0010745F00105656030464B610B617B
:10DDE000C3F80CE0C3F808E05F609A50083400F014
:10DDF0007BF9D5E64A6873E608F1010818F0030FCD
:10DE00000CF1080C7FF47FAE30E0DC68A34208BF61
:10DE100002303FF435AEB3E60B440C465A68C9688D
:10DE200054F8085F42F001025A603046E9608D60A4
:10DE300000F05AF9B4E603F15C0E03F15B004FEA1F
:10DE40004E0307E69A0902F1390149003832A1E789
:10DE5000BC424A4B3FF400AF9C68626822F0030268
:10DE60005AE759F80839994540F0828010F0030FBD
:10DE700000F1FF30F5D17B6823EA04037B60640086
:10DE80009C423FF6BDAE002C3FF4BAAE1C42404669
:10DE90007FF435AE64001C4200F10400FAD02EE697
:10DEA000B3F5AA7F18D8E80B00F1780E4FEA4E03BD
:10DEB0007730CFE54FF48051EBE60121D8F80430FC
:10DEC000921001FA02F21A43C8F80420614677E77B
:10DED0000123CBF8043025E740F25452934220D876
:10DEE000A80C00F17D0E4FEA4E037C30B2E51032F3
:10DEF000A4E6542A26D81A0B02F16F0149006E32AB
:10DF000048E7BC68626822F0030205E7CAF30B0029
:10DF100000287FF4A8AE4244BB6842F001025A6078
:10DF2000ECE6FE234FF07F0E7E2093E501224FF0BA
:10DF30000009C1E604F10801304600F097FCD9F869
:10DF40000010DBE6B2F5AA7F05D8DA0B02F1780102
:10DF5000490077321EE740F254518A4205D89A0CA4
:10DF600002F17D0149007C3214E7FE217E2211E797
:10DF70007B6884E7E808431C5B00F8E59496FF1F84
:10DF80008842F0B50DD98B1898420AD28118002A20
:10DF900051D09A1A13F8014D01F8014D9342F9D16D
:10DFA000F0BD0F2A48D941EA00039B0746D100F192
:10DFB000100401F11003154653F8106C44F8106C6E
:10DFC00053F80C6C44F80C6C53F8086C44F8086C6B
:10DFD000103D53F8046C44F8046C0F2D03F110034A
:10DFE00004F11004E8D8A2F1100323F00F0302F0AB
:10DFF0000F0E1033BEF1030F1944034421D91E1F25
:10E000000D467446043C55F8047B46F8047F032C07
:10E01000F8D8AEF1040424F003040434234421446A
:10E0200002F0030262B1013B0A4411F8014B03F80C
:10E03000014F8A42F9D1F0BD0346F3E70346F2E708
:10E04000F0BD7246EEE700BF70B4840746D0541EA0
:10E05000002A41D0CDB2034602E0621EE4B314466A
:10E0600003F8015B9A07F8D1032C2ED9CDB245EA0B
:10E0700005250F2C45EA054519D903F1100226465E
:10E08000103E0F2E42F8105C42F80C5C42F8085C1F
:10E0900042F8045C02F11002F2D8A4F1100222F05E
:10E0A0000F0204F00F041032032C13440DD91E4646
:10E0B0002246043A032A46F8045BFAD8221F22F0CB
:10E0C00003020432134404F003042CB1C9B21C440B
:10E0D00003F8011BA342FBD170BC704714460346F2
:10E0E000C2E700BF704700BF704700BF024B0A463F
:10E0F0000146186800F002B89096FF1F2DE9F04F16
:10E10000174683B0002900F0C1800E46814607F112
:10E110000B05FFF7E7FF56F804EC162D2EF003046D
:10E12000A6F1080840D810221546AF4241D89442C3
:10E1300075DAC94B996808EB04008842416800F021
:10E14000D98021F0010303445B68DB077DD51EF015
:10E15000010F35D039464846FFF75AFC0746E0B173
:10E1600056F8043C23F001034344A0F108029A420C
:10E1700000F04481221F242A00F23181132A00F288
:10E1800004810346324611681960516859609268EB
:10E190009A603146484600F069FB4846FFF7A4FF05
:10E1A000384603B0BDE8F08F25F00705002D2A465C
:10E1B000BBDA0C230020C9F8003003B0BDE8F08FB3
:10E1C00056F8083CC3EB080ADAF8043023F0030CD5
:10E1D00004EB0C039342BDDB5746DAF80C1057F8FA
:10E1E000080F221F242AC160886000F21781132AB9
:10E1F00040F212813168CAF808107168CAF80C1030
:10E200001B2A00F22B8108360AF1100231681160D6
:10E2100071685160B16891603E461C46D046631BF0
:10E220000F2B1DD8D8F8043003F0010323434444D6
:10E23000C8F80430636843F0010363604846FFF7A1
:10E2400053FF304603B0BDE8F08F21F003012144B5
:10E25000914221DBC36882680C46D3609A60DEE796
:10E26000D8F8042008EB050102F00102154343F041
:10E2700001020B44C8F804504A605A6842F0010297
:10E2800008315A60484600F0F1FAD7E7114603B06A
:10E29000BDE8F04FFFF7BCBB1EF0010F7FF45AAF93
:10E2A00056F8083CC3EB080ADAF8043023F0030CF4
:10E2B00001EB0C0E96458BDBC36882685746D36032
:10E2C0009A6057F8081FDAF80C30CB60221F242A16
:10E2D000996000F29980132A62D93368CAF808302D
:10E2E0007368CAF80C301B2A00F2A08008360AF1C5
:10E2F000100356E021F0030BA34405F11000834501
:10E3000059DA1EF0010F7FF425AF56F8081CC1EB57
:10E31000080ADAF8041021F0030CE34458453FF7EB
:10E3200057AF5746DAF80C1057F8080F221F242A67
:10E33000C160886000F2B480132A40F2A580316881
:10E34000CAF808107168CAF80C101B2A00F2AF80D6
:10E3500008360AF110023168116071685160B168C5
:10E3600091600AEB0501C5EB0B0242F001029960D6
:10E370004A60DAF8043003F001031D434846CAF846
:10E380000450FFF7B1FE38465CE7336803607368FA
:10E3900043601B2A27D800F1080306F10802F2E6C1
:10E3A0003B4632681A6072685A60B2689A603E46AC
:10E3B0007446D04633E708EB0501C5EB0B0B4BF079
:10E3C000010299604A6056F8043C03F001031D43C2
:10E3D000484646F8045CFFF787FE304632E7314690
:10E3E000FFF7CEFDD5E6B3688360F368C360242AE7
:10E3F00028D000F1100306F11002C4E650F8043CE6
:10E4000023F003031C440AE7314638467446D046DD
:10E41000FFF7B6FD3E4602E73A46F7E63146384694
:10E420001C46D046FFF7ACFD3E46F8E6B368CAF896
:10E430001030F368CAF81430242A1BD010360AF1C1
:10E440001803AEE7336903617369436106F118028B
:10E4500000F1180397E600BF9496FF1FB168CAF851
:10E460001010F168CAF81410242A0FD010360AF1DF
:10E470001802CBE63369CAF818307369CAF81C3041
:10E4800018360AF120038CE73A4664E73269CAF885
:10E4900018207269CAF81C2018360AF12002B5E665
:10E4A000314638460193FFF76BFD019B59E7B16890
:10E4B000CAF81010F168CAF81410242A03D01036D4
:10E4C0000AF1180247E73269CAF818207269CAF8D7
:10E4D0001C2018360AF120023DE700BF38B5074C72
:10E4E0000023054608462360FBF7E0FE431C00D0EE
:10E4F00038BD2368002BFBD02B6038BDACA1FF1FBB
:10E5000090F800F06DE9024520F007016FF0000C73
:10E5100010F0070491F820F040F049804FF000041B
:10E520006FF00700D1E9002391F840F000F10800F6
:10E5300082FA4CF2A4FA8CF283FA4CF3A2FA8CF32E
:10E540004BBBD1E9022382FA4CF200F10800A4FA95
:10E550008CF283FA4CF3A2FA8CF3E3B9D1E90423E9
:10E5600082FA4CF200F10800A4FA8CF283FA4CF320
:10E57000A2FA8CF37BB9D1E9062301F1200182FADA
:10E580004CF200F10800A4FA8CF283FA4CF3A2FAE0
:10E590008CF3002BC6D0002A04BF04301A4612BAEE
:10E5A000B2FA82F2FDE8024500EBD2007047D1E9F1
:10E5B000002304F00305C4F100004FEAC50514F080
:10E5C000040F91F840F00CFA05F562EA05021CBF51
:10E5D00063EA050362464FF00004A9E7002A41D030
:10E5E00040EA010313F00303F0B425D1032A23D931
:10E5F00004680D68AC421FD1043A35D0A4F101354E
:10E6000025EA040414F0803F31D1071D0D1D0DE0F3
:10E6100057F8043B0E68A3F10134B34224EA030423
:10E620000AD1043A20D014F0803F23D1032A29468E
:10E63000384605F10405EBD803780C789C4202F1CA
:10E64000FF320CD182B114B916E06AB17BB110F877
:10E65000013F11F8014FA34202F1FF32F5D0181B20
:10E66000F0BC7047104670471046F0BC7047184623
:10E67000F0BC70470020F3E72046F1E740EA0103D1
:10E680009B0770B42BD1032A29D90C460346214697
:10E6900054F8046BA6F1013525EA060515F0803F14
:10E6A00006D1043A032A43F8046B2146EFD8A2B1FD
:10E6B0000C781C70013A013301313CB16AB111F898
:10E6C000014B03F8014B013A002CF7D12AB11A444F
:10E6D000002103F8011B9A42FBD170BC704703462E
:10E6E000E5E700BF2DE9F047254C2568D5F84841FE
:10E6F0000646884692469946C4B360681F2817DCD0
:10E70000431C76B104EB80050122C5F888A0D4F83B
:10E71000881182401143022EC4F88811C5F808916F
:10E720001ED00230636044F820800020BDE8F087EE
:10E73000144B03B34FF4C870FFF75AF90446D0B135
:10E74000D5F84831002780E88800C5F848413846A8
:10E750000123C4F88871C4F88C71002EE1D0D1E790
:10E76000D4F88C110A43C4F88C21DAE705F5A674B5
:10E77000C5F84841C1E74FF0FF30BDE8F08700BF62
:10E7800040070100F1D90000024B13B1024800F02C
:10E7900005B8704700000000A9E70000002301460B
:10E7A0001A461846FFF79EBF38B5074D074C2C1B7D
:10E7B000A41005D0013C55F8043D9847002CF9D130
:10E7C000BDE8384001F0CEBF0000000000000000AE
:10E7D000F8B5234F0C460646FFF784FCBB685D681E
:10E7E00025F00305291B01F6EF7121F47F6121F06B
:10E7F0000F01A1F58054B4F5805F07DB002130469E
:10E80000FFF76CFEBB682B44984204D03046FFF7FC
:10E810006BFC0020F8BD61423046FFF75FFE01301F
:10E820000DD0104BBA6819682D1B45F00105304614
:10E83000091B55601960FFF757FC0120F8BD002146
:10E840003046FFF74BFEBA68831A0F2BDEDD064C0D
:10E850000449246843F00103001B53600860D5E7B6
:10E860009496FF1F50A0FF1FA09AFF1F002945D0BC
:10E870002DE9F0410D468046FFF734FC55F8047C45
:10E880006A4927F00103A5F10804E2188E68506870
:10E89000B24220F0030062D0FE0750600BD455F85E
:10E8A000087CE41B01F1080EA56875453B446FD058
:10E8B000E768EF60BD6015186D68ED0742D543F05D
:10E8C00001026260E350B3F5007F18D2DB085A1CE6
:10E8D0004D6851F83270A76001209B1000FA03F3D5
:10E8E00001EBC2001D430838E0604D6041F8324042
:10E8F000FC604046BDE8F041FFF7F6BB70475A0A9E
:10E90000042A53D89A0902F139077F0002F1380529
:10E9100001EB870051F827204449083890424DD038
:10E92000516821F003018B4202D292689042F7D1E4
:10E93000D068E060A2608460D4604046BDE8F041E9
:10E94000FFF7D2BB95683A4FBD4203443FD0D06831
:10E95000E86043F0010285606260E350B3E7FF07BF
:10E96000034407D455F8082CA41A1344A068E2689D
:10E97000C26090602F4A126843F0010093426060C9
:10E980008C60B6D32C4B40461968FFF721FFB0E7E7
:10E9900011184968C90744D49168D268CA60034411
:10E9A00043F0010091606060E350A2E7142A17D899
:10E9B00002F15C077F0002F15B05A9E7AA104B6832
:10E9C000012505FA02F213434B600246B1E743F01A
:10E9D00001024C610C61E560A5606260E35088E76C
:10E9E000542A06D81A0B02F16F077F0002F16E0558
:10E9F0008EE7B2F5AA7F06D8DA0B02F178077F001E
:10EA000002F1770584E740F25450824206D89A0C0E
:10EA100002F17D077F0002F17C0579E7FE277E2564
:10EA200076E743F001026260E35062E79496FF1FCD
:10EA30009C96FF1F9C9AFF1F4CA0FF1F00007805AB
:10EA40003408540B800C3C0F5C12E015FA19141EAC
:10EA50006022AC265C2B0C30BC34023AFF3FFFFF37
:10EA600084ED000060ED00003CED000018ED0000BA
:10EA700048EB000094EA0000B8EA0000DCEA00007D
:10EA800000EB00004CEC000070EC00003CEA0000E1
:10EA900028EC00000000580246056608540BD80E0A
:10EAA0005C12E015FA19141E6022AC265C2B0C30A7
:10EAB000BC34023AFF3FFFFF000090012003140521
:10EAC000D0075A0AAC0DCC10B4146A18E81C3421D3
:10EAD00080252A2B70301437FF3FFFFF0000C8004D
:10EAE000F4018403140508072E091C0CD80EF81134
:10EAF000AE159619401F1C25F22B5834FF3FFFFF1F
:10EB000000006400C8009001BC021A04DC059E07E6
:10EB1000F609800CA00F2413A2174C1D5424442F77
:10EB2000FF3FFFFF40067805B004E803840320039D
:10EB3000BC025802F40190012C01FA00C8009600B2
:10EB4000640032001900FFFF0000FF03FF07FF0B06
:10EB5000FF0FFF13FF17FF1BFF1FFF23FF27FF2BD5
:10EB6000FF2FFF33FF37FF3BFF3FFFFF0102010194
:10EB70000201010102010101020101000101010282
:10EB80000001010201010101010102000101020174
:10EB90000102010101020100010201010201010162
:10EBA0000000000102010102010101010000010257
:10EBB0000101020101000202020102010102010041
:10EBC000020202020102010102000102020202012C
:10EBD0000201010000000202020201020101010023
:10EBE000000202020201020100020202020202020B
:10EBF00001020002020102020202020101000202FD
:10EC000002020202020201000002020002020202EB
:10EC100002000201020202020202020200020002DB
:10EC200002020202020202FF0000D007800CD80E8E
:10EC30000010C012EC130C17FA19141E6022AC2637
:10EC40005C2B0C30BC34023AFF3FFFFF000058023F
:10EC500046056608540BD80E5C127017FC21F82A82
:10EC600070305834DC37663A8C3C803EFF3FFFFF03
:10EC70000000580246056608540BA00FD41728233D
:10EC8000F82A442F643284354038663A8C3C803E02
:10EC9000FF3FFFFFF2FFFFFFF3FFFFFFF4FFFFFF68
:10ECA000F4FFFFFFF5FFFFFFF6FFFFFFF7FFFFFF9A
:10ECB000F8FFFFFFF9FFFFFFFAFFFFFFFBFFFFFF7A
:10ECC000FCFFFFFFFDFFFFFFFDFFFFFFFEFFFFFF5C
:10ECD000FFFFFFFF000000002C011301FA00E1001C
:10ECE000C800AF0096007D0064004B0032001900A0
:10ECF00000000000CDCC4C3DCDCCCC3D9A99193EC6
:10ED0000CDCC4C3E0000803E9A99993E3333B33EC1
:10ED1000CDCCCC3E6666E63E00007805220B0410A2
:10ED2000B4143219B01DFC214826FE29822D383139
:10ED300026344637663A223DFF3FFFFF0000D007EA
:10ED4000100E88133219AA1E282374275C2B442F17
:10ED5000643284354038663A8C3C803EFF3FFFFF8A
:10ED60000000540BEC13FA1908201C253629EC2C52
:10ED70000C302C33E8357238663AF63B863D163F48
:10ED8000FF3FFFFF0000CC10581BFC21AC26C62A19
:10ED90007C2E3831F4334C36A438983A5A3C543DE2
:10EDA000803E7A3FFF3FFFFF18EE0000829BFF1F6F
:10EDB0000000FF0F4C9CFF1F0000FF0F153A0000E2
:10EDC000E4ED0000489CFF1F32005E0100000000DF
:10EDD00000000000B539000054485200534E530063
:10EDE0004D415800544F5543482053454E5345001C
:10EDF000455854524120434F4E54524F4C4C45526B
:10EE00000000000050495443482042454E44000051
:10EE1000424954450000000042524541544800FF19
:10EE2000F0ED0000E09AFF1FF401A00FAA9BFF1F66
:10EE3000F401A00FC139000010EE00003A9BFF1F43
:10EE4000BC025C12249CFF1FBC025C12F93900005A
:10EE500004EE0000FE9BFF1FF401A00F089BFF1FA4
:10EE6000F401A00FDD39000008F6000010F60000E4
:10EE70000CF50000CCF50000E8F50000ECF5000012
:10EE8000F0F50000F4F50000F8F50000FCF50000D6
:10EE900000F60000D4F5000004F600000CF50000B8
:10EEA00008F50000DCF50000E0F50000E4F50000E6
:10EEB0000CF50000CCF50000D0F50000D4F5000002
:10EEC000D8F50000BCF50000C0F50000C4F5000056
:10EED00028FA0000C8F5000018F600001CF6000033
:10EEE00020F6000024F6000028F600002CF60000B2
:10EEF00030F6000034F6000038F600003CF6000062
:10EF000040F6000044F6000048F600000100000052
:10EF1000A0F7000006000000B0F6000000000201AB
:10EF20000A000000488BFF1F00000000A0F800004E
:10EF300070F80000029BFF1F00003000000000007E
:10EF40001D530000DD430000000000000100000030
:10EF5000C0F7000003000000010000004CF60000B4
:10EF60000700000000000000A8F6000074F6000092
:10EF7000F09AFF1F0000090000000000614A000035
:10EF80000D44000000000000000000007CF80000BC
:10EF900070F80000109CFF1F00003000000000000F
:10EFA0002D53000089450000000000000100000012
:10EFB000A8F70000050000000100000090F7000025
:10EFC00008000000000000004CF700004CF70000B3
:10EFD000F49AFF1F00000C0003000000ED56000033
:10EFE000FD430000000000000000000064F8000085
:10EFF00070F80000129CFF1F0000300000000000AD
:10F000002D530000894500000000000000000000B2
:10F01000010000003D47000001000000B4F70000BF
:10F020000400000000000000C8F70000D0F7000056
:10F03000B49BFF1F01001000060000008159000072
:10F04000ED4300009D4D00002C0100007D460000B6
:10F050000600000009000000C48DFF1F3CF80000FE
:10F060000000030106000000208CFF1F00000000CC
:10F0700001000000215C000098F70000000005017D
:10F0800007000000BC8BFF1F0100000098F7000084
:10F090000900000024F70000000001010800000042
:10F0A000788EFF1F0000000094F8000070F8000048
:10F0B0000C9CFF1F00003000000000002D530000DA
:10F0C00089450000000000004CF600000000040527
:10F0D00008000000A48DFF1F000000004CF8000095
:10F0E00058F800001C9BFF1F0000010001000000F9
:10F0F0003D4A0000CD430000000000000000000079
:10F1000001000000D14F00000000000000000000DE
:10F1100000000000000000000000000000000000EF
:10F1200000000000000000000000000000000000DF
:10F1300000000000000000000000000000000000CF
:10F1400000000000000000000000000000000000BF
:10F1500000000000000000000000000000000000AF
:10F16000000000000000000000000000000000009F
:10F17000000000000000000000000000000000008F
:10F18000000000000000000000000000000000007F
:10F19000000000000000000000000000000000006F
:10F1A000000000000000000000000000000000005F
:10F1B000000000000000000000000000000000004F
:10F1C000000000000000000000000000000000003F
:10F1D000000000000000000000000000000000002F
:10F1E000000000000000000000000000000000001F
:10F1F000000000000000000000000000000000000F
:10F2000000000000000000000000000000000000FE
:10F2100000000000000000000000000000000000EE
:10F22000000000000000000000000000007FFFFF61
:10F23000000003F9FFFFFC0000000000007FFFFF5B
:10F24000800007F9FFFFFE000000000000600001E1
:10F25000C0000E198000070000000000006FFFFCD6
:10F26000C0001DD9BFFFF30000000000006FFFFECB
:10F27000C0003BD9BFFFFB0000000000006C00068F
:10F28000C00077D9B0001B0000000000006C000631
:10F29000C000EED9B0001B0000000000006C0006AA
:10F2A000C001DCD9B0001B0000000800006C0006A3
:10F2B000C003B8D9B0001B0000001800006FFFFEAB
:10F2C000C0077FD9B0001B0000001800006FFFFCD2
:10F2D000C00EFFD9B0001B0000C018000060000184
:10F2E000C01C0019B0001B0000C03800006FFBFFFD
:10F2F000803BFFD9B0001B0000C03000006FFDFF55
:10F300000077FFD9B0001B0001E03000006C0EE078
:10F3100000EE00D9B0001B0001E03000006C077067
:10F3200001DC00D9B0001B0001B03000006C03B854
:10F3300003B800D9B0001B0001B03000006C01DC44
:10F34000077000D9B0001B00019820C0406C00EE8F
:10F350000EE000D9B0001B00030C20C0C06C007789
:10F360001DC000D9BFFFFB00030C20C0C06C003BD8
:10F37000BB8000D9BFFFF300030620C1C06C001D95
:10F38000F70000D98000070003032083806C000E83
:10F39000EE0000D9FFFFFE000303B183806C00077D
:10F3A0005C0000D9FFFFFC000301F1878000000032
:10F3B00000000000000000000300F18D800000004C
:10F3C0000000000000000000030071B98000000090
:10F3D0000000000000000000030031F18000000088
:10F3E0000000000000000000030000C180000000D9
:10F3F000000000000000000003000000000000000A
:10F4000000000000000000000300000000000000F9
:10F4100000000000000000000200000000000000EA
:10F4200000000000000000000000000000000000DC
:10F4300000000000000000000000000000000000CC
:10F4400000000000000000000000000000000000BC
:10F4500000000000000000000000000000000000AC
:10F46000000000000000000000000000000000009C
:10F47000000000000000000000000000000000008C
:10F48000000000000000000000000000000000007C
:10F49000000000000000000000000000000000006C
:10F4A000000000000000000000000000000000005C
:10F4B000000000000000000000000000000000004C
:10F4C000000000000000000000000000000000003C
:10F4D000000000000000000000000000000000002C
:10F4E000000000000000000000000000000000001C
:10F4F000000000000000000000000000000000000C
:10F5000000000000000000004F4E00004F46460083
:10F51000424154004C4F5720000000005553420018
:10F520004D454E552020202020202020205858587E
:10F5300020592E595600000058000000524F540028
:10F540004D454C0044594E006D7300004254480034
:10F55000424954004C5652004E524D0052455600FE
:10F56000312F0000415400004D4F440050424400F0
:10F5700045433200454353004C564C004C56500016
:10F58000474C4400762E0000312E342E350000000A
:10F590004E755241440000006669726D7761726574
:10F5A00020762E0053455400434C5200444F4E27C2
:10F5B0005400000050414E494300000045574900A7
:10F5C0004557580053415800455652004D570000CA
:10F5D00046500000434600005350000053570000BF
:10F5E00053454C005345450042520000564C000024
:10F5F000455800004D572B0042522B00564C2B0013
:10F6000045582B00554E4F00425254480000000010
:10F6100050544348000000002D3400002D330000FA
:10F620002D3200002D3100004C494E002B310000DE
:10F630002B3200002B3300002B340000533100002C
:10F64000533200005A3100005A32000056494252EB
:10F6500041544F00444952454354494F4E00000025
:10F66000434F4E54524F4C00535155454C43482044
:10F67000420000004C4556454C00000053454E5397
:10F680004520425445000000535155454C43482005
:10F690004C00000053454E5345204C56520000008C
:10F6A00052455455524E0000444550544800000005
:10F6B0005345545550204354524C530045585452CE
:10F6C0004120504B4559000046494E474552494E4E
:10F6D000470000004C4556454C20434300000000C5
:10F6E0004D4F44204B4559004445474C49544348ED
:10F6F00000000000455843545220434332000000AC
:10F70000455854524120435452000000504954433C
:10F710004842454E44000000504F52542F474C443D
:10F720000000000053455455502042524541544872
:10F730000000000056454C20424F4F53540000003B
:10F7400056454C2044454C41590000004355525603
:10F750004500000056454C4F4349545900000000F5
:10F760004252454154482041540000004343322056
:10F77000524953450000000042525448204343324E
:10F780000000000042525448204343310000000072
:10F7900041424F5554000000455854524153000017
:10F7A000524F5441544F52005345545550204354E6
:10F7B0004C000000534554555020425200000000B8
:10F7C00041444A55535400004D49444920434800A0
:10F7D0004D4944492043484E4C000000574C2043BB
:10F7E00048414E00574C20504F57455200000000F2
:10F7F0004641535420424F4F54000000444143209F
:10F800004F55540053504543204B455900000000CC
:10F810004C45474143592042520000004C45474166
:10F8200043592050420000004F43544156450000C8
:10F830005452414E53504F5345000000524F5441D3
:10F84000544F522053455455500000005052494FD8
:10F8500052495459000000004D4F4E4F205052491C
:10F860004F000000524F5441544520340000000026
:10F8700053454D49544F4E4553000000524F54419B
:10F880005445203300000000524F5441544520326B
:10F8900000000000524F5441544520310000000048
:10F8A000504152414C4C454C00FFFFFF000000000E
:10F8B00088F8000070F800000E9CFF1F0000300068
:10F8C000000000002D5300008945000000000000EA
:10F8D0000021110202000000002111020504FFFFB7
:10F8E000003E7FFF4E7545564963303100000000F1
:10F8F0007676764E75455649636363007676764E26
:10F9000075455649633034656576767676767676D3
:10F9100076000000496E76616C696420636F6E66E4
:10F92000696720666F726D6174000000496E7661D0
:10F930006C696420636865636B73756D000000001B
:10F94000496E76616C696420636F6E6669672073C7
:10F95000697A6500496E76616C696420636F6E66D2
:10F9600069672076657273696F6E00004E75455643
:10F9700049000000496E76616C6964206D6573739F
:10F980006167652E00000000653030006330300094
:10F9900053656E64696E6720636F6E6669672E2EAD
:10F9A0002E000000436F6E6669672073656E742ECB
:10F9B000000000006330330053656E64696E672099
:10F9C00076657273696F6E2E00000000633032003E
:10F9D000526563656976696E6720636F6E666967F5
:10F9E0002E2E2E004E657720636F6E66696720733A
:10F9F000617665642E000000556E6B6E6F776E2029
:10FA00006D6573736167652E00000000653031001D
:10FA1000436F6E666967206D676D7400506F776520
:10FA200072206F6666204E7545564900746F2065DA
:10FA30007869740052656164792E00FF3480044057
:10FA4000400000001211FFFFFF020200000013102F
:10FA5000FFFFFF0202000000180000003480044095
:10FA6000800000001EFFFFFFFF02000000001DFFDE
:10FA7000FFFFFF020000000019000000000000006E
:10FA800000000000A17700006577000019770000F2
:10FA9000617700001D77000029770000497700009A
:10FAA000000103070F1F3F7F2200FF2100FFFFFF20
:10FAB0000080C0E0F0F8FCFE000000000000000044
:10FAC000F9960000559B0000197700002581000081
:10FAD000BD810000A18F0000558F0000898F0000BC
:10FAE000618F0000758F0000718E0000A18F0000F3
:10FAF000C98F0000B9830000018C00009D8B0000BD
:10FB000099900000A58F0000FD9000009D910000DD
:10FB1000DA02818FDA1281FF00006000000000002D
:10FB2000000000000000000000E0000000000000F5
:10FB30000000000000000001E000000000000000E4
:10FB400000000000000001F00000000000000000C4
:10FB5000000000000003F0000000000000000000B2
:10FB60000000000007F0000000000000000000009E
:10FB700000000007F8000000000000000000000086
:10FB800000000FF800000003C0007E000001E0004C
:10FB90007F0FF800000003C000FE000001E000FF3E
:10FBA000EFF800000003C000FE000001E000FFFFCE
:10FBB000F800000003C000F00000000F007FFE7F8F
:10FBC000C0000003C000F00000000F003FFE7FF8FF
:10FBD0003FF1FBCFFCFEF3BC3DEFE01FFE7FFF7F5C
:10FBE000FBFFDFFEFEFFBC3DEFE01FC6FFFF7FFB1C
:10FBF000FFDFFEFEFFBC3DEFE00FE3C7FE787BC3F7
:10FC0000DE1EF0FFBC3DEF0007FF87FC787BC3DE04
:10FC10001EF0F83C3DEF0001FFFFF0007BC3C01E6B
:10FC2000F0F03C3DEF0001F37FE03FFBC3CFFEF07F
:10FC3000F03C3DEF0003E33F807FFBC3DFFEF0F0CD
:10FC40003C3DEF0007E73C00787BC3DE1EF0F03C54
:10FC50003DEF0007FFBE00787BC3DE1EF0F03C3DA9
:10FC6000EF0007FFFE00787BC3DE1EF0F03C3DEFA7
:10FC7000000FFFFE007FFBFFDFFEF0F03FFDEFE037
:10FC80000FFFFF007FFBFFDFFEF0F03FFDEFE00F17
:10FC9000F9FF003E79F9CF9EF0F01F3DE7E01FF13C
:10FCA000FF0000000000000000000000001F80FFB7
:10FCB000007FFFFFFFFFFFFFFFFFFFE01C007F0053
:10FCC0007FFFFFFFFEB46D888D18E000001F007FEE
:10FCD000FFFFFFFE95AD7DB577E000000F007FFFD1
:10FCE000FFFFFEA5AD9D8D19E0000006007FFFFF20
:10FCF000FFFEB5ADEDB57EE0AED580A8D300408D5A
:10FD00002000A1C8DB40A4A62EAFFFFF000000002A
:10FD100000018000000000000000000003800000DF
:10FD20000000000000000007C0000000000000000C
:10FD3000000007C00000000000000000000FC0002D
:10FD400000000000000000001FE0000000000000B4
:10FD50000000001FE00000000000000000003FE085
:10FD60000000000000000000003FF0000000000064
:10FD7000000000007FF0000000000000001FF87F7E
:10FD8000F0000000000000003FFE7FF000000000D7
:10FD90000000003FFF7FF0000000000000001FFF98
:10FDA000FBE0000000000000000FFFF9FFC00000B2
:10FDB000000000000FFFF9FFF8000000000000073E
:10FDC000FFF1FFFF00000000000003FC73FFFF8055
:10FDD000000000000001FE3FFFFF80000000000067
:10FDE00000FF1E0FFF000000000000007FFE1FFC50
:10FDF000000000000000003FFFFFF80000000000CE
:10FE000000000FDFFFE0000000000000001F19FFEE
:10FE1000C0000000000000003F3CFF0000000000A8
:10FE20000000007E7CF800000000000000007FFE63
:10FE30007C0000000000000000FFFFFC000000004C
:10FE400000000000FFFFFE0000000000000000FFB7
:10FE5000FFFE0000000000000001FFEFFE000000B8
:10FE60000000000001FFCFFE0000000000000003C2
:10FE7000FF07FE0000000000000003FC07FE00007A
:10FE8000000000000003F003FE000000000000007E
:10FE9000018000FE000000000000000000007E0065
:10FEA0000000000000000000003E00000000000014
:10FEB000000000000C000000000000078000FC00B3
:10FEC0000003C0000000078001FC000003C0000028
:10FED00000078001FC000003C0000000078001E073
:10FEE0000000001E000000078001E00000001E006E
:10FEF0007FE3F79FF9FDE7787BDFC0FFF7FFBFFDEA
:10FF0000FDFF787BDFC0FFF7FFBFFDFDFF787BDFE4
:10FF1000C0F0F787BC3DE1FF787BDE00F0F787BCDF
:10FF20003DE1F0787BDE0000F787803DE1E0787B03
:10FF3000DE007FF7879FFDE1E0787BDE00FFF7873B
:10FF4000BFFDE1E0787BDE00F0F787BC3DE1E078C3
:10FF50007BDE00F0F787BC3DE1E0787BDE00F0F768
:10FF600087BC3DE1E0787BDE00FFF7FFBFFDE1E00D
:10FF70007FFBDFC0FFF7FFBFFDE1E07FFBDFC07C61
:10FF8000F3F39F3DE1E03E7BCFC0000000000000A6
:10FF90000000000000FFFFFFFFFFFFFFFFFFFFC0AB
:10FFA000FFFFFFFFFD68DB111A31C0FFFFFFFFFD00
:10FFB0002B5AFB6AEFC0FFFFFFFFFD4B5B3B1A3381
:10FFC000C0FFFFFFFFFD6B5BDB6AFDC0DA0281FF54
:10FFD0000000000000000000F9960000559B0000A2
:10FFE0001977000025810000D9A20000A18F000030
:10FFF000558F0000898F0000618F0000758F000011
:020000021000EC
:10000000718E0000A18F0000C98F0000C58F000015
:10001000ED8F00004590000099900000A58F000032
:10002000FD9000009D91000000000000003E5B4F2D
:100030005B3E3E6B4F6B3E1C3E7C3E1C183C7E3C48
:10004000181C577D571C1C5E7F5E1C00183C180056
:10005000FFE7C3E7FF0018241800FFE7DBE7FF30E6
:10006000483A060E2629792926407F050507407F54
:1000700005253F5A3CE73C5A7F3E1C1C08081C1CC7
:100080003E7F14227F22145F5F005F5F06097F01BD
:100090007F006689956A606060606094A2FFA294A8
:1000A00008047E040810207E201008082A1C080876
:1000B0001C2A08081E101010100C1E0C1E0C3038C4
:1000C0003E3830060E3E0E06000000000000005FC5
:1000D00000000007000700147F147F14242A7F2AE1
:1000E00012231308646236495620500008070300A3
:1000F000001C2241000041221C002A1C7F1C2A08EF
:10010000083E080800807030000808080808000051
:1001100060600020100804023E5149453E00427FC5
:10012000400072494949462141494D331814127F14
:100130001027454545393C4A4949314121110907B4
:100140003649494936464949291E00001400000035
:100150004034000000081422411414141414004107
:1001600022140802015909063E415D594E7C1211C4
:10017000127C7F494949363E414141227F414141FC
:100180003E7F494949417F090909013E4141517377
:100190007F0808087F00417F41002040413F017FE8
:1001A000081422417F404040407F021C027F7F04B0
:1001B00008107F3E4141413E7F090909063E4151F9
:1001C000215E7F09192946264949493203017F01E9
:1001D000033F4040403F1F2040201F3F4038403FEA
:1001E000631408146303047804036159494D430000
:1001F0007F4141410204081020004141417F040237
:1002000001020440404040400003070800205454CD
:1002100078407F28444438384444442838444428AB
:100220007F385454541800087E090218A4A49C78FE
:100230007F0804047800447D40002040403D007F5A
:100240001028440000417F40007C047804787C083A
:100250000404783844444438FC182424181824240E
:1002600018FC7C08040408485454542404043F44F3
:10027000243C4040207C1C2040201C3C4030403C22
:1002800044281028444C9090907C4464544C440082
:1002900008364100000077000000413608000201E6
:1002A0000204023C2623263C1EA1A161123A4040D2
:1002B000207A38545455592155557941225454784F
:1002C00042215554784020545579400C1E527212E8
:1002D0003955555559395454545939555454580071
:1002E00000457C410002457D420001457C407D1275
:1002F00011127DF0282528F07C54554500205454D7
:100300007C547C0A097F4932494949323A44444481
:100310003A324A4848303A4141217A3A42402078BC
:10032000009DA0A07D3D4242423D3D4040403D3CBD
:1003300024FF2424487E4943662B2FFC2F2BFF09E2
:1003400029F620C0887E09032054547941000044D6
:100350007D413048484A32384040227A007A0A0AC1
:10036000727D0D19317D2629292F28262929292634
:1003700030484D4020380808080808080808382F79
:1003800010C8ACBA2F102834FA00007B0000081403
:100390002A142222142A14085500550055AA55AAD9
:1003A00055AAFF55FF55FF000000FF00101010FF79
:1003B00000141414FF001010FF00FF1010F010F0D4
:1003C000141414FC001414F700FF0000FF00FF14C5
:1003D00014F404FC141417101F10101F101F141411
:1003E000141F00101010F0000000001F101010105B
:1003F0001F10101010F010000000FF10101010104F
:1004000010101010FF10000000FF140000FF00FF8C
:1004100000001F10170000FC04F414141710171428
:1004200014F404F40000FF00F7141414141414144A
:10043000F700F7141414171410101F101F141414BD
:10044000F4141010F010F000001F101F0000001F27
:1004500014000000FC140000F010F01010FF10FF5A
:10046000141414FF141010101F00000000F010FFEF
:10047000FFFFFFFFF0F0F0F0F0FFFFFF00000000D3
:1004800000FFFF0F0F0F0F0F3844443844FC4A4A57
:100490004A347E02020606027E027E02635549410C
:1004A000633844443C04407E201E2006027E020243
:1004B00099A5E7A5991C2A492A1C4C7201724C3057
:1004C0004A4D4D303048784830BC625A463D3E492E
:1004D0004949007E0101017E2A2A2A2A2A44445FD2
:1004E000444440514A444040444A51400000FF01C6
:1004F00003E080FF000008086B6B083612362436D4
:10050000060F090F06000018180000001010003038
:1005100040FF0101001F01011E00191D1712003CC0
:100520003C3C3C00000000000D0AFFFF050E0809DE
:100530000D0C06070F0400130393050E08090D0C9C
:1005400006070F04FFFFC585848687C4FFFF0013DD
:1005500003931A9217FFFFFF6FF07F030370037876
:1005600013F0800FFBD070474008FE4340A00440CA
:100570004408FE4344A004400018FE4300C0044069
:100580003000FE43309004403400FE433490044079
:100590001C18FE431CC004401018FE4310C0044049
:1005A0000818FE4308C004400C18FE430CC0044069
:1005B0000C10FE430CB004401010FE4310B0044079
:1005C0001810FE4318B004401C10FE431CB0044039
:1005D0001410FE4314B004400418FE4304C0044049
:1005E0000010FE4300B004400008FE4300A0044099
:1005F0000408FE4304A004400C08FE430CA0044081
:100600000808FE4308A004401418FE4314C0044028
:100610001818FE4318C004400410FE4304B0044000
:100620000810FE4308B004401400FE431490044038
:100630004C08FE434CA004400420FE4304D0044078
:100640002410FE4324B004402010FE4320B0044098
:100650002810FE4328B004402C10FE432CB0044068
:100660000020FE4300D004404808FE4348A0044058
:100670001000FE4310900440090AFFFFFFFFFFFF38
:10068000FFFFFFFFFFFFFF0D00060807FFFF0E0F34
:10069000FF0CFFFFFFFFFFFF0B05FFFF15191519EB
:1006A000000100008491FF1F120000000002000002
:1006B000B091FF1F73000000002201002492FF1F71
:1006C00021000000002101000C92FF1F0900000022
:1006D000000300004892FF1F00000000010309040E
:1006E0009891FF1F0000000002030904948FFF1F70
:1006F00000000000030309044C92FF1F00000000EB
:10070000000000000000000000000000657870009C
:10071000000000000000E03F000000000000E0BF1B
:10072000763C7935EF39EA3D763C7935EF39EABDEB
:100730000000E0FE422EE63F0000E0FE422EE6BF53
:100740006892FF1FF8B500BFF8BC08BC9E46704712
:1007500089E700003504000059390000D553000036
:04076000957300008D
:04076400F8B500BF25
:1007680038B5084B1C681C6054B1074D94FAA4F3C3
:10077800B3FA83F355F823309847631E1C40F5D12C
:1007880038BD00BFA0D004407491FF1F38B5084B96
:100798001C681C6054B1074D94FAA4F3B3FA83F3B0
:1007A80055F823309847631E1C40F5D138BD00BF6B
:1007B800A0C004405491FF1F38B5084B1C681C604A
:1007C80054B1074D94FAA4F3B3FA83F355F82330E0
:1007D8009847631E1C40F5D138BD00BFA0B0044047
:1007E8002491FF1F38B5084B1C681C6054B1074D95
:1007F80094FAA4F3B3FA83F355F823309847631EA9
:100808001C40F5D138BD00BFA0A00440D490FF1F04
:1008180038B5084B1C681C6054B1074D94FAA4F312
:10082800B3FA83F355F823309847631E1C40F5D17B
:1008380038BD00BFA09004409C90FF1F000000003E
:10084800002000000000F041280000000C0000001B
:100858005A000000F3FFFFFFDFFFFFFFA3FFFFFFCA
:10086800AEFFFFFF730000007600000002000000EA
:1008780004000000D8FFFFFFB5FFFFFFA2FFFFFF46
:1008880002000000FBFFFFFF000000000000000066
:100898000000000000000000000000000000000050
:1008A800000000000000000001000000002000001F
:1008B8000020000000100000AB0A00000008000043
:1008C80066060000550500009204000000040000C0
:1008D8008E03000033030000E8020000AB020000B2
:1008E8000020000014050000000102070B010207A8
:1008F8000B4A140002000C0024000000A8FFFFFFB0
:10090800BCFFFFFFE1FFFFFF0D0000000400000037
:100918007800000079000000BCFFFFFFABFFFFFF7D
:10092800DEFFFFFF17000000570000001000000066
:100938000A00000008000000150000001800000070
:10094800290000000200FFFFFFFF0000A8ED0000E3
:1009580038EE000050EE000020EE0000C0ED000070
:1009680000000000C8F60000C8F60000CC9AFF1F7F
:10097800000004000100000000000000000000006A
:10098800000000000000000088F6000074F6000077
:10099800D689FF1F01001E000000000000000000B3
:1009A800000000000000000000000000E4F7000064
:1009B800E4F700001C9DFF1F00000300000000007A
:1009C800000000000000000000000000000000001F
:1009D80094F6000074F60000D489FF1F01000C0093
:1009E80000000000000000000000000000000000FF
:1009F80000000000010000000000000000000000EE
:100A080060F7000060F700007A9BFF1F00000100FC
:100A180001000000000000000000000000000000CD
:100A28000000000034F7000034F70000D09AFF1FE0
:100A380000000900010000000000000000000000A4
:100A48000000000000000000A0F6000074F600009E
:100A58006089FF1F00000400000000000000000083
:100A68000000000000000000BC8EFF1F5C8DFF1F0F
:100A7800E08EFF1F58EF0000A48CFF1F548EFF1F4D
:100A8800048FFF1FFC8BFF1F408AFF1F708BFF1F07
:100A9800000000000CF700000CF70000269BFF1F69
:100AA80000000C0000000000000000000000000032
:100AB800000000000000000028F8000028F80000EE
:100AC800089CFF1F00000600000000000000000056
:100AD800000000000000000001000000D88BFF1F8C
:100AE800808DFF1FC88CFF1F988EFF1F288FFF1F48
:100AF800888AFF1F148DFF1F000000001CF80000EB
:100B08001CF80000389BFF1F0000010001000000D6
:100B180000000000000000000000000000000000CD
:100B2800BCF60000BCF60000749CFF1F0000190012
:100B380000000000000000000000000000000000AD
:100B480028EF0000A4F00000ACF8000088EF0000D7
:100B5800E8EF0000D8F000000000000078F700007F
:100B680078F700002A9CFF1F00007F0001000000AA
:100B7800000000000000000000000000000000006D
:100B880040F7000040F70000749BFF1F00001E00A4
:100B9800010000000000000000000000000000004C
:100BA800000000006CF700006CF70000DC9AFF1FE3
:100BB80001000A0001000000000000000000000021
:100BC8000000000000000000E8F60000E8F6000061
:100BD800349CFF1F000046000000000000000000D9
:100BE80000000000000000000000000004F8000001
:100BF80004F80000069CFF1F00000100010000002F
:100C080000000000000000000000000000000000DC
:100C180030F8000030F80000DE9AFF1F00001800CE
:100C280000000000000000000000000000000000BC
:100C38000400000000000000DCF70000DCF7000002
:100C4800108DFF1F0400500000000000000000008D
:100C580000000000000000000000000054F6000042
:100C680054F600006C9BFF1F00000100010000000B
:100C7800000000000000000000000000000000006C
:100C880000F7000000F700001E9BFF1F0000040093
:100C9800010000000000000000000000000000004B
:100CA8000000000010F8000010F80000769BFF1FFD
:100CB800000001000100000000000000000000002A
:100CC800000000004C8FFF1F64EF0000248BFF1F03
:100CD800388DFF1FAC8AFF1F648AFF1FE88DFF1F36
:100CE8000C8EFF1FEC8CFF1F948BFF1F24F000005D
:100CF8004CEF000018F00000ACEF00000CEF000013
:100D080088F00000B8EF0000000000007CF600004A
:100D180074F60000248AFF1F010011000000000083
:100D280000000000000000000000000000000000BB
:100D380068F6000074F600002C89FF1F01001E00F1
:100D4800000000000000000000000000000000009B
:100D58000000000084F7000084F70000F09BFF1FEC
:100D680000000A0001000000000000000000000070
:100D78000000000000000000E0F60000E0F60000BF
:100D8800269CFF1F00001D0000000000000000005E
:100D98000000000000000000308EFF1F388CFF1F8D
:100DA800808CFF1FDC8AFF1F708FFF1FC4EF0000BD
:100DB8005C8CFF1F008BFF1F00000000FCF7000089
:100DC800FCF70000049CFF1F000001000000000069
:100DD800000000000000000000000000000000000B
:100DE80018F7000018F70000869BFF1F000004009A
:100DF80001000000000000000000000000000000EA
:100E080000000000F4F60000F4F60000369CFF1F16
:100E180000007F000100000000000000000000004A
:100E28000000000000000000D4F60000D4F6000026
:100E3800589BFF1F00007F00010000000000000019
:100E4800000000000000000000000000F0F70000B3
:100E5800F0F70000FA9BFF1F0000010000000000EF
:100E6800000000000000000000000000000000007A
:100E780060F6000060F60000A69BFF1F000002005D
:100E88000100000000000000000000000000000059
:100E98000000000054F7000054F70000E49AFF1F18
:100EA80000007F00010000000000000000000000BA
:100EB8000000000016034E0075004500560049006A
:100EC80020004D00490044004900000084FA000059
:100ED80000000000E8030000000000000060064079
:100EE8003CFA0000000000000000000000000000C4
:100EF80000000000000000000000000000000000EA
:100F080000000000000000000000000000000000D9
:100F180000000000000000000000000000000000C9
:100F280000000000000000000000000000000000B9
:100F3800000000000000000084FA0000000000002B
:100F4800E803000000000000007006405CFA0000A2
:100F58000000000000000000000000000000000089
:100F68000000000000000000000000000000000079
:100F78000000000000000000000000000000000069
:100F88000000000000000000000000000000000059
:100F98000000000000000000000000000000000049
:100FA80000000000299A0000299A0000299A0000F0
:100FB800299A00000A040000B0A1FF1F65A30000E1
:100FC80065A3000065A3000065A3000065A30000F9
:100FD80065A3000065A3000065A3000065A30000E9
:100FE80065A3000065A3000065A3000065A30000D9
:100FF80065A3000065A3000065A3000065A30000C9
:1010080065A3000065A3000065A3000065A30000B8
:1010180065A3000065A3000065A3000065A30000A8
:1010280065A3000065A3000065A3000065A3000098
:1010380065A3000065A3000065A3000065A3000088
:1010480065A3000065A3000065A3000065A3000078
:1010580065A3000065A3000065A3000065A3000068
:1010680065A3000065A3000065A3000065A3000058
:1010780065A3000065A3000065A3000065A3000048
:1010880065A3000065A3000065A3000065A3000038
:1010980065A3000065A3000065A300000800000028
:1010A800FFFFFFFF1201100100000040C016850479
:1010B8007502010203010000180354006500650071
:1010C8006E00730079006400750069006E006F009F
:1010D80009027300020100C0320904000002010382
:1010E8000000072401000125000624020101000672
:1010F8002402020200092403010301020100092459
:101108000302040101010009050402400000000077
:10111800052501010109058302400000000005259D
:101128000101030904010002030000000921110163
:101138000001222100070581034000010705020381
:101148002000020006C9FF0904A15C7508150026E5
:10115800FF00954009758102952009769102950452
:101168000976B102C0000000040309040C03000062
:101178000000000000000000000000000000000067
:101188000000010000000000000000005495FF1F4F
:10119800BC95FF1F2496FF1F000000000000000000
:1011A8000000000000000000000000000000000037
:1011B8000000000000000000000000000000000027
:1011C8000000000000000000000000000000000017
:1011D8000000000000000000000000000000000007
:1011E80000000000000000000000000000000000F7
:1011F80000000000000000000000000000000000E7
:1012080000000000000000000000000000000000D6
:1012180000000000000000000000000000000000C6
:1012280000000000000000000000000000000000B6
:1012380001000000000000000E33CDAB34126DE653
:10124800ECDE05000B0000000000000000000000BC
:101258000000000000000000000000000000000086
:101268000000000000000000000000000000000076
:101278000000000000000000000000000000000066
:101288000000000000000000000000000000000056
:1015B8006892FF1F00000000000000009496FF1FC3
:1015C8009496FF1F9C96FF1F9C96FF1FA496FF1FD3
:1015D800A496FF1FAC96FF1FAC96FF1FB496FF1F83
:1015E800B496FF1FBC96FF1FBC96FF1FC496FF1F33
:1015F800C496FF1FCC96FF1FCC96FF1FD496FF1FE3
:10160800D496FF1FDC96FF1FDC96FF1FE496FF1F92
:10161800E496FF1FEC96FF1FEC96FF1FF496FF1F42
:10162800F496FF1FFC96FF1FFC96FF1F0497FF1FF1
:101638000497FF1F0C97FF1F0C97FF1F1497FF1F9E
:101648001497FF1F1C97FF1F1C97FF1F2497FF1F4E
:101658002497FF1F2C97FF1F2C97FF1F3497FF1FFE
:101668003497FF1F3C97FF1F3C97FF1F4497FF1FAE
:101678004497FF1F4C97FF1F4C97FF1F5497FF1F5E
:101688005497FF1F5C97FF1F5C97FF1F6497FF1F0E
:101698006497FF1F6C97FF1F6C97FF1F7497FF1FBE
:1016A8007497FF1F7C97FF1F7C97FF1F8497FF1F6E
:1016B8008497FF1F8C97FF1F8C97FF1F9497FF1F1E
:1016C8009497FF1F9C97FF1F9C97FF1FA497FF1FCE
:1016D800A497FF1FAC97FF1FAC97FF1FB497FF1F7E
:1016E800B497FF1FBC97FF1FBC97FF1FC497FF1F2E
:1016F800C497FF1FCC97FF1FCC97FF1FD497FF1FDE
:10170800D497FF1FDC97FF1FDC97FF1FE497FF1F8D
:10171800E497FF1FEC97FF1FEC97FF1FF497FF1F3D
:10172800F497FF1FFC97FF1FFC97FF1F0498FF1FEC
:101738000498FF1F0C98FF1F0C98FF1F1498FF1F99
:101748001498FF1F1C98FF1F1C98FF1F2498FF1F49
:101758002498FF1F2C98FF1F2C98FF1F3498FF1FF9
:101768003498FF1F3C98FF1F3C98FF1F4498FF1FA9
:101778004498FF1F4C98FF1F4C98FF1F5498FF1F59
:101788005498FF1F5C98FF1F5C98FF1F6498FF1F09
:101798006498FF1F6C98FF1F6C98FF1F7498FF1FB9
:1017A8007498FF1F7C98FF1F7C98FF1F8498FF1F69
:1017B8008498FF1F8C98FF1F8C98FF1F9498FF1F19
:1017C8009498FF1F9C98FF1F9C98FF1FA498FF1FC9
:1017D800A498FF1FAC98FF1FAC98FF1FB498FF1F79
:1017E800B498FF1FBC98FF1FBC98FF1FC498FF1F29
:1017F800C498FF1FCC98FF1FCC98FF1FD498FF1FD9
:10180800D498FF1FDC98FF1FDC98FF1FE498FF1F88
:10181800E498FF1FEC98FF1FEC98FF1FF498FF1F38
:10182800F498FF1FFC98FF1FFC98FF1F0499FF1FE7
:101838000499FF1F0C99FF1F0C99FF1F1499FF1F94
:101848001499FF1F1C99FF1F1C99FF1F2499FF1F44
:101858002499FF1F2C99FF1F2C99FF1F3499FF1FF4
:101868003499FF1F3C99FF1F3C99FF1F4499FF1FA4
:101878004499FF1F4C99FF1F4C99FF1F5499FF1F54
:101888005499FF1F5C99FF1F5C99FF1F6499FF1F04
:101898006499FF1F6C99FF1F6C99FF1F7499FF1FB4
:1018A8007499FF1F7C99FF1F7C99FF1F8499FF1F64
:1018B8008499FF1F8C99FF1F8C99FF1F9499FF1F14
:1018C8009499FF1F9C99FF1F9C99FF1FA499FF1FC4
:1018D800A499FF1FAC99FF1FAC99FF1FB499FF1F74
:1018E800B499FF1FBC99FF1FBC99FF1FC499FF1F24
:1018F800C499FF1FCC99FF1FCC99FF1FD499FF1FD4
:10190800D499FF1FDC99FF1FDC99FF1FE499FF1F83
:10191800E499FF1FEC99FF1FEC99FF1FF499FF1F33
:10192800F499FF1FFC99FF1FFC99FF1F049AFF1FE2
:10193800049AFF1F0C9AFF1F0C9AFF1F149AFF1F8F
:10194800149AFF1F1C9AFF1F1C9AFF1F249AFF1F3F
:10195800249AFF1F2C9AFF1F2C9AFF1F349AFF1FEF
:10196800349AFF1F3C9AFF1F3C9AFF1F449AFF1F9F
:10197800449AFF1F4C9AFF1F4C9AFF1F549AFF1F4F
:10198800549AFF1F5C9AFF1F5C9AFF1F649AFF1FFF
:10199800649AFF1F6C9AFF1F6C9AFF1F749AFF1FAF
:1019A800749AFF1F7C9AFF1F7C9AFF1F849AFF1F5F
:1019B800849AFF1F8C9AFF1F8C9AFF1F0000020059
:0419C800FFFFFFFF1F
:00000001FF
